:100000000C945F0F0C948E0F0C948E0F0C948E0F2B
:100010000C948E0F0C948E0F0C948E0F0C948E0FEC
:100020000C948E0F0C948E0F0C9459150C94296E11
:100030000C94A7700C945A6E0C948E0F0C94BC15F3
:100040000C9447150C948E0F0C9462760C946D757D
:100050000C948E0F0C948E0F0C948E0F0C948E0FAC
:100060000C941B710C9407160C94C86E0C945F7161
:100070000C948E0F0C948E0F0C948E0F0C948E0F8C
:100080000C948E0F0C948E0F0C948E0FBF17C41708
:1000900089178F17951795179517B517BA17BF17A3
:1000A000C417C917CE17D4170C42CC41D741E6412B
:1000B000EC41F041F5417C499249A049B549C34919
:1000C000D249E4490A4A334A414A674A854A934A2F
:1000D000A14AAF4AF968E768E168EA68EE68F26841
:1000E000E468F668FB688F72917294729972AC72D0
:1000F000BD72CD72D872EA72FC7201731A731D73ED
:100100002173237325732A732E733A733E734673D8
:100110004D7351735373577359735B735D7361738D
:1001200065736A736F73747379737E73204F6C6435
:100130002056657273696F6E20454550524F4D20B1
:100140002020434845434B2053455454494E475380
:100150002F43414C494200416C61726D73204469E8
:100160007361626C656400506C65617365205265F3
:10017000736574205377697463686573005468729B
:100180006F74746C65206E6F742069646C650052C6
:1001900065736574207468726F74746C650045458E
:1001A00050524F4D206C6F77206D656D004C4F4164
:1001B00044494E47006D537461636B206F666C6FEA
:1001C00077006D537461636B2075666C6F77004DBB
:1001D00045535341474500707265737320616E79D2
:1001E000204B657900507265737320616E79206BC6
:1001F000657920746F20736B697000034F46464128
:100200004253525573525525454C73454C2554481D
:1002100073544825414C73414C25503120503125B1
:10022000503220503225503320503325002D2D2DB3
:10023000004348002D2D2D20000450312020503245
:1002400020205033202048414C4646554C4C4359C1
:100250004331435943324359433350504D31505049
:100260004D3250504D3350504D3450504D3550500C
:100270004D3650504D3750504D384348312043484B
:1002800032204348332043483420434835204348F4
:1002900036204348372043483820434839204348D4
:1002A0003130434831314348313243483133434898
:1002B0003134434831354348313633504F53475634
:1002C0003120475632204756332047563420475670
:1002D00035204756362047563720002D2D2D2D002E
:1002E000000064281007030152554420454C452066
:1002F0005448522041494C2000414C455254000181
:100300000203040103020404020301040302014F77
:100310004E20004F464600544852525544454C45E5
:1003200049443049443149443241494C474541549C
:10033000524E535731535732535733535734535701
:100340003553573653573753573853573953574107
:10035000535742535743001B1E272D36394B4E63CC
:100360006C7278878D939CB1B4C6C9D2D8E1E4533E
:10037000706C6173680080400000000000000000A5
:10038000000000000000000000000000000000006D
:10039000000000000000000000000000000000005D
:1003A000000000000000000000000000000000004D
:1003B000000000000000000000000000000000003D
:1003C00000000080C0E0E0F0F8F8FCFCFCF8F8F871
:1003D000F04000000000008080800000000000006D
:1003E0000000000000000000000000000080C0C00D
:1003F000E0E0E0F0F0F0E0C00000000000C0F8FF36
:10040000FF9F878383838383838383838383838320
:10041000838383838383838383038380838383832F
:10042000838383838383838383838383838383839C
:10043000838383C3E3733F1F0000000080E0F0F874
:10044000FCFEFFFFFFFF7F3F1F1F0F0783C3E1E19C
:10045000E0E0C0000E1F3F7F7FFFF3E0E080000080
:10046000000000000000000080F0FCFEFFFFFFFF26
:100470007F3F0F0301010100000080F0FEFFFFC776
:10048000C1C1C1C1C1C1C1C1C1C1C1C1C1C1C1C15C
:10049000C1C1C1C1C1C101C1F0FEFF3F0F070F0DB6
:1004A0000D0D1D191919193131313171616161E178
:1004B000C1C1C18100000080E0F8FCFFFFFFFF2FF9
:1004C000170F038180C0E0F0F8FCFEFFFFFFFFFF85
:1004D000FF7F010000000000000001010307070E7C
:1004E0001E1C3870E0F0F8FEFFFF7F1F0F030001B5
:1004F00000000000000000000000000000000000FC
:1005000000000000000000000000000000000000EB
:1005100000000000000000000000000000000000DB
:1005200000000000000000000000000000000000CB
:100530000000000000007EFFFFFFFFFFFFFBF8FC54
:10054000FCFEFF7F3F1F0F07C3FFFFFFFFFFFF7F83
:10055000070000000000000000000000000000C0D4
:10056000E0F8FEFFFF7F1F0F1F3D7CF8F8F0E080F2
:10057000000000000000000000000000000000007B
:10058000000000000000000000000000000000006B
:10059000000000000000000000000000000000005B
:1005A000000000000000000000000000000000004B
:1005B0000000000000000000010101010103070725
:1005C000070301000000E0FCFFFFFFFFFF1F030027
:1005D00000000000000000000000C0F078DE2713DB
:1005E000090E0703000000000000000001030F7F58
:1005F000FFFC7878F8000000000000000000000018
:10060000808080808080808080008080008080006A
:1006100000000000000080808080808080808080DA
:1006200080808080808080800000000000000000CA
:1006300000000000000000000000000000000000BA
:1006400000000080F0FEFFFFFFFF3F0F01000000F1
:100650000000000000C0E0381E0F03000100000091
:10066000000000000000000000000000000000008A
:100670000000000303010000000000000000000073
:100680000E0E02020202020303000F0F000F0F08FA
:100690000808080808080F0F08080808080F0F00C6
:1006A0000000000F0F00000000000000000000002C
:1006B000000000000000000000000000000000003A
:1006C00000C0F8BFFFFFFF1F7F0100000000000017
:1006D0000000F0FCFF7F7830000000000000000008
:1006E000000000000000000000000000000000000A
:1006F00000000000000000000000000000000000FA
:1007000000000000000000000000000000000000E9
:1007100000000000000000000000000000000000D9
:1007200000000000000000000000000000000000C9
:100730000000000000000000000000000000003089
:100740001C070E0F07010000000000000000000061
:100750000000000000000000000000000000000099
:100760000000000000000000000000000000000089
:10077000000000000000000000204D4F443A2046D9
:1007800052534B592020203132382020002053561C
:100790004E3A20657239782D723830300054494D08
:1007A000453A2032313A32323A32320044415445ED
:1007B0003A2031302E30372E323031330056455208
:1007C000533A2056312E313134332D4D696B65004B
:1007D00056343D0756353D0E56363D0056313D07E1
:1007E00056323D0E56333D00096D706800537064FB
:1007F0003D096B7473204D61783D00416C743D0977
:100800006D2020204D61783D004C6F6E3D004C61A5
:10081000743D0041323D0041313D000A52504D00CF
:100820004675656C0022047C5E54546D0003457867
:1008300070457846466E654D656443727300115489
:100840004F54000153544B115354250001544D454E
:1008500011545357005354415400035B4D454E55BA
:100860005D20746F207265667265736800746D61D7
:10087000696E0F6D7300746D7231204A697474650E
:10088000720F757300746D72314C6174206D696EF6
:100890000F757300746D72314C6174206D61780F47
:1008A0007573005354415432004D6F646500496EB6
:1008B000742E204672736B7920616C61726D0043F7
:1008C000726F73735472696D00456E61626C65205E
:1008D00050504D53494D0042616E64476170005362
:1008E0007469636B5363726F6C6C00506F74536305
:1008F000726F6C6C00416C61726D205761726E6931
:100900006E67004D656D6F7279205761726E696E0A
:10091000670044656661756C742053770054687293
:100920006F74746C65205761726E696E67005370E6
:100930006C617368204E616D650053706C61736803
:100940002073637265656E004C69676874206F6E12
:100950002053746B204D76004C69676874206F6675
:1009600066206166746572004261636B6C696768DA
:100970007420696E76657274004C696768742073C0
:10098000776974636800466C617368206F6E2062DB
:10099000656570004265657020636F756E74646F85
:1009A000776E004D696E75746520626565700054E0
:1009B00068726F74746C6520726576657273650019
:1009C000496E616374697669747920616C61726DD6
:1009D000136D0042617474657279207761726E697B
:1009E0006E6700436F6E74726173740020486170AB
:1009F00074696320537472656E6774680020537065
:100A000065616B657220506974636800566F6C7520
:100A10006D65000A4265657065722020202050696E
:100A200053706B72202020204265657072566F698A
:100A30006365506953706B566F6963654D65676197
:100A4000536F756E642000536F756E64204D6F6434
:100A50006500065175696574204E6F4B6579207885
:100A600053686F727453686F7274204E6F726D208A
:100A7000204C6F6E672020784C6F6E6720004265B7
:100A800065706572004F776E6572204E616D65000E
:100A9000524144494F20534554555000036D6F64F3
:100AA000650A2520737263202073770043616C0010
:100AB0004D756C7469706C696572000363683163AD
:100AC000683263683363683400036F6666202B3DC9
:100AD000203A3D0007536C61766500000303030371
:100AE00000545241494E45520056455253494F4ECB
:100AF000005472696D2D202B0005204D656E752008
:100B00004578697420446F776E20202055705269B3
:100B1000676874204C65667400444941470012427E
:100B20004700414E4100034D4F5645205354494321
:100B30004B532F504F54530005534554204D4944B7
:100B4000504F494E5400035B4D454E555D20544F68
:100B50002053544152540043414C4942524154495C
:100B60004F4E000966726565004D4F44454C534534
:100B70004C00434F4C20446972656374696F6E008A
:100B800041494C20446972656374696F6E00454C3D
:100B90004520446972656374696F6E0053776173B1
:100BA000682052696E6700436F6C6C656374697688
:100BB0006500062D2D2D20202031323020202031BF
:100BC000323058202031343020202039302020206D
:100BD00020005377617368205479706500004845A0
:100BE0004C492053455455500020464D0020464D59
:100BF000300F52455441004D4F44455300547269E3
:100C00006D7300537769746368000003464C204D90
:100C10004F4445000152455441004175746F204CCA
:100C2000696D697473005432546854726967005472
:100C30007261696E657200452E204C696D6974732E
:100C40000003504F534E4547005368696674205364
:100C5000656C0050504D20317374204368616E0004
:100C60004C50342F4C5035202044534D326F6E6C15
:100C7000792044534D322F44534D580044534D2056
:100C8000547970650053656E64205278204E756DFE
:100C9000626572205B4D454E555D0050504D2046BB
:100CA000724C656E0D6D536563000B52784E756D19
:100CB000000434434820364348203843482031302C
:100CC00043483132434831344348313643480013B6
:100CD00075530011755365630050504D202020500E
:100CE000585820202044534D32202050504D31364A
:100CF0002050504D53494D0050726F746F00524553
:100D00005441313233004265657020436E740054A3
:100D100072696D2053770006457870202020457851
:100D200046696E6546696E6520204D656469756D1E
:100D3000436F61727365005472696D20496E630080
:100D4000542D4578706F00542D5472696D000A431C
:100D50006F756E7420446F776E436F756E74205597
:100D6000702020005472696767657242005472698E
:100D70006767657200566F69636520496E646578C0
:100D8000114D454E55004E616D6500000900010092
:100D90000000000000000602005345545550004476
:100DA00075706C69636174696E67206D6F64656CE2
:100DB0000044454C455445204D4F44454C00445556
:100DC000504C4943415445204D4F44454C004472DA
:100DD0005377320044725377310002576569676870
:100DE0007400024578706F00044452204869000482
:100DF0004452204C6F7700044452204D6964000037
:100E00004558504F2F445200012B2A52004D49584B
:100E10004552000320202020202020200044454C63
:100E2000455445204D49583F00035B4D454E555DA7
:100E30000B5B455849545D00035945530B4E4F0019
:100E40005072657373205B455849545D20746F2060
:100E500061626F7274004D6178206D69786572739C
:100E60002072656163683A2033320002536C6F77F9
:100E7000202055700002536C6F772020446F776EEE
:100E8000000244656C6179205570000244656C6114
:100E90007920446F776E0008416464202020202070
:100EA0004D756C7469706C795265706C6163652006
:100EB00000024D756C74707800025761726E696E35
:100EC0006700025377697463680043757276650042
:100ED0000D4469666600025472696D0002466C4DED
:100EE0006F64657472696D0002466978204F6666AA
:100EF000736574004F666673657400466D5472695D
:100F00006D56616C00025765696768740002536F23
:100F1000757263650045444954204D4958200003CB
:100F20002D2D2D783E30783C307C787C663E3066C6
:100F30003C307C667C633120633220633320633431
:100F400020633520633620633720633820633920DF
:100F50006331306331316331326331336331346350
:100F60003135633136000D4F6E00072D2D2D2D20AC
:100F70002020763E6F66732020763C6F66732020BB
:100F80007C767C3E6F66737C767C3C6F6673414EEC
:100F900044202020204F522020202020584F522033
:100FA00020202076313D3D7632207631213D76324B
:100FB0002076313E7632202076313C763220207603
:100FC000313E3D76322076313C3D76322054696D9B
:100FD000654F66660053000003435553544F4D2040
:100FE000535749544348455300064F4E2020202074
:100FF0004F4646202020424F54482020313553652B
:10100000637333305365637336305365637356616E
:101010007269626C00565300072038205365637371
:101020003132205365637331362053656373004E4C
:10103000756D62657220566F696365205377000095
:10104000000253414645545920535749544348459B
:101050005300434C454152204D49584553205B4D68
:10106000454E555D00205245544100014368616E74
:101070006E656C204F726465720054454D504C4152
:1010800054455300032D2D2D52746D45746D5474C9
:101090006D41746D52454E525544454C455448522D
:1010A00041494C503120503220503320633120636D
:1010B0003220633320633420633520633620633766
:1010C000206338206339206331306331316331323A
:1010D0006331336331346331356331360047560051
:1010E0000001474C4F42414C20564152530002539D
:1010F000656E7369746976697479000253776974EF
:10110000636800042D2D2D2D7673706441322020EC
:1011100000566172696F3A20536F757263650046BD
:101120004153204F666673657400437573746F6D29
:1011300020446973706C617900477073416C744D21
:1011400061696E00566F6C742054687265733D005F
:10115000034F464631323234303000416C74416CBA
:1011600061726D004E756D20426C61646573006D37
:10117000416820416C61726D00547852535349614B
:101180006C726D00000101010054454C454D455401
:1011900052593200013C3E00616C726D0001762DA7
:1011A0005641004120206368616E6E656C00034DFE
:1011B0006574496D700005467248756257534868FA
:1011C000690055737250726F746F00000101020262
:1011D000010254454C454D4554525900434F505916
:1011E000205452494D205B4D454E555D0000034C47
:1011F000494D4954530043560043555256455300F8
:101200005052455345540000435552564500032D56
:101210002D2D494E56004756005B4D454E555D20DD
:101220005748454E20444F4E450053454C45435486
:1012300000434F5059004D4F56450044454C4554CE
:1012400045004544495400494E5345525400434FCC
:101250005059004D4F56450044454C455445007B80
:101260004EE8291D27A2262426992B7D55DB59F906
:101270003330315A4C945ACB4AE753F25B4B27B484
:101280002C8E4B452912081200081C0808081C085F
:101290000000082200490022080000000000227F10
:1012A0002200000008220049002208000008220055
:1012B00049002208000000227F22000000000008F0
:1012C0002200490022080000081C0808081C080029
:1012D00001010100000002020202020202020202F7
:1012E00000020202020202020200000000000000EE
:1012F00002065761726E31205761726E3220436868
:101300006561702052696E672020536369466920C9
:10131000526F626F74204368697270205461646117
:101320002020437269636B74536972656E20416C4F
:101330006D436C6B5261746174615469636B2020FE
:1013400048617074633148617074633248617074CD
:1013500063330054696D65720041203D00032D2DFB
:101360002D59656C4F726752656400545245303197
:101370003241470052783D0054783D0020414243BD
:101380004445464748494A4B4C4D4E4F50515253A5
:101390005455565758595A6162636465666768695F
:1013A0006A6B6C6D6E6F7071727374757677787925
:1013B0007A303132333435363738395F2D2E0000EC
:1013C000010203FEFF0406080A0B0C0D0E0F23FD9D
:1013D000202425261D1E1F27F6F7F8F9FAFBFCF539
:1013E000042D2D2D2D41313D2041323D20525353AE
:1013F000495453534954696D3154696D32416C7489
:101400002047616C744773706454313D2054323D01
:101410002052504D204655454C4D6168314D616814
:101420003243766C7442617474416D70734D6168BF
:101430002043746F7446617356416363584163631C
:10144000594163635A5673706447767231477672B6
:101450003247767233477672344776723547767202
:1014600036477672374677617400537769746368DC
:10147000205761726E696E670067656E7772697476
:1014800065206572726F7200454550524F4D20467F
:101490006F726D617474696E6700426164204545C6
:1014A00070726F6D2044617461004D4F44454C2053
:1014B00020202020004D452020202020202020001A
:1014C000454550524F4D206F766572666C6F7700C0
:1014D000E2AEA1A6A4A2C02F258122AF0000000089
:1014E00000000000000000000000000000000000FC
:1014F000000000000000000000000000333B1F0F50
:1015000000000000C0C0C0C0C0C0C0C0C0C000005B
:1015100000000000000000000000000000000000CB
:1015200000000000183C3C18000000000000008093
:10153000C0E070381C0C0C0E070301000000000016
:101540000000FCFE87C3E377FEFC00000F1F3B3169
:1015500030381F0F00000C0EFFFF000000000000DD
:1015600030303F3F3030000000000C0E0783C3E7EF
:101570007E3C00003C3E3733313030300000030306
:10158000C3C3C3E7FE3C00003030303030391F0F9A
:101590000000C0E070381C0EFFFF000003030303CF
:1015A00003033F3F00003F3F33333373E3C3000087
:1015B0000C1C383030381F0F0000FCFEC7C3C3C7F7
:1015C0008E0C00000F1F383030391F0F000003034E
:1015D000C3E3733B1F0F000000003F3F000000000B
:1015E00000003CFEE7C3C3E7FE3C00000F1F39309C
:1015F00030391F0F00003C7EE7C3C3E7FEFC00004C
:10160000000030381C0E07030000183C3C18000096
:1016100000000000060F0F0600000000F0F8DCCE0E
:10162000C7C7CEDCF8F03F3F0000000000003F3F9E
:10163000FFFFC3C3C3C3C3E7FE3C3F3F303030307E
:1016400030391F0FFCFE0703030303070E0C0F1FA7
:101650003830303030381C0CFFFF030303070E1CFA
:10166000F8F03F3F303030381C0E0703FFFFC3C394
:10167000C3C3C3C303033F3F30303030303030305A
:10168000FFFFC3C3C3C3C3C303033F3F0000000046
:1016900000000000FCFE0703C3C3C3C7CECC0F1F6E
:1016A0003830303030303F3FFFFFC0C0C0C0C0C016
:1016B000FFFF3F3F0000000000003F3F000003032A
:1016C000FFFF03030000000030303F3F30300000D8
:1016D000000000000303FFFF03030C1C3830303808
:1016E0001F0F0000FFFFC0E0F0381C0E07033F3F54
:1016F000000103070E1C3830FFFF0000000000004F
:1017000000003F3F3030303030303030FFFF0E1CB3
:10171000F8F81C0EFFFF3F3F0000000000003F3FB5
:10172000FFFF3870E0C08000FFFF3F3F0000000176
:1017300003033F3FFCFE070303030307FEFC0F1FE9
:101740003830303030381F0FFFFFC3C3C3C3C3E787
:101750007E3C3F3F0000000000000000FCFE07034D
:1017600003030307FEFC0F1F383033371E1C3F33C3
:10177000FFFFC3C3C3C3C3E77E3C3F3F0000030773
:101780000E1C38303C7EE7C3C3C3C3C78E0C0C1C91
:101790003830303030391F0F03030303FFFF0303DA
:1017A0000303000000003F3F00000000FFFF0000B7
:1017B00000000000FFFF0F1F3830303030381F0F9F
:1017C000FFFF000000000000FFFF03070E1C383879
:1017D0001C0E0703FFFF000000000000FFFF0F1FAB
:1017E00038381F1F38381F0F0F1F38F0E0E0F0386F
:1017F0001F0F3C3E0703010103073E3C3F7FE0C053
:101800008080C0E07F3F000000013F3F01000000FA
:1018100003030383C3E3733B1F0F3C3E3733313075
:101820003030303000000000000000000000303098
:1018300030303030303030300000303030303070C8
:10184000E0C00C1E3F33333333333F3FFFFFC0E074
:1018500070303070E0C03F3F3030303030381F0FD4
:10186000C0E070303030303000000F1F3830303082
:1018700030381C0CC0E070303070E0C0FFFF0F1F2C
:101880003830303030303F3FC0E070303030307072
:10189000E0C00F1F3B33333333330303C0C0FCFEC0
:1018A000C7C303070E0C00003F3F0000000000000C
:1018B000F0F89C0C0C0C0C0CFCFC000133333333A3
:1018C000333B1F0FFFFFC0E070303070E0C03F3F80
:1018D0000000000000003F3F00003030F3F3000044
:1018E0000000000030303F3F3030000000000000BA
:1018F0003030F3F300000C1C383030381F0F00007C
:10190000FFFF0080C0E0703000003F3F03070F1C66
:101910003830000000000303FFFF0000000000005B
:1019200030303F3F30300000F0F03070E0E0707059
:10193000E0C03F3F0000030300003F3FF0F0C0E085
:1019400070303070E0C03F3F0000000000003F3FBB
:10195000C0E0703030303070E0C00F1F38303030B1
:1019600030381F0FF0F03030303030F0E0C03F3F03
:101970000303030303030100C0E0F0303030E0C094
:10198000F0F000010303030303033F3FF0F0C0E066
:1019900070303070E0C03F3F0000000000000000E9
:1019A000C0E0F0303030303000003031333333338A
:1019B000333F1E0C3030FFFF3030000000000000CD
:1019C0000F1F383030381C0CF0F000000000000011
:1019D000F0F00F1F383030381C0C3F3FF0F00000A3
:1019E00000000000F0F003070E1C38381C0E07033F
:1019F000F0F0000000000000F0F00F1F38381C1C51
:101A000038381F0F3070E0C08080C0E07030303850
:101A10001C0F07070F1C3830F0F08000000000009A
:101A2000F0F0000133333333333B1F0F30303030AD
:101A300030B0F0F0703030383C3E37333130303039
:101A400050085000000000000000006F0000070078
:101A50000700147F147F14242A7F2A12231308649A
:101A60006236495522500005030000001C22410047
:101A70000041221C0014083E081408083E08080013
:101A800050300000080808080800606000002010BE
:101A9000080402003E49453E0000427F400062517A
:101AA00049460041494936001814127F0027454530
:101AB00039003E494932000179050300364949366B
:101AC000000649291E000036360000005636000088
:101AD00008142241141414141441221408000201A1
:101AE00051090600060909067E0909097E7F494950
:101AF00049363E414141227F4141221C7F494949AB
:101B0000417F090909013E4149497A7F0808087F58
:101B100000417F41002040413F017F081422417F66
:101B2000404040407F020C027F7F0408107F3E410E
:101B300041413E7F090909063E4151215E7F091955
:101B40002946264949493201017F01013F40404071
:101B50003F1F2040201F3F4030403F631408146364
:101B600007087008076151494543007F4141000261
:101B7000040810200041417F00040201020440409B
:101B8000404040000102040020545454787F4844EF
:101B900044383844444420384444487F38545454EA
:101BA00018087E0901020C5252523E7F0804047844
:101BB00000447D40002040443D007F102844000048
:101BC000417F40007C041804787C08040478384481
:101BD0004444387C14141408081414187C7C080439
:101BE00004084854545420043F4440203C404020C2
:101BF0007C1C2040201C3C4020403C4428102844B1
:101C00000C5050503C4464544C4400083641000091
:101C1000007F000000413608000808221C08081C4C
:101C20002208084080080420100201536572766F74
:101C30002054657374004779726F20536574757012
:101C40000048656C6920536574757000456C657655
:101C50006F6E5C44656C746100562D5461696C0054
:101C6000537469636B7920542D43757400542D436C
:101C700075740053696D706C6520342D4348007392
:101C80001C6D1C601C591C4C1C411C361C2B1C0060
:101C900000891112239B322446AD573665BF744824
:101CA0008CC19D5AAFD3BE6CCAE5DB7EE9F7F881E3
:101CB00010080193331A22A5562C47B7753E64C904
:101CC0009C408DDBBF52AEEDDA64CBFFF976E802C3
:101CD000218B30100299132667AF763444BD554AE4
:101CE000ADC3BC588ED19F6EEBE7FA7CC8F5D983A3
:101CF000310A2091121803A7772E66B5543C45CBC4
:101D0000BD42ACD99E508FEFFB66EAFDD874C90482
:101D1000428D5316619F702004A9153227BB364CA3
:101D2000CEC5DF5EEDD7FC6888E1997AABF3BA8562
:101D3000520C4397711E60A1142805B3373A26CD83
:101D4000DE44CFDFFD56ECE9986089FBBB72AA0642
:101D5000638F7214409D512225AB343006B9174E63
:101D6000EFC7FE5CCCD5DD6AA9E3B8788AF19B8722
:101D7000730E6295501C41A3352A24B1163807CF43
:101D8000FF46EEDDDC54CDEBB962A8F99A708B0802
:101D90008481951AA793B62CC2A5D33EE1B7F04033
:101DA00008C919522BDB3A644EED5F766DFF7C89D2
:101DB0009400859BB712A6ADD224C3BFF136E0C113
:101DC000184809D33B5A2AE55E6C4FF77D7E6C0AB2
:101DD000A583B4188691972EE3A7F23CC0B5D142F3
:101DE00029CB38500AD91B666FEF7E744CFD5D8B92
:101DF000B502A499961087AFF326E2BDD034C1C3D3
:101E0000394A28D11A580BE77F6E6EF55C7C4D0C71
:101E1000C685D71EE597F42880A1913AA3B3B244B2
:101E20004ACD5B5669DF78600CE91D722FFB3E8D51
:101E3000D604C79FF516E4A9902081BBB332A2C592
:101E40005A4C4BD7795E68E11C680DF33F7A2E0E31
:101E5000E787F61CC495D52AA1A3B03882B1934672
:101E60006BCF7A5448DD59622DEB3C700EF91F8F11
:101E7000F706E69DD414C5ABB122A0B9923083C752
:101E80007B4E6AD5585C49E33D6A2CF11E780F28D9
:101E9000860A0C0D0B1028280728282828282884B3
:101EA00088979A111314151609181B122828282828
:101EB00005191C1D1E1F2720A12228284E7A112437
:101EC0001FBECFEFD0E1DEBFCDBF11E0A0E0B1E09B
:101ED000E2E9F6EF00E00BBF02C007900D92A034DC
:101EE000B107D9F71EE0A0E4B1E001C01D92AA330A
:101EF000B107E1F71EE1CEEBDEE100E006C022977C
:101F00000109FE010BBF0E94027BCC3BD10780E0A0
:101F10000807A9F70E9472780C94477B0C94000084
:101F2000E4E4F5E040E0842F806487B9369A36997E
:101F3000FECF24B135B1369A3699FECF84B195B132
:101F4000820F931F819391934F5F483061F70895FB
:101F5000853050F0883020F08E3020F482E00895F3
:101F600081E0089583E0089580E008952AE0829F4B
:101F7000C00111248D5F9D4F089525E0829FC0010F
:101F800011248D5B9C4F08958F929F92AF92BF92C8
:101F9000DF92EF92FF920F931F93CF93DF93C82F9F
:101FA000D62F5A01122FF02E822F8470D82E57FF71
:101FB00010C0882311F08CE101C08FE0212F4DE289
:101FC0006D2F9C2F981B892F0E945B64B194A19464
:101FD000B108212F2F214AE36D2F8C2F0E945B64C3
:101FE0006CE370E0C5010E94A77A4B015C01012FF0
:101FF00000619B0140E050E062E0E62E6D2F8C2FE7
:102000000E942A66DD2011F08AE101C08FE00F2DC9
:102010000061950140E050E092E0E92E6D2F8C0FB9
:102020000E942A66DF91CF911F910F91FF90EF9050
:10203000DF90BF90AF909F908F900895CF93DF93E4
:10204000D62FC22F206250E00E943A67C7FD09C018
:102050002C2F46E76D2F80915D0CDF91CF910C9472
:102060005B64DF91CF910895242F409102010C947D
:102070001E100F93022F24FF03C00F7E9CE201C0AD
:1020800094E2411104C024E04BED52E015C045300C
:10209000B0F4E0911D0594E0E99FF001112431971F
:1020A000E40FF11DE150FD4FE49194E0E99FA001A0
:1020B00011244C515D4F24E00E94ED640DC0941733
:1020C00028F02BEF240F49E352E004C02CED240F3D
:1020D00040EE53E10E940F650F9108950F93CF9347
:1020E000DF93C82FD62F022F411104C024E044E310
:1020F00052E00EC04A3010F086E101C081E18C0F41
:1021000050E0202F6D2F0E943A6722E041E352E019
:102110006D2F8C2F0E94ED64DF91CF910F91089568
:102120000F931F93CF93DF93D62FC42F022F16E068
:10213000180F442341F0463151F04A3E61F423E048
:1021400043E153E016C023E04DE252E012C023E029
:102150004FE053E00EC047FF04C041E20E945B64C1
:10216000C195C1504C2F440F4C0F50E0495E5C4F5D
:1021700023E06D2F812F0E94ED64DF91CF911F919D
:102180000F910895DF92EF92FF920F931F93CF93D9
:10219000DF93F82ED62F142FE22EC091F40181E0A8
:1021A0008217E0F14FE04C0F4F31D0F42C2F332742
:1021B00027FD309537FF03C0319521953109012F57
:1021C0004BEF51E06D2F8F2D0E940F65CF3FC4F56F
:1021D000212F41E26D2F8AEF8F0D0E945B6430C08A
:1021E00074E2D72EDC0E0AEF0F0D88E48D1520F077
:1021F0001C1674F441EF09C0212F4DE682E18F0DCA
:102200000E945B641C161CF44CED4C0F01C04D2D5C
:10221000212F6D2F802F0E94901012C082E0281372
:1022200013C0212F409164046D2F8AEF8F0DDF9131
:10223000CF911F910F91FF90EF90DF900C94901031
:10224000E11002C0C13069F3DF91CF911F910F916E
:10225000FF90EF90DF900895EF92FF920F931F93FE
:10226000CF93DF93790124E0629F800111240A5704
:102270001B4FD801EC91F0E0442311F0EE0FFF1F4B
:102280009F01DC010E945A7AE8012B81207C203CCE
:1022900059F424E630E040E050E00E94BB7AF701B8
:1022A00080818062808318C0E436F10578F4660F7F
:1022B000771F881F991F23E330E040E050E00E9421
:1022C000BB7AD7018C9180638C9306C02FEF30E0EE
:1022D00040E050E00E94BB7AC901DF91CF911F918D
:1022E0000F91FF90EF900895DF92EF92FF920F937E
:1022F0001F93CF93DF931F92CDB7DEB7D82EF62E64
:10230000842FA22F098394E0299F800111240A576A
:102310001B4F50E060E070E0F8019381907C9038B2
:1023200021F4EE2081F041E003C0EE2089F040E08E
:102330009E012F5F3F4F6A2F90E00E942C11AC014D
:1023400060E070E018C0440F551F661F771F13C070
:10235000903C89F4282F30E0AFEFB0E00E945A7A29
:1023600024E630E040E050E00E94BB7ABA01A901C7
:10237000898180628983F801838186FD14C0098187
:102380000062B5E0EB2E9A01AB016F2D8D2D0E94FE
:102390002A66298127FD1BC046E76F2D80915D0CC1
:1023A0000E945B6414C029816F2D8D2D0E943A67B5
:1023B000F8018381807C803C61F4298127FD0BC07A
:1023C00041E46F2D80915D0C0E945B6404C086E740
:1023D00003C080E201C081E40F90DF91CF911F9193
:1023E0000F91FF90EF90DF9008958C3038F4E82F34
:1023F000F0E0EE0FFF1FE455F84F22C08431C0F427
:10240000482F50E0DA01AA0FBB1FA65DBE4F2D91E9
:102410003C91803148F4FA01EE0FFF1FED50FB4F65
:1024200080819181281B390BC901880F991F08955C
:10243000843248F4E82FF0E0EE0FFF1FEC59F84F1C
:10244000808191810895853418F484520C94871FFB
:1024500080E090E008950E946E788111FCCF109288
:102460008E0C08950F931F93CF93DF938C01EB0194
:102470000E940B6424E049EF52E060E082E20E9497
:102480002365B80180E20E944365BE0188E20E9494
:10249000436565EE71E080E30E944365DF91CF9173
:1024A0001F910F910C94E1670F93462F50E0495E06
:1024B0005C4F00E023E060E10E94ED640F9108951D
:1024C0000F931F93CF93DF93082FC9EED1E01AE04B
:1024D000499124E0602F812F0E945B64155F1837BB
:1024E000B9F7DF91CF911F910F9108951F93CF936B
:1024F000DF93EC01162F0E940B64BE0188E10E945D
:102500004365111109C047ED51E068E38CE10E9479
:10251000496549EF52E002C04FEC51E024E060E031
:1025200082E20E942365DF91CF911F910C94E567B1
:1025300061E00E9476120C94E16770E0882399F0C4
:1025400090E0019725E0289FF001299FF00D1124CC
:10255000E60FF71FEE0FFF1FE255FB4F80819181C1
:102560008B509E4F0895FB01EE0FFF1FED5FFE4F56
:102570000190F081E02D8081992787FD9095089545
:102580001F93CF93DF93D82F162FC4E0DD2399F04C
:10259000612F8D2F0E949D129C01253F81E03807FD
:1025A00064F08BE0820F8D1710F08CE0820FC15029
:1025B00029F0D82FEBCFC0E001C0CD2F8C2FDF91B9
:1025C000CF911F910895CF93C62F0E94C0126C2FF8
:1025D000CF910C949D120F931F93CF93DF93EA0139
:1025E000062F10E08823B9F00E94C012882399F0CA
:1025F00090E0019725E0289FF001299FF00D11241C
:10260000E00FF11FEE0FFF1FE255FB4FC55FD140FA
:10261000D183C08317C0CE0183589F4F8B3F910554
:1026200040F01C161D061CF4CDE7D0E002C0C3E844
:10263000DFEFF801EE0FFF1FED5FFE4F0190F0811D
:10264000E02DC08386E0DF91CF911F910F910C9414
:10265000715F9F92AF92BF92CF92DF92EF92FF9203
:102660000F931F93CF93DF938C017B016A01922E0E
:10267000B090CB019B2D9F7D943439F080918A07D7
:10268000882309F487C0933439F4E801219683E163
:102690000E948A7385E00BC0953419F0923409F0DA
:1026A0007CC0E801219784E10E948A7384E00E9443
:1026B000C368811164C0E114F104E1F481E0C8163B
:1026C000D104C1F480E6B81619F08EE2B81212C037
:1026D00010928A07C1E00115110509F0C0E0D0E0B1
:1026E0008B2D0E9412698EE2B81206C081E08093A1
:1026F000BA0702C0A12C02C0AA24A3944091580199
:1027000050915901C41BD50B8091BA07833031F425
:102710008091D401C80FD11D87FDDA95CC16DD0656
:1027200044F48B2D0E94126983E10E948A73E601B2
:102730000AC0CE15DF053CF48B2D0E94126984E19E
:102740000E948A73E701C017D107B1F0209761F4A6
:10275000A11003C08B2D0E94026917FF02C083E104
:1027600001C084E10E948A73892D83700E94715F89
:1027700081E08093600113C01092600110C0CC27EB
:10278000DD27C01BD10B85E00E94126984E00E9406
:10279000126991CF953409F484CFE8018CCFCE0132
:1027A000DF91CF911F910F91FF90EF90DF90CF902D
:1027B000BF90AF909F900895552747FD509577277C
:1027C00067FD7095992787FD90950E9429130895BC
:1027D00022E00C94DC13462F22E060E00C94DC1322
:1027E00021E00C94DC13462F21E060E00C94DC1314
:1027F000E0916101F0E0EE0FFF1FEC59FE4F808188
:1028000091810895FC01A0916101B0E0AA0FBB1F66
:10281000AE59BE4FED93FC938FEB099587E10C9475
:102820008A73EBEBF7E0108E168A158A178A0895E3
:10283000EEE2FDE037A1303180F420A541E0420F07
:1028400040A7DF01A20FB11DA20FB11D8D939C9374
:10285000403108F010A63F5F37A3089590E08C5FE9
:102860009E4F0C94181490E00C9418148091350528
:10287000992787FD909509970C941814FC01909165
:10288000280580A191FF74C091A1882311F0946064
:1028900001C09B7F91A386A1813059F5C79A37A1CA
:1028A00021A1332321F181A541E0480F41A7DF0198
:1028B000A80FB11DA80FB11D8D919C9195A384A364
:1028C000403108F011A6315037A397FD02C031E125
:1028D00001C038E233A32C7F97FD226021A381A1A0
:1028E0008BBBC7988FE182A382E086A308952BBBA0
:1028F00048C081110CC0C79A81A1836081A38BBBA2
:1029000080915E0C8D3308F43CC086E02FC082308D
:1029100009F438C081A18BBBC79ABF9800C00000E2
:1029200000C086B38078BF9A96A1933049F488237B
:1029300029F083A1815083A3811123C084E016C0B4
:10294000943021F48823E9F083E00EC0953039F407
:1029500083A1815083A3811114C081E007C0963008
:1029600081F4882371F084E183A385E086A309C004
:102970009091250596FB992790F9891711F0C79A30
:102980000895C79808951BBA8FE18ABB00C099B318
:102990008FEF8ABBECECF1E08781882311F080E2B5
:1029A00002C0892F807E8483292F207C8081281774
:1029B00059F08074880F90783181891711F0315067
:1029C00001C03F5F3183208382819381891711F099
:1029D00083838183089590911D0590FD02C093E04B
:1029E0008927E82FF0E0EE0FFF1FE455F84F208114
:1029F0003181220F331FE32F131624F0332321F0EC
:102A0000E19502C080E801C080E0E8300CF0E7E02A
:102A1000F0E0E052FD4FE491EE2319F099E090933D
:102A20006C018E2B0895833021F0811103C083E067
:102A300001C080E0E82FF0E0EE0FFF1FEC5BFA4FE3
:102A4000808191810895FF920F931F93CF93DF931D
:102A5000F12CC0E0D0E08F2D0E941315092F10E05B
:102A6000C00FD11FF39484E0F812F5CFCE01DF91AF
:102A7000CF911F910F91FF9008950E9413152091FF
:102A80001F0520FF03C091958195910908957894C1
:102A90001F920F920FB60F9211248F9380914001D5
:102AA0008F5F809340018F910F900FBE0F901F900A
:102AB000189578941F920F920FB60F9211240BB6AF
:102AC0000F922F938F939F93EF93FF93F89487B771
:102AD0008F7B87BF78942091950180919701909189
:102AE0002805882359F090FF07C08091370E820F88
:102AF0008093370E87FF02C01B9A01C01B9891FF7D
:102B00002AC080915C08811126C0EEE2FDE086A11A
:102B1000823009F583A1882311F081501BC021A1C7
:102B2000C79A82A180FD09C02D7F84A195A196FD41
:102B30002260880F991F95A384A381E082278BBB15
:102B400081A3C79882A1815082A3811104C083E030
:102B500086A385E083A3F89487B7806487BF7894C1
:102B6000FF91EF919F918F912F910F900BBE0F903E
:102B70000FBE0F901F90189578941F920F920FB66A
:102B80000F9211240BB60F922F933F934F935F93A5
:102B90006F937F938F939F93AF93BF93EF93FF9325
:102BA00081B7845681BF83E991E00E94BF710E9482
:102BB00021690E94757780919B0C826080939B0CA9
:102BC000EBE0F1E08081815011F0808304C084E665
:102BD000808381E081838281815011F0828304C0EF
:102BE0008AE0828381E08383FF91EF91BF91AF916F
:102BF0009F918F917F916F915F914F913F912F9115
:102C00000F900BBE0F900FBE0F901F9018957894E9
:102C10001F920F920FB60F9211240BB60F922F93A3
:102C20003F934F935F936F937F938F939F93AF9354
:102C3000BF93EF93FF932091800030918100F8942F
:102C400080917D008F7D80937D00789480913E05FA
:102C500090913F05A901481B590BCA01969587958C
:102C600030933F0520933E059C01215A3F402F3D64
:102C70003E4220F481E08093410129C0E09141016E
:102C80002FEF2E0F283018F59C01215233402737A3
:102C90003540D8F421E02E0F20934101F0E0EE0FF3
:102CA000FF1FE05CFE4F9C012C5D354040912305E9
:102CB000465F429FC001439F900D11246AE070E07F
:102CC0000E94A77A7183608302C010924101F89438
:102CD00080917D00806280937D007894FF91EF91D8
:102CE000BF91AF919F918F917F916F915F914F9124
:102CF0003F912F910F900BBE0F900FBE0F901F9022
:102D0000189590E0880F991F8258924FFC01F89413
:102D1000808191817894089584E00E9481162091A9
:102D2000B3063091B406820F931F08959C0165E0AD
:102D3000359527956A95E1F7280F391FAC01440FA7
:102D4000452F441F550B241B350B892F990F990BC9
:102D50008595820F931F08959DE7980F9B3F88F0FC
:102D60008E57E82FF0E0EE0FFF1FE056FB4F8081FB
:102D700086171CF46083862F0895481714F4408347
:102D8000842F089544E66CE90C94AC1620911D053F
:102D9000217092E0921B21E0981320E0822F089589
:102DA0009091FA0194FD0C94C61680E0089549E2D2
:102DB000840290011124359527953595279587FD37
:102DC000815C86FB880F880B80F9A901481B51099B
:102DD00087FD5395CA0108955F926F927F928F92FB
:102DE0009F92AF92BF92CF92DF92EF92FF920F939A
:102DF0001F93CF93DF93982E742E45E0471508F468
:102E0000FCC0882309F4F7C056E1851721F08AEE4B
:102E1000981203C0F2C081E0F1C096E199150CF45C
:102E2000ECC0892D992787FD909597FF03C0919558
:102E3000819591098A3040F4825F0E94C368191419
:102E40000CF4DCC091E01DC08A50282F30E05901FD
:102E5000AA0CBB1C8501020F131F015C1B4FF8015C
:102E600082818F7009F4C9C0A90142595E4F6A017D
:102E700055E0751208C0F601908119140CF4B9C020
:102E800081E08927BBC0F801608051800E94A80FB3
:102E900081111BC08FEF860D0E94F5117C01F80196
:102EA000808185326CF0CBED8C2E880E6181882D6F
:102EB0000E94101FEC01882D0E94FA1E882E1BC054
:102EC000F80181810E94D7160CC0823071F48FEF17
:102ED000860D0E94F5117C01F801818181500E94CC
:102EE000F511EC018824839406C088248394C0E003
:102EF000D0E0E12CF12CF80182818F7090E0FC0190
:102F00003197EE30F10508F070C0EA5BFF4F0C948A
:102F1000FC7AF7FE34C0F194E194F10830C0F7FE7A
:102F200033C0F194E194F1082FC0D1E0D70D4D2FBB
:102F300060E0862D0E94EC16C82F4D2F60E0852D95
:102F40000E94EC16982FF80122812F70253031F461
:102F5000CC2309F44AC0811146C047C0263019F479
:102F6000C11141C029C09C2727C091E0EC16FD0685
:102F7000C9F422C091E0EC16FD06F1F413C091E013
:102F8000CE15DF05CCF00EC091E0EC16FD06A4F0E6
:102F900009C091E0EC16FD067CF404C091E0CE156A
:102FA000DF0554F490E008C0F501E658FE4F91812A
:102FB0009095991F9927991F8820B9F09923B1F00E
:102FC000F8018281982F907F61F082958F7089300F
:102FD0000CF08F5F41E0470D60E00E94EC16982FE7
:102FE00005C091E003C08110EBCF90E0F601908323
:102FF00044CF892F03C0862F01C080E0DF91CF919D
:103000001F910F91FF90EF90DF90CF90BF90AF9006
:103010009F908F907F906F905F90089540E060E068
:1030200080910A050E94EC16811114C08091530111
:1030300090915401892B71F410924E0D80915E0C89
:1030400090914305981751F0809343058EE29DE0DF
:103050000C943E1481E080934E0DF0CF08952091A2
:103060005301309154012115310511F021503109DE
:10307000882319F08091210501C080E090915201D0
:10308000992329F090912905891708F4892F4AEF8F
:10309000849FC0011124880F991F8217930708F499
:1030A000C90190935401809353010C940E18CF9250
:1030B000DF92EF92FF920F931F93CF93DF93809154
:1030C0005F0C9091600C90914205282F291B209352
:1030D00055018093420560E085E697E00E94453BFC
:1030E00080915501882309F490C2EBEBF7E08789C2
:1030F00080FF0DC0808D91E0980F908F943638F04E
:103100008356808F858996890196968B858B80E082
:103110000E94835F0E940B640E945768182F082F3B
:103120000F700650C091FB01C43021F0C33019F478
:10313000C4E001C0C8E0083008F09EC0D02ED6948C
:103140008091390580FF03C083E08D19D82E6D2D45
:10315000809154050E94C012C82E6D2D0E94E3126A
:103160009C01C1110CC0EC0197FF04C0CC27DD27E6
:10317000C81BD90BD595C795D595C795CF5F8091BD
:103180001D0580FBEE24E0F8F12C42E050E04E19E2
:103190005F098D2D90E04817590761F48091FA017D
:1031A00080FF31C281E0C4E090911F0590FF03C011
:1031B000C19501C080E0DD27C7FDD09500FF03C0A9
:1031C000C20FD31F04C0A9014C1B5D0BEA0120975D
:1031D00021F09D2F932797FF11C081110FC0232B42
:1031E00069F040E050E06D2D8C2D0E94EB12812F94
:1031F0000E94126986E10E948A733DC0CE01845804
:103200009F4F893F910580F4AE016D2D8C2D0E945A
:10321000EB12D7FF03C0D195C195D109D595C795BC
:10322000D595C7954C2F21C01C161D061CF44DE7E3
:1032300050E002C043E85FEF6D2D8C2D0E94EB1231
:10324000CE0183589F4F8B3F9105A8F4D7FF03C051
:10325000D195C195D109D7FD2396AE0155954795D6
:1032600055954795519541955109445C65E183E930
:1032700091E00E94747210E0E6E5F1E08091B807F9
:103280009091B90720813181281B390B37FF02C08B
:10329000215E3F4FB5E035952795BA95E1F72115A9
:1032A000310561F024813581281B390B37FF02C0BD
:1032B0002F5F3F4F35952795918380839583848336
:1032C00080911F0585FF02C020E030E03383228318
:1032D000CCECD1E02D818981821B8F3F09F480E005
:1032E00087FD8F5F85958887982F990F920F9D8313
:1032F000812B0E942F18E0916101F0E0EE0FFF1F7B
:10330000EE59FE4F8081918181529444B9F48885B1
:103310008823A1F02E81992787FD9095820F911D1A
:1033200027FD9A958E37910514F08DE705C08338F7
:10333000EFEF9E070CF483E88E83188680912505B5
:1033400087FF3BC080916D018823B9F180916C01AA
:103350008823A9F18091410587FD03C08F5F809389
:10336000410582E00E94EB14982F9F7789F020910D
:103370004105921720F510924105111120C0182F18
:103380001095111F1127111F83E6811B182F17C0DD
:1033900083E00E94EB14982F9F7789F020914105DC
:1033A000921768F410924105111109C0182F109559
:1033B000111F1127111F1C5902C010926C0181E0CE
:1033C00080936D0151EAE52E54E0F52EC0EAD4E079
:1033D0006AE0C62ED12CF7018081882309F462C0EF
:1033E000853068F40E94466AE82FF0E0EE0FFF1F78
:1033F000EF5FFE4F0190F081E02D808104C08530A9
:1034000021F48091D20188834DC08A30B8F4855070
:103410000E94466AE82FF0E0EE0FFF1FE655F84FD6
:103420008081918197FD079623E0959587952A9550
:10343000E1F78338FFEF9F07DCF015C08D30D0F443
:10344000E82FF0E0EE0FFF1FE056F84F80819181EA
:1034500097FD079603E0959587950A95E1F78338E0
:103460002FEF92072CF08D3791056CF28DE7CBCFC3
:1034700083E8C9CF8D31B0F4E82FF0E0EE0FFF1FE5
:10348000EE58F84F80819181B6010E94A77A633887
:103490004FEF74072CF06D3771051CF06DE701C01C
:1034A00063E8688352E0E50EF11C22968FEAE81685
:1034B00084E0F80609F08FCF8091E7019091E80150
:1034C000009761F060E00E9476120E946E78882377
:1034D00099F01092E8011092E7010EC01093CB0111
:1034E000E0916101F0E0EE0FFF1FEE59FE4F0190F9
:1034F000F081E02D812F09950E94E567C09165005C
:1035000083E991E00E94AB71882311F084E105C04A
:103510008091390E882321F081508093390E06C0A6
:1035200080916300869581708093380E8091380E6B
:103530008093E501882309F464C08091250585FD09
:1035400060C0CF7EC093650080915E0C8F71823029
:1035500009F054C08091520590915305AC01F4E0FC
:10356000440F551FFA95E1F797FD0796BC01E3E07C
:1035700075956795EA95E1F720910905332727FDB1
:1035800030952A5F3F4F629FC001639F900D729FED
:10359000900D1124840F951F20911F0526FD05C055
:1035A000609100017091010102C060EF70E00E9423
:1035B000937A80910201680F711D6F5F7F4F75953F
:1035C00067956093020180914005805F809340057C
:1035D000811114C080910805681780F4623370F07F
:1035E0006EE281E10E94907380911F0583FF06C007
:1035F00082E390E090935401809353011092520122
:1036000004C0C0619FCF80E0CFCDDF91CF911F91EB
:103610000F91FF90EF90DF90CF900895CF93DF93BD
:10362000C62F2091E601222329F09093E801809390
:10363000E70133C060E00E947612C11103C080919F
:10364000070501C089E10E94D26767E182E10E941B
:1036500090730E942B12D1E00E946E7881111DC0E0
:1036600080919B0C833019F4A89510929B0C40E03C
:1036700060E080910A050E94EC16811106C08091DD
:103680002105811102C0CC2329F0D0934E0D0E9458
:103690000E18E2CF10924E0DFACFDF91CF91089520
:1036A00090916101911103C0811106C017C0811171
:1036B00003C08FEF890F01C080E08093610187E133
:1036C0000E948A73E0916101F0E0EE0FFF1FEE5956
:1036D000FE4F0190F081E02D8EEB099460E082ECCA
:1036E00091E00C940E1BCF93DF93EC01809161016C
:1036F000843038F060E085EB91E0DF91CF910C945D
:103700000E1B87E10E948A73A0916101AF5FA093B5
:103710006101B0E0AA0FBB1FAE59BE4FCD93DC9341
:103720008FEBFE01DF91CF9109941F93CF93DF932D
:10373000C6EBD4E090E0888111E0190F882341F0B6
:1037400040E060E00E94EC16882311F0812F05C054
:10375000912F2A96143079F780E0DF91CF911F9155
:103760000895BF92CF92DF92EF92FF920F931F9333
:10377000CF93DF9380914001C2B7909140018913AC
:10378000F9CFD0E0D82BA0E1DA2E80916504D81AC9
:103790000E94900F1EE517B90E94C3140E9457188B
:1037A00017B9369A3699FECF84B195B104964091F7
:1037B00000015091010167E0649F9001659F300D09
:1037C0001124820F931FF3E096958795FA95E1F700
:1037D000909301018093000180919B0C833019F438
:1037E000A89510929B0C2091400182B790914001C6
:1037F0002913F9CF90E0922B8C1B9D0B2091B506DD
:103800003091B6062817390720F49093B6068093B6
:10381000B50680910E01882309F43CC180913C05D6
:1038200090913D05019690933D0580933C05CD2CEC
:10383000FFE0FC1508F476C00C2D10E0E801CC0F79
:10384000DD1FCA59DB4F8881E82EE294E694E7E059
:10385000EE22F98095E09E1550F0EAEFEF1538F46E
:10386000EF2DF0E0EE0FFF1FE055FD4FF0808F7160
:1038700009F456C040E060E00E94EC16B82E80913A
:103880000E010B521E4F823009F448C08E2D8570F8
:1038900051F4F8018081811106C0BB2021F08F2DE9
:1038A00090E00E9418148FEF8E0D823058F4F801CA
:1038B0008081813099F5B11031C0F2E0EF122AC059
:1038C000F39428C085E08E1550F4F80180818111B1
:1038D00025C0BB2019F189810E94DF1F1FC0F2E0C3
:1038E000FE15E0F4BB20D1F084E0E81631F095E05D
:1038F000E91631F066E970E005C06CE271E002C0E3
:1039000068E572E080913C0590913D050E94937AB4
:10391000892B21F48F2D90E00E941814F801B082B9
:10392000C39486CF5FE3E52E54E0F52E0AE711E05D
:10393000F701C2808C2D8F700E94A80F8330E1F5B3
:10394000F801C081D181209771F4F701C081C7FDD2
:1039500006C0C095FAE0CF02E001112419C0DD27AE
:10396000C7FDD09515C0D7FF12C0219689F4F70185
:10397000C181C7FD06C0CF5FFAE0CF02E00111248C
:1039800006C0DD27C7FDD095C095D09501C0219711
:103990008C2D807F71F08C2D82958F7089300CF08A
:1039A0008F5F40E060E00E94EC16811102C0CFEF13
:1039B000DFEFF801D183C083F3E0EF0EF11C0E5F5F
:1039C0001F4F81E00239180709F0B2CF10920E01A3
:1039D0008091D604882309F45DC040E060E08091C6
:1039E000D7040E94EC16882309F454C080913B054B
:1039F000882319F0815080933B0580913B0581110C
:103A000049C08091D604813069F487E20E94811612
:103A1000EC016091D8046230C8F070E00E94A77A8F
:103A2000EB0114C081E00E948116805891099C012D
:103A30002E5F3F4F2530310510F480E090E020915B
:103A4000D804289FE001299FD00D11242097C9F0A8
:103A5000D7FF06C0D195C195D10946E462E202C004
:103A600046E461E283E991E00E947472CB34D105AF
:103A700054F0CD37D1054CF0CF3AD10544F484E071
:103A800007C080E005C088E003C086E001C082E096
:103A900080933B0580910C01882309F415C1809126
:103AA000080E882309F44FC08091F501807CD9F07D
:103AB000803819F4C0E9D1E002C0CAE7D0E00E9422
:103AC0008C166AE070E00E94A77ACB012091F50184
:103AD00023FD03C025FD0E94D81EC817D9071CF47A
:103AE00081E00E948A7300E01CED90E0C0E0D0E02D
:103AF00080915F0D0817B0F4E02FF0E0E05AF24F2C
:103B00008081C80FD11D811708F4182F911107C0AB
:103B100020916304821720F48DE10E948A7391E062
:103B20000F5FE6CFCE0165E070E00E94937A70935C
:103B3000C90D6093C80D1C3D31F0812F90E090932A
:103B4000C50D8093C40D8091090E81110BC0809129
:103B50003A058F5E982F977F903608F044C0909377
:103B60003A0544C006E814E0C0E0D0E0F8018081E6
:103B7000882389F1FE01EE0FFF1FEE0FFF1FE757AD
:103B8000FB4F80818295869586958370833019F5E9
:103B900080918F048823F9F08C2F825F0E94811618
:103BA00036E0959587953A95E1F720918F0430E0BE
:103BB0008217930784F08091280581FF05C081E377
:103BC00090E00E94181407C046E46091900483E9D5
:103BD00091E00E94747221960C5F1F4FC230D10594
:103BE00009F4B5CFC3CF877080933A05C9EED1E011
:103BF000F12CFD1409F45FC08E0103581D4FF8012C
:103C00008081982F907C9034C9F4880F880F40E011
:103C100060E0859585950E94EC16882379F0809167
:103C2000280580FF05C0FE01E258FD4F608101C0FC
:103C300061E046E483E991E00E947472F8018081BA
:103C4000982F907C9038A1F520913A05880F880F25
:103C5000859585958731E4F0992787FD909547975D
:103C60008130910539F08230910541F0892B01F5C1
:103C7000237001C0207F21111BC003C02770223098
:103C8000B9F4FE01E258FD4F80810E94DF1F10C091
:103C900020FD0EC040E060E00E94EC16882341F059
:103CA000FE01E258FD4F8081805890E00E94181478
:103CB000F39422969ECF10920C0180916C01882380
:103CC00019F0815080936C01DF91CF911F910F917A
:103CD000FF90EF90DF90CF90BF9008951F93CF9308
:103CE000DF93D82F162FC42FB9010E9443651123EB
:103CF00029F06FE08C2F0E94EB13C82F4C2F50E05F
:103D0000212F6D2F80E60E943A678C2FDF91CF9193
:103D10001F910895813649F40E94126981E00E9442
:103D2000501B8AE59CE40E94731B66E57EE080E1FF
:103D30000E94436560E47EE080E20C944365FF925C
:103D40000F931F93CF93DF93182FF62E0AE08AE08C
:103D5000189FE0011124CD5FDD4F2FE130E0211BE2
:103D60003109029FA001039F500D1124BE01CE0115
:103D70000A960E94157BFF2049F0BE016A50710926
:103D80004AE050E0CE010E94157B0AC0FE0111926C
:103D90000A95E9F78091F8078883898384E68A8306
:103DA0001093FA07DF91CF911F910F91FF90089523
:103DB0009C01220F331F280F391F959587959595E4
:103DC0008795280F391F9595879595958795959592
:103DD0008795820F931F0895429643E7489F90016D
:103DE000499F300D1124C901E6E095958795EA9524
:103DF000E1F70895E82FF0E0E053FD4EE491EE2363
:103E000069F0E13021F48091090E811107C081E051
:103E10009091080E911103C080E0089581E008950B
:103E2000E82FFF27E7FDF095E154FC4EE491262FA3
:103E3000332727FD3095C90183589F4FEC3009F493
:103E40004AC09CF4E43021F14CF4E53F09F454C03D
:103E50000CF45CC0EE5FE230C8F00895E630C1F0CB
:103E60000CF454C0EA30FCF50895E43209F43FC084
:103E700044F4EE300CF44AC0E031CCF1E332C9F145
:103E80000895E732B4F1E732E9F108952AE024C059
:103E9000803491059CF0880F991F80549109813CD2
:103EA000910564F0880F991F805C9109813C51E075
:103EB000950724F0880F991F885E91402AE0AC0195
:103EC000249FC001259F900D11242091F50125FF0D
:103ED0001DC00C94D81E24E6AC01249FC001259F70
:103EE000900D11240895C901815A9F4F089522E32E
:103EF000F3CF880F991F0895F3E0880F991FFA9563
:103F0000E1F708955AE06502C00111240895CF93A6
:103F1000DF93E82FFF27E7FDF095E154FC4E8491F5
:103F2000853FC9F486E20E948116EC0180E20E947E
:103F30008116D595C7959C0135952795C29FC001DF
:103F4000C39F900DD29F900D112469E170E00E94F3
:103F5000A77ACB0131C08D3F54F4E82FEE0FFF0B51
:103F6000EC54FB4F8081992787FD909525C08F3FAA
:103F700009F044F48E3F84F48D3FD1F48091020126
:103F800090E01AC0843081F0833291F483E20E9481
:103F90008116880F991F10C0E82FEE0FFF0BE15418
:103FA000F84F8389948908C0DF91CF910C948C16C7
:103FB000DF91CF910C948116DF91CF910895CF922C
:103FC000DF92EF92FF920F931F93CF93DF931F9295
:103FD000CDB7DEB7082F19820E94871F7C01802F82
:103FE0000E94FA1E811105C08AE30E94331411E079
:103FF00001C010E0E02FFF27E7FDF095E154FC4EF3
:1040000064916230F4F467FF48C06D3F44F4663F4A
:10401000D4F5653F09F088C060E04BE394C06D3F84
:1040200009F485C06CE370E0C7010E94A77A6B01B8
:104030007C0146E260E0C6010E94997360E045E3BE
:1040400082C0603209F475C054F4643009F444C08D
:104050000CF46AC06A50623008F45DC065C0673213
:104060003CF465320CF063C0633209F465C05CC097
:10407000673209F059C0C7016AE070E00E94A77A70
:104080007B0161E052C0E62FEE0FFF0BEC54FB4FBB
:10409000E080FF24E7FCF09447C084E06802F00170
:1040A0001124EA57FB4F038102950695069503708C
:1040B000D08041E0023009F040E09E012F5F3F4F89
:1040C000C7010E942C117C01033099F1013061F18C
:1040D00083E68D1588F52BC09091F501892F8072AC
:1040E00093FF03C0882349F006C0882331F0C7013D
:1040F0000E94D81E7C0148E101C048E388EEE81622
:1041000083E0F806E4F0C7016AE070E00E94A77A55
:104110007B0160E018C08091F50185FF12C0C701E6
:104120000E94EC1E7C010DC060E040E00CC061E02C
:1041300004C061E043E307C062E044E204C061E020
:1041400002C060E04FE2111103C0C7010E949973E1
:104150000F90DF91CF911F910F91FF90EF90DF9023
:10416000CF9008959F92AF92BF92CF92DF92EF923D
:10417000FF920F931F93CF93DF93C82EB62EF42E8A
:10418000E901102FAE2C8E2D8170982EE0FE15C007
:1041900000E021E0240F40EE53E18C2D0E940F65DA
:1041A00012FD04C0E8E1DE2EDC0C08C07CE1D72E55
:1041B000DC0C88EFB80E0CE002C0DC2C06E08A2D87
:1041C0008870E82EA3FC1F7BEF2DFF27E7FDF095FD
:1041D000E154FC4EF49086E0F81609F475C08F1592
:1041E000C4F08FEF8F1564F08EEFF816CCF585EFE5
:1041F000F81609F4A4C08DEFF81609F482C084C043
:1042000081E08F150CF042C084E0F81609F45CC020
:104210007BC083E2F81609F472C08F1574F08AE04F
:10422000F8160CF471C08BE08F150CF042C080E2E0
:10423000F8126AC0106201E468C085E2F8160CF456
:1042400063C086E28F150CF05CC087E2F8125CC098
:104250001062CE016AE070E00E94A77AEB0154C0C0
:1042600012FD02C08CEFD80E992011F08AE0D80E12
:104270001770012F212FAE016B2D8AEF8D0D0E943B
:10428000C40F03E30F0D8AEFC80E48C0912F90684A
:104290004C2FEE2019F08DE38C0D02C08D2D801B6C
:1042A000EE24E394092F2F2D6B2D0E947411082FFB
:1042B00035C08091F50185FF44C0CE010E94EC1EFF
:1042C000EC01D01A06E421C08091F50185FF07C0FA
:1042D00083FD07C0CE010E94D81EEC0102C00DE68E
:1042E00001C006E6C83E83E0D80714F410620DC092
:1042F000CE016AE070E00E94A77AEB0106C010636D
:1043000001C0106206E701C000E2EE20E1F08DE39B
:104310008C0D212FAE016B2D0E943A678A2D86707D
:10432000A1F0A2FE04C08AE08C0D1B7F02C0809128
:104330005D0C212F402F6B2D0E945B6406C007E7A8
:10434000E4CF03E4E2CF8D2DE4CF802FDF91CF9136
:104350001F910F91FF90EF90DF90CF90BF90AF90A3
:104360009F9008950F931F93CF93DF93C82FD62F5D
:10437000042F122F46E152E10E94236540E3400FD3
:10438000212F6D2F8CE08C0FDF91CF911F910F911A
:104390000C945B64DF92EF92FF920F931F93CF9385
:1043A000DF93182FF62EC42FD22EDE2DD370A1F05E
:1043B0008091CB01803881F48DE7840F8B3F40F0F2
:1043C000E42FF0E0EE0FFF1FEC55FC4FC08101C061
:1043D000CEE782E00E94715F8DE78C0F2E2D8B3F20
:1043E000A0F043E84C0F6F2D8EEE810F0E94B2219A
:1043F000DD2309F122E042E850E06EE770E08C2F07
:1044000090E00E942913C82F16C04C2F552747FD56
:1044100050956F2D812F0E943A67DD2361F0402F68
:104420006D2D8C2FDF91CF911F910F91FF90EF9009
:10443000DF900C94E8138C2FDF91CF911F910F9197
:10444000FF90EF90DF900895CF93DF939EE0899FD8
:10445000E0011124C751DE4FFE01EA54FE4F40E057
:1044600060E080810E94EC16882359F0C954DE4F29
:1044700040E060E088810E94EC16811104C081E078
:1044800003C080E001C082E0DF91CF910895EF92F8
:10449000FF920F931F93CF93DF93F82EE62EC42F36
:1044A000D42FD695062F0D1B182F1D1B602F812F83
:1044B0000E94DE656D2F6E0D4C2F812F0E94DB65F3
:1044C0004C2F602F8D2F8F0D0E94DE654C2F602F9B
:1044D000812FDF91CF911F910F91FF90EF900C945E
:1044E000DB6521E0AC0160E080E00C9423651F9364
:1044F000CF93DF93182FCFE0D1E083EA98E00E94BA
:1045000071221136B1F068F41036D1F48FEF888340
:1045100019821092B6061092B50687E10E948A733E
:104520000FC0123619F0133621F00AC08CEE92E259
:1045300002C081E294E4DF91CF911F910C940214A8
:1045400064E978E088E00E9443654981469550E03F
:1045500068E084E50E94496765E878E080E10E94B0
:1045600043654881469550E060E184E50E944967D3
:1045700066E778E088E10E944365498150E08881E0
:10458000481B510957FF02C04F5F5F4F5595479534
:1045900068E184E50E9449676DE678E080E20E9468
:1045A00043658091B5069091B60629E1289FA00148
:1045B000299F500D1124569547955695479520E310
:1045C00060E284E50E943A676AE578E088E3DF917B
:1045D000CF911F910C9443650F931F93CF93DF935B
:1045E000182FCBEBD7E085E598E00E9471221136B9
:1045F00078F0133628F0133659F487E792E202C0B8
:1046000081E294E4DF91CF911F910F910C940214F9
:104610006CE478E088E00E9443654A815B8100E0B9
:1046200020E068E08AE20E94C40F4C815D8120E0B6
:1046300068E08EE40E94C40F63E478E080E10E94A9
:1046400043654E815F8120E060E18AE20E94C40FF1
:104650004885598514E0569547951A95E1F720E06D
:1046600060E18EE40E94C40F6EE378E080E00E9477
:1046700043654881598120E060E08EE40E94C40FC8
:104680004EE76CE382E00E94DB6543E26CE185E08B
:104690000E94DE65CBE043E06BE38C2F0E94DE6579
:1046A000CA5FC338C1F71091B8068091B706893741
:1046B00010F4C0E001C0C12FD6E00CE3EC2FF0E015
:1046C000E754F94F4081602F641B8D2F0E94DE65F7
:1046D000CF5FC83708F0C0E0C11719F0DF5FDE37E1
:1046E00069F7DF91CF911F910F91089591E021110A
:1046F00001C090E0442319F04FE053E002C043E1D1
:1047000053E0292F0C9423650F9301E0211101C080
:1047100000E0242F4EE052E10E940F650F910895B2
:104720007F928F929F92AF92BF92CF92DF92EF9241
:10473000FF920F931F93CF93DF93EC01162FD42E8C
:104740004901B09064074091B4075091B50720919A
:10475000B6073091B707E6E5F1E086819781841BC3
:10476000950B97FDCF96A6E095958795AA95E1F7CD
:10477000682F8093870780859185821B930B97FD17
:10478000CF9676E0959587957A95E1F7982F809367
:104790008507662311F057834683992311F03187EB
:1047A000208780918607811104C080911F0585FFB5
:1047B00006C01092870710928507109286072091F5
:1047C0008707211108C080918507811104C082816B
:1047D0009381892B61F0809121053AEF839FC0017D
:1047E0001124880F991F90935401809353018114D1
:1047F0009104B1F18881811197C18091BA07882312
:1048000009F49DC1813009F4ACC12111B1C1153643
:1048100009F4D1C1143609F4D8C177247394809176
:10482000BA07811102C082E0782E402F50E0272D78
:1048300060E08FE70E943A670A3008F47EC10FE615
:10484000272D4FE260E0802F0E945B644D2D50E0E9
:104850004F5F5F4F272D60E08FEF800F0E943A6718
:10486000E114F10451F098818C2D9C1508F4892FE6
:10487000F701E80FF11DE49101C0E0E08091BA0773
:10488000813081F58091D40118166CF4BE1610F4B5
:10489000B39411F588818A1518F48F5F888301C05D
:1048A0001882B12C19C08823B9F0B11014C08881C6
:1048B000882319F08150888301C0A882E114F10493
:1048C00059F098818C2D9C1508F4892FF701E80F79
:1048D000F11DB49001C0BA941092D4011E3249F473
:1048E00083E005C0833029F41E3219F481E08093FF
:1048F000BA07E114F10451F098818C2D9C1508F44D
:10490000892FF701E80FF11D549101C050E080910B
:104910008A07811145C080918507882301F148816C
:10492000481B47FD40E08A2D90E0242F332727FDC8
:104930003095281739070CF04A2D4883E114F1040B
:1049400059F0C41608F44C2DF701E40FF11DE49161
:10495000EB1518F4BE2E01C0B12C109285072881EA
:104960002223F1F0809187078823D1F0B81AB7FC91
:10497000B12C8B2D992787FD9095E114F10479F0E6
:104980003C2D2C1508F4322FF701E30FF11DE491B3
:104990002E2F30E0821793071CF0BE2E01C0B12CE1
:1049A000103669F190F4123409F473C028F411320E
:1049B000A9F11E3221F197C0143409F446C008F45D
:1049C00076C0153409F451C08EC0153609F451C0B3
:1049D00040F4133609F46EC0D8F5123609F45CC001
:1049E00082C01E38C1F01F3B31F0113809F07BC086
:1049F00010928A0721C0188210928A0738C08881D5
:104A0000882309F470C081E090918A07911180E0B9
:104A100080938A0768C08EE80E94126980918A0795
:104A2000882319F010928A075EC08881882311F0CC
:104A3000892831F41092BA0780E00E94501B53C0BD
:104A400087E10E948A7318824EC0B51609F44BC0E4
:104A5000EF2809F448C080918A07811144C0B51637
:104A600010F4B39411C0B12C0FC0B11002C0B12C1E
:104A70003AC0EF28C1F180918A07811134C0BB2070
:104A800011F0BA9401C0B52E552369F11092CB01F3
:104A90002AC088818A1539F180918A07811123C043
:104AA00088818A1510F48F5F0DC018820EC088812E
:104AB0008823C9F080918A07811115C088818823D5
:104AC00019F08150888301C0A882E114F10479F2C1
:104AD00088818C1508F4C82EF701EC0DF11DE490C7
:104AE000EB1408F4BE2C80918A0781110AC021E0E2
:104AF0008091580190915901892B09F420E0822F6F
:104B000001C081E080938907B0926407DF91CF9163
:104B10001F910F91FF90EF90DF90CF90BF90AF90DB
:104B20009F908F907F90089580918A07811103C094
:104B300081E08093BA07712C72CE05E781CE809117
:104B4000D401181624F0882319F015E601C014E6E4
:104B50001092D4011E3209F058CE81E08093BA073A
:104B600005C01E3209F051CE1092BA0710E04DCEAA
:104B700080918A0781114BCEED2DE21BE7FDE0E02D
:104B8000202F30E08E2F992787FD9095821793076D
:104B900014F0EFEFE00FFF27E7FDF0958D2D90E08B
:104BA000E817F90729F0EE0FFF1FE80DF91D1EC0E9
:104BB000109287072CCED11001C0D02EF401ED0D3C
:104BC000F11DED0DF11D329711C02D2D30E0802F1C
:104BD00090E00197281739071CF411E01D0D01C062
:104BE00010E0810E911C810E911CF401859194912D
:104BF000DF91CF911F910F91FF90EF90DF90CF90B9
:104C0000BF90AF909F908F907F900C940214AF92C2
:104C1000CF92EF92FF920F93AE2CC12CE12CF12C8E
:104C20000E9490230F91FF90EF90CF90AF90089546
:104C3000EF920F93E42E00E020E030E040E00E948D
:104C400007260F91EF900895BF92CF92DF92EF92D7
:104C5000FF920F931F93CF93DF93C82F82E29BE0C5
:104C60000E947122EE24E39406E02FE532E144E055
:104C70006C2F81EE97E00E940726B090E10710921A
:104C80006D01CCEAD7E010E000E0C12CB4E0DB2EEF
:104C9000E12CF12C41E4612F88E10E94EA6441E3B8
:104CA000400F612F8EE10E94EA64802F0E9413154D
:104CB000AC01612F8AE20E944C65073081F0A88127
:104CC000B98124E630E00E94697AA70196010E942A
:104CD000DD7AA901612F8AE50E9449670AC081E057
:104CE000B81611F040E201C041E2612F8AE50E944E
:104CF00034100F5F185F2296083061F66EE17BE09A
:104D000088E20E944365409100015091010160E3F7
:104D100088E70E94496781E0B8120AC0B09286070E
:104D20004FE761E8809109050E94F013809309051F
:104D3000DF91CF911F910F91FF90EF90DF90CF9077
:104D4000BF900895EF920F931F93CF93DF93C82FD7
:104D500089E19BE00E947122E12C06E02FE532E11F
:104D600043E06C2F80EE97E00E940726D0E0C0E081
:104D7000C43018F018EF1D0F01C01D2F8FE08C0FED
:104D80000E94C368082FCF5F20E04C2F612F8AE27A
:104D90000E94901040E3400F202F612F84E40E9476
:104DA0005B64D85FC93021F7D8E3C0E08C2F0E9444
:104DB000C368182F00E02C2F49EF5AE06D2F80E0D8
:104DC0000E940F6540E3410F212F6D2F80E20E946A
:104DD0005B64CF5FD850C63049F741EF5AE068E1D5
:104DE00084E50E94496516E0C0E2D0E02D2F45E839
:104DF00052E16C2F84E50E941664812F0E94C368E3
:104E000040E3480F282F6C2F8CE60E945B6481E002
:104E1000810F0E94C36840E3480F282F6C2F88E75A
:104E20000E945B64DF5FC85F1E5FD430F9F6DF91DC
:104E3000CF911F910F91EF900895EF920F93CF9321
:104E4000C82F89EE9AE00E947122E12C06E02FE53E
:104E500032E142E06C2F8FED97E00E9407266DE86B
:104E600077E080E10E9443656DEB77E088E10E9486
:104E700043656CEA77E080E20E9443656DE977E084
:104E800088E20E94436569E777E080E3CF910F9164
:104E9000EF900C9443652F923F924F925F926F92E6
:104EA0007F928F929F92AF92BF92CF92DF92EF92BA
:104EB000FF920F931F93CF93DF9300D000D000D0C9
:104EC000CDB7DEB7D82E82ED91E10E94712247E086
:104ED000A42E56E0C52E6BECE62E61E1F62E0DE019
:104EE0002BE632E149E06D2D81EF97E00E9490239F
:104EF0006090F107109164078EED8D0D843028F4D9
:104F000080918A0781110E943D7880918A078823C9
:104F100019F022E0298302C031E0398362EC71E1AB
:104F200088E00E9443658091F50183FB882780F922
:104F300091E069120DC011110BC061E00E94EB13EA
:104F40009091F50180FB93F99093F50101E001C088
:104F500000E0282F46EB51E168E08CE30E940F65EA
:104F60008091F50185FB882780F9E1E06E120DC084
:104F7000113059F461E00E94EB139091F50180FB30
:104F800095F99093F50101E001C000E0282F4EEA69
:104F900051E168E080E60E940F6526E834E03E8338
:104FA0002D839CEE892E9DE0992E31E33A8322E0F9
:104FB000722E30E1F32E898180688C8363EA71E17F
:104FC0008F2D0E9443659A8191539B834A816F2D57
:104FD00086E00E94EA64671004C0111102C00C81CF
:104FE00001C000E8E12C2B81ED81FE8140816F2D15
:104FF00080E60E947411EE24E39400E82B81F40112
:1050000040816F2D8EE70E947411671002C011302D
:1050100011F000E001C00981ED81FE81238122951C
:105020002695269523704DE951E16F2D80E60E946B
:105030000F65671031C080918A07811106C0809189
:10504000580190915901892B39F11123B9F0113090
:1050500019F5ED81FE81838163E0829586958695C1
:1050600083700E94EB138295880F880F807CED81FE
:10507000FE8193819F73982B93830EC0ED81FE81F7
:10508000808122E04FEF50E060E070E090E00E940D
:105090002913ED81FE81808344244394470C88E0EA
:1050A000582E5F0CAD80BE80C12CD12CED81FE81CD
:1050B0008381982F9F70492F50E09601220F331F54
:1050C00002C0559547952A95E2F7F42FF3702F2EDD
:1050D0008295837090E00C2C02C0959587950A9478
:1050E000E2F7282F2170322E641411F0E12C01C058
:1050F000E98020E048E951E1652D84E00E942365C4
:10510000112311F000E001C00E2D222D4DE553E1D9
:10511000652D84E20E940F65113011F000E001C09E
:105120000E2D232D44E951E1652D82E40E940F6587
:10513000123019F40E2D006801C000E83FEFA31AE9
:10514000B30AEE24E3942B81ED81FE81EC0DFD1D6D
:105150004181652D80E60E947411641060C08091C9
:105160008A07811107C08091580190915901892BBC
:1051700009F455C0113079F180F0123009F04FC0B8
:10518000F501808122E04FEF50E060E070E090E0B8
:105190000E942913F501808342C022E043E060E0D1
:1051A000822D0E94DC13ED81FE812381C114D10484
:1051B00039F0F4E08F9FC0011124922F937002C048
:1051C000922F9C70982B9F70ED81FE818381807F50
:1051D000892B838324C022E041E060E0832D0E947C
:1051E000DC13ED81FE81238122952370C114D1044B
:1051F00029F0982F990F2D7F922B03C0922F9E7F1D
:10520000982B93709295907FED81FE8183818F7CA6
:10521000892B83838091600181110E943D784394A2
:10522000F8E05F0E2FEFC21AD20A32E0C316D104A3
:1052300009F03CCF83E0780E98E1F90EEA81EF5F48
:10524000EA832D813E812C5F3F4F3E832D8337E0E3
:10525000830E911C7F12B2CE26960FB6F894DEBF55
:105260000FBECDBFDF91CF911F910F91FF90EF90B7
:10527000DF90CF90BF90AF909F908F907F906F9076
:105280005F904F903F902F9008954F925F926F9252
:105290007F928F929F92AF92BF92CF92DF92EF92C6
:1052A000FF920F931F93CF93DF93C82F82EE90E16D
:1052B0000E947122E7E0AE2ECC24C394F0EEEF2ED4
:1052C000F0E1FF2E0DE02BE632E14CE06C2F8FEE8B
:1052D00097E00E9490236090EF0780906407A1EA16
:1052E000EA2EA4E0FA2EC0EAD4E0AA24A394B12CBA
:1052F00018E0712C992487FC9094C12CD12C70E378
:10530000472E4A0C0C2D6DED70E1812F0E944365F4
:10531000442D612F8CE00E94EA646A147B0449F4F6
:105320008C149D0431F480918A07811105C021E01D
:1053300001C020E0512C03C022E0552453940130D9
:1053400099F0022FF701208144E850E1612F88E4B1
:105350000E940F655520C1F06CE1F70180810E9429
:10536000EB13F701808310C04881552747FD509506
:10537000612F8CE60E943A67552031F04DE763E8D3
:1053800088810E94E8138883FFEFCF1ADF0A82E04A
:10539000C816D10409F0B6CFE2E0EE0EF11C229659
:1053A000185FFFEFAF1ABF0A103409F0A6CFDF91E4
:1053B000CF911F910F91FF90EF90DF90CF90BF9012
:1053C000AF909F908F907F906F905F904F900895D7
:1053D0007F928F929F92AF92BF92CF92DF92EF9285
:1053E000FF920F931F93CF93DF93D82E81EE9AE015
:1053F0000E94712256E0A52E65E0C62E7BEDE72EB9
:105400007AE0F72E06E02FE532E141E06D2D8EEDDA
:1054100097E00E949023C090DE07809064078091FF
:10542000630081FF04C064ED7AE088E1FCC0CA94A7
:1054300080918A07882319F043E0942E02C09924B2
:105440009394C3E1D5E0B12C10E1AA24A394AB0C52
:1054500020E04A2D612F80E00E943910F12CCB1002
:1054600002C08F1411F000E001C0092D802F82705E
:10547000782E92E0F91609F444C0E3E0FE1609F430
:1054800055C0F1E0E980FF16D1F0E294E694E6948D
:1054900033E0E3222E2D49EC5AE0612F88E10E948F
:1054A0000F65772009F45AC062E08E2D0E94F31335
:1054B0008295880F880F807C99819F731FC0EE0CA6
:1054C000EE0CE594E5948E2D9DE08902F001112407
:1054D000F7FD3396AF015595479555954795202F84
:1054E000612F82E40E943A677720C1F14FE161EEBB
:1054F0008E2D0E94F0138F739981907C982B998345
:105500002DC0E880EE2DE770EE2E2E2F4BEB5AE0EB
:10551000612F88E40E940F65772001F163E08E2DF2
:105520000E94F31387709881987F16C0E880E594F5
:10553000E594E594202F4E2D612F8AE50E9490106E
:10554000772061F04FE061EF8E2D0E94F013880FFD
:10555000880F880F98819770982B9883F394F4E0C4
:10556000FF127DCF185F2296AF1611F0BA2C6DCFC7
:1055700060EB7AE080E30E94436584E0C8120AC0D1
:1055800048E266EF809123050E94F0138093230583
:1055900021E201C020E240912305552747FD5095A7
:1055A000465F5F4F60E38EE40E943A67EE24E39427
:1055B00095E0C912E12C2E2D4CEA5AE068E380E018
:1055C0000E94236502E411E0CBE0D5E090E3F92EE0
:1055D000F801419151918F0169917991461B570BC7
:1055E000440F551F20E268E38F2D0E943A67F8E1CF
:1055F000FF0E80E9F812ECCFEE2091F090E6D91280
:105600000FC088E0E2E4F1E0ABE0B5E001900D927C
:105610008A95E1F781E00E94715F87E10E948A73B9
:105620006CE97AE088E0DF91CF911F910F91FF90B4
:10563000EF90DF90CF90BF90AF909F908F907F9032
:105640000C944365FF920F931F93CF93DF93F82E33
:10565000EB018A0147E16CE20E94472243E06BE2E2
:105660008F2D0E94DE6543E06CE28FEF8F0D0E946C
:10567000DB65C8016FE87FEF0E94A77A2CE2260F56
:10568000CE0161E770E00E94A77A862F45E0622F85
:105690008F0DDF91CF911F910F91FF900C944722B6
:1056A000CF92DF92EF92FF920F931F93CF93DF93EE
:1056B000CCEAD7E04A815B81688179818AE20E94E5
:1056C000222B4C815D816E817F8186E50E94222B99
:1056D0002896EAE3FE2E0DE510E0F7E3CF2E899140
:1056E00099919C5FB8010E94A77ADD24D394D60ECD
:1056F000EC2CE61A4D2D6E2D8F2D0E94DE654D2D62
:105700006E2D81E08F0D0E94DE654D2D6E2D82E0A5
:105710008F0D0E94DE6585E0F80E89E4F812DFCF78
:10572000DF91CF911F910F91FF90EF90DF90CF907D
:105730000895DF92EF92FF920F931F93CF93DF9321
:10574000F82E87E59BE00E947122EE24E39406E0A8
:105750002FE532E145E06F2D82EE97E00E940726AB
:105760001092E207C5E4D7E010E0812F0E941315E4
:1057700048815981841795070CF4AC0149935993DA
:105780002C853D85281739070CF49C013D872C8713
:10579000143060F0FE017097240F351F37FF02C0F0
:1057A0002F5F3F4F35952795318320831F5F17303B
:1057B000E1F6809161078093860790E2F91621F067
:1057C0008FEBF8120EC00BC08F5F809361078330A0
:1057D00041F487E10E948A7381E00E94715F109218
:1057E000610780916107813089F050F0823009F0C3
:1057F00072C010926D01CAEDD4E0E5E4F7E01FC07D
:1058000066E47BE088E10E94436565C0C7E3D7E0BA
:10581000D12C18E9E12E1AE3F12E08E615ECFF86EB
:10582000EE861D8F0C8F8D2D0E94131589939993F1
:10583000D39497E0D912F3CF68E37BE043C0619142
:105840007191848595859B01281B390B37FF03C017
:10585000319521953109233331053CF1DF01509712
:105860004D915C91598348839A01261B370BB901EE
:1058700037FF02C0615C7F4FB6E075956795BA95BA
:10588000E1F7261B370B3F872E87841B950B9C0166
:1058900097FF02C0215C3F4FA6E035952795AA955A
:1058A000E1F7821B930B9D8F8C8F229687E0E33567
:1058B000F80729F60E94CB5D9093050580930405B7
:1058C00066E27BE080E10E94436549E152E168E1E4
:1058D00082E10E944965DF91CF911F910F91FF9066
:1058E000EF90DF900C94502BFF920F931F93CF9368
:1058F000DF93182F062FEA01F22E222321F061E018
:105900000E94F313182FBE01802F0E9443652F2D94
:10591000412F602F86E60E947623812FDF91CF9161
:105920001F910F91FF900895FF920F931F93CF93B4
:10593000DF93182F062FEA01F22E222321F061E0D7
:105940000E94EB13182FBE01802F0E9443652F2D5C
:10595000412F602F86E60E947623812FDF91CF9121
:105960001F910F91FF9008957F928F929F92AF9217
:10597000BF92CF92DF92EF92FF920F931F93CF933C
:10598000DF93C82F89E891E10E947122D1E1AD2E09
:1059900014E0C12E04E8E02E01E1F02E0DE02BE62C
:1059A00032E14AE06C2F80EF97E00E949023109143
:1059B000F0079090640790918A07C23278F0C6325F
:1059C00030F0CF3B59F48091590D806405C0992384
:1059D00051F08091590D80638093590D992319F0EE
:1059E000B2E0FB2E02C0FF24F394183008F02EC161
:1059F000E2EEAE2EEDE0BE2EF0EECF2EFDE0DF2E7D
:105A0000E50188248394A8E07A2E69E771E1872D67
:105A10000E9443658C2F8A19813029F442E5672D55
:105A200080E00E94EA64181102C0992011F000E0A1
:105A300001C00F2DF60120814DE553E1672D82E471
:105A40000E940F65181103C0F1E09F1611F000E0ED
:105A500001C00F2D288130E040E050E073E0E72ED8
:105A6000672D86E60E942A66181120C080918A0759
:105A7000811106C08091580190915901892BB1F094
:105A800091100AC022E043E060E0F60180810E94AC
:105A9000DC13F60180830AC0F1E09F1207C022E008
:105AA00048E760E088810E94DC138883839488E063
:105AB000780E2196EFEFCE1ADE0AF3E08F12A5CF13
:105AC000C0918F0480E4C89FE00111246FE671E16A
:105AD00088E10E944365133041F4911006C0809123
:105AE0008A07882321F002E003C000E001C001E042
:105AF000202FAE0168E184E50E943A67023061F42C
:105B000080918F0422E048EC50E060E070E090E08B
:105B10000E94291380938F04133049F4E1E09E1210
:105B200006C080918A07882321F0C2E003C0C0E04C
:105B300001C0C1E00C2F2091900441EF52E168E1D7
:105B40008AE50E940F65C23039F46FE080919004BD
:105B50000E94EB138093900464E671E180E20E945E
:105B60004365143051F442E361E0809191040E9456
:105B7000E8138093910421E001C020E0409191045A
:105B800050E060E284E50E943A67C091F501C29559
:105B9000C695C695C3706BE571E188E20E944365C6
:105BA000153091F462E08C2F0E94EB13C82F982FD0
:105BB0009295990F990F907C8091F5018F73892BA5
:105BC0008093F5010F2D01C000E02C2F40E551E13D
:105BD00068E282E40E940F6564E471E180E30E9460
:105BE0004365163069F48091630422E042ED50E091
:105BF00060E070E090E00E9429138093630401C08C
:105C0000F12C209163040F2D006330E0220F331F2D
:105C1000442737FD4095542F64E0E62E60E384E589
:105C20000E942A6621E0173009F020E08091F501FA
:105C300049E351E168E3829581700E94942C909130
:105C4000F50180FB94F99093F5019FC01E3028F573
:105C50006AE271E188E00E944365CAE9D4E080E12C
:105C6000F82E98E0D92EDC1A8C2F8D0D181307C052
:105C700061E288810E94EB13888301E001C000E0AB
:105C8000299140EE53E16F2D80E00E940F6588E07E
:105C9000F80EE0E4FE12E8CF78C06FE171E188E031
:105CA0000E9443651E3089F480918E046FE08295D6
:105CB0008F700E94EB138295807F90918E049F706D
:105CC000982B90938E0421E201C020E240918E0433
:105CD00042954F7050E068E084E50E943A67C0E169
:105CE000F12CD1E08FE08F0D1813D0E0F11018C027
:105CF00061E171E180E10E9443650D2F2091D6049E
:105D000043E051E16C2F8AE50E940F65DD23C1F16C
:105D100062E08091D6040E94EB138093D60430C0D9
:105D2000F1E0FF1217C06BEF70E18C2F0E9443650A
:105D30002D2F4091D7046C2F8AE50E949010DD230F
:105D4000F9F046E16BEE8091D7040E94E81380934E
:105D5000D70416C06EEE70E18C2F0E94436540910F
:105D6000D80450E02D2F6C2F86E60E943A67DD2381
:105D700039F062E38091D8040E94EB138093D80439
:105D8000F394C85F83E0F812ACCFDF91CF911F91FD
:105D90000F91FF90EF90DF90CF90BF90AF909F90CA
:105DA0008F907F9008951F93CF93DF93D62F122F5C
:105DB0000E94942CC82F212F482F6D2F86E60E9419
:105DC00084238C2FDF91CF911F910895CF93482F7B
:105DD000CAE02AE0829FC00111248D5F9D4F2FE110
:105DE00030E0241B3109C29FA001C39F500D112434
:105DF000BC01665F7F4F0E94157BE9E3F3E0DF01A2
:105E00001D92CA95E9F782E00E94715FCF910C94D0
:105E100010600F93CF93C42F0E949010002339F08D
:105E200046E16AEE8C2FCF910F910C94E8138C2FE2
:105E3000CF910F9108950F931F93CF93DF93D82F96
:105E4000162FC42F022F47FF08C041E28AEF8D0FA3
:105E50000E945B6486E08C1BC82F2C2F4FE15FE013
:105E6000612F8D2F0E940F65DF91CF911F910F91B0
:105E700008950F931F93CF93DF93162F8132C0F5B0
:105E8000811103C0611108C033C0803219F4662348
:105E900029F02EC0662311F001E001C00FEF080FBA
:105EA0000E94B60FEC01802F0E94B60FFC01988172
:105EB0008FEF890F8031E0F420812131C8F429135C
:105EC00002C08BE009C0112329F0903188F49F5F54
:105ED00098830EC088830CC0815029F0908128815E
:105EE00021939993F9CF82E00E94715F0093F907A3
:105EF000DF91CF911F910F910895809139038823ED
:105F000029F08AE89EE10E94731B81E00895BC019C
:105F100088E00E94436568E37EE088E20E94436572
:105F200069E27EE080E30C944365CF93C82F81360D
:105F300069F08F3B39F0803699F4809136070E94E2
:105F4000E62E04C080E00E948A730AC08C2F0E9453
:105F5000126981E00E94501B8AE59CE40E94731B39
:105F60008DE19EE0CF910C94872F0F93CF93C82F94
:105F70004FE067E377E0809132070E94415E00E1E5
:105F80002AE047E357E060E181E00E94ED644FE3DF
:105F900060E182E40E94EA6480913307882319F06B
:105FA0008EEB9DE002C081EB9DE00E94872FC13601
:105FB00051F1CF3B19F0C03691F505C080E0CF918B
:105FC0000F910C948A73809133078823A9F08FE98D
:105FD0009DE00E949812809132070E94B65E88234D
:105FE00039F087E10E948A7382E08093330709C009
:105FF00080E00E948A7305C0809132078F5F0E9403
:10600000936180E601C081E60E94126981E00E94EE
:10601000501B86E495E3CF910F910C94731BCF91A5
:106020000F9108959091D40181E0191624F09111F7
:1060300001C080E081951092D4010895CF93C82FBC
:106040000E941230909135072091CB012136E1F06A
:1060500028F4203249F02E3239F008C0233671F08E
:1060600038F02E3889F002C081E00FC0181624F4F1
:106070009C1730F49F5F04C0882311F09111915058
:106080009093350780E001C082E0CF9108950F938F
:106090001F93CF93DF93EC01062F000F000F000F2B
:1060A00018E0011788F063E17EE0812F0E944365CC
:1060B000AE01612F88E10E944965FE01849121961D
:1060C0008111FBCF185FEDCF2AEF210F40E367E08E
:1060D00082E1DF91CF911F910F910C944C67CF9289
:1060E000DF92EF92FF92CF93DF93FC01EB019C01D3
:1060F000DC010E945A7A9B01AC01DE010E94707A99
:10610000272F382F492F5527DF010E94707A6B0106
:106110007C013CE0F694E794D794C7943A95D1F784
:1061200024E630E02C1B3D0B0E945A7A6E5C7F4FB8
:106130008F4F9F4F6C0D7D1D8E1D9F1D24E630E0FF
:1061400040E050E00E94BB7AC901DF91CF91FF90FF
:10615000EF90DF90CF9008951F93CF93DF93611559
:10616000710529F1192F111F1127111F19F0919590
:106170008195910977FF10C0719561957109C0E013
:10618000D4E09E01281B390BC9010E946F309E018B
:10619000281B390BC90102C00E946F30112329F05E
:1061A00022273327281B390B01C09C01C901DF912D
:1061B000CF911F910895EF920F93CF93DF93962F76
:1061C000642F322F402F8823E1F121E001E0C091BC
:1061D000F7078EE0C89FE0011124CD56DC4F33361F
:1061E00031F44C85892F0E94092F8C8734C03236B8
:1061F00031F44D85892F0E94092F8D872CC0E42F03
:10620000F0E0E30FF11DE30FF11DEE0FFF1FEE0DA8
:10621000F11DEC0FFD1FEF01411108C0E22E04E655
:106220002CE94881892F0E94CA2109C048814C5914
:10623000E22E04E620E0892F0E94CA21845688833A
:106240000AC001E0E0915801F0915901EF2B09F4E7
:1062500000E020E0BCCFDF91CF910F91EF90089547
:106260002F923F924F925F926F927F928F929F9266
:10627000AF92BF92CF92DF92EF92FF920F931F9354
:10628000CF93DF9300D000D01F92CDB7DEB7182F89
:1062900080E09EE00E947122B5E0AB2EC12C0FEF92
:1062A000E02E0DE0F02E0DE02BE632E143E0612F11
:1062B00089EE97E00E949023F090E907F11002C068
:1062C00020E00FC010926D0121E0F212F9CF20E022
:1062D00043E060E08091F7070E94DC138093F707AA
:1062E00021E04091F7074F5F68E080E00E9439109D
:1062F0008091F7070E942422D82E31E0831731F0D5
:1063000082E0D81206C06FEE7DE005C067EF7DE049
:1063100002C068EE7DE088E00E9443658091F70747
:10632000E82FF0E0EE0FFF1FE455F84F4081518158
:10633000453651052CF44C395F4F24F012E003C070
:1063400010E001C011E00E94D016811110E062EE51
:106350007DE080E10E944365112319F081E0E2E0D5
:10636000FE1280E0EE24E39400E02D2D48E168E188
:106370000E94DB30113019F081E0F2E0FF1280E082
:10638000E12C00E02D2D48E160E30E94DB306AED56
:106390007DE080E20E944365112319F081E023E053
:1063A000F21280E0EE24E39401E02D2D48E268E152
:1063B0000E94DB30113019F081E033E0F31280E00D
:1063C000E12C01E02D2D48E260E30E94DB3064ED1A
:1063D0007DE080E30E94436581E094E0F91280E073
:1063E000E12C00E023E640E36EE10E94DB306EEC3E
:1063F0007DE088E30E94436581E0E5E0FE1280E0F5
:10640000E12C00E022E648E36EE10E94DB3040919F
:10641000F707FEE04F9FA001112424E0D29E400D1B
:10642000511D112447515E4FFA01E655FE4FDA0126
:10643000A555BE4F1C91DA01A455BE4FFC9034E621
:10644000F30EDA01A355BE4F0C910C5980810E94C6
:10645000C216682E812F0E94C216782E44E660E094
:106460008F2D0E94AC16982E44E660E0802F0E948B
:10647000AC16882E8091F7070E94D016E62DFF27D4
:10648000E7FDF095FD83EC83092D112707FD10959D
:10649000882309F45DC0C12CD12C7601B12C61E2B6
:1064A000262E312C74E6472E512C6C817D81D7012C
:1064B000C601B595A795979587950E94AC30880F32
:1064C000991FB1010E94A77A609FC001619F900D42
:1064D000709F900D11245FE3A52EAB0CB2010E94BA
:1064E000937AF0E4F61B6F2F8A2D0E948E658B2D18
:1064F0008370B394811108C06FE38A2D0E948E656A
:106500006B2D8FE30E948E6521E2C20ED11CE11C2F
:10651000F11C3EE3B312C9CFE091F707F0E0EE0FB4
:10652000FF1FE455F84F00811181C80161E270E05E
:106530000E94A77A862F4EE361E0825A0E94DE65B0
:106540008091F7070E94D016882309F49CC069C087
:10655000E12CF12C512C81E2C82ED12C94E6A92EED
:10656000B12C872D992787FD90959B838A83282CB2
:10657000332427FC30946C817D81C7010E94AC30AC
:10658000B6010E94A77A609FC001619F900D709F25
:10659000900D1124BEE54B2E450CB5010E94937A57
:1065A00090E2961B692F842D0E948E65E52DE37085
:1065B000E983E11109C060E2842D0E948E6560E2EA
:1065C000650D8EE50E948E656A817B81C7010E9400
:1065D000AC30B6010E94A77A629DC001639D900D08
:1065E000729D900D1124AEE54A2E4518B5010E940A
:1065F000937A605E842D0E948E65F981F11109C045
:1066000060E2842D0E948E6560E265198EE50E942D
:106610008E65539421E2E20EF11C3FE15312ABCFA1
:106620007BCFC8019C5F97FD01966C817D8195951C
:1066300087950E94AC309C01220F331FA92D97FC37
:10664000AD5FA595A595BB27A7FDB0950E94527A91
:1066500029E130E040E050E00E94DD7A69017A01F2
:10666000C90161E270E00E94A77A80E4861B4EE3D4
:10667000682F8FE30E94DB65C601D7FC01967C0181
:10668000F594E7942EC0101611060CF4762C672DA5
:10669000772767FD7095C8010E94AC30101611066F
:1066A00014F4A92D01C0A82DA7FDAD5FA595A59552
:1066B0009C01BB27A7FDB0950E94527A29E130E0EA
:1066C00040E050E00E94DD7A7901C90161E270E0AA
:1066D0000E94A77A80E2861B4EE3682F8FE30E9418
:1066E000DB6589E1809FA001819F500D112457FF38
:1066F00002C041505F4F852F880F880B452F582FC0
:1067000060E382E70E94496789E18E9DA0018F9D29
:10671000500D112457FF02C041505F4F852F880F45
:10672000880B452F582F68E084E50F900F900F904D
:106730000F900F90DF91CF911F910F91FF90EF90ED
:10674000DF90CF90BF90AF909F908F907F906F9091
:106750005F904F903F902F900C94496790E0E92F05
:10676000F0E0E458FC4EE491E81721F0EE2321F02C
:106770009F5FF5CF892F089580E00895823430F42B
:10678000E82FF0E0E458FC4E8491089580E20895EB
:10679000FF920F931F93CF93DF93C82FD62FF42E22
:1067A000122F622F842F0E949D12FC01E53F81E091
:1067B000F80794F09BE09E0F9F1510F09CE09E0F51
:1067C00040E3490F202F6D2F8C2FDF91CF911F9128
:1067D0000F91FF900C945B64212F44E15CE06D2FDE
:1067E0008C2F0E940F65DF91CF911F910F91FF9029
:1067F0000895BF92CF92DF92EF92FF920F931F9373
:10680000CF93DF93C82F87EF9BE00E94712224E093
:10681000E22E0DE02BE632E142E06C2F86EE97E0AF
:106820000E940726D090E607C03611F0CE3669F4F4
:10683000DD2059F08FEF8D0D8093FC078C2F0E9487
:10684000126982E794E30E94731B6DEE7BE080E1A6
:106850000E944365C9EED1E098E1F92E11E0BB2416
:10686000B3941D11B12C69EE7BE08F2D0E9443651E
:1068700040E3410F6F2D82E10E94EA642B2DFE015F
:10688000E353FD4F40816F2D8AE20E9490108AE50C
:10689000C82EE12C0B2D2E2D412F6F2D8C2D0E94FB
:1068A000C833E39486E0C80E84E0E812F3CF1F5F9C
:1068B00088E0F80E2A96153091F60E94951B682FF5
:1068C000660F660F660F615F29E04AE180E0DF91A5
:1068D000CF911F910F91FF90EF90DF90CF90BF90DD
:1068E0000C944C678F929F92AF92BF92CF92DF929F
:1068F000EF92FF920F931F93CF93DF93C82F809057
:10690000FC072AE0829E40011124C40182559B4F5E
:106910004C018CE09CE00E947122AA24A394CC2418
:10692000C3945AE0E52E5CE0F52E00E020E030E074
:1069300040E06C2F87EE97E00E9490234091FC0787
:106940004F5C60E080E30E94EA64A090E707B090AB
:106950008A0718E0D12CAD1005C01B142CF442E0BE
:10696000E42E04C0E12C02C0EE24E39491E0D91699
:1069700081F063E07CE0812F0E9443650E2D2E2D77
:10698000F4014085612F80E30E94092FF401808784
:1069900051C06DEF7BE0812F0E94436530E3C32E31
:1069A000F12C809164078F1511F000E001C00E2DCD
:1069B0004091FC074F5F2F2D612F8C2D0E94C83313
:1069C000EE2091F1209164072F112EC01B1434F09A
:1069D0008091580190915901892B31F1E401C20F46
:1069E000D11DC20FD11DE881F981CF018B509E4F7F
:1069F000843FF1E09F0714F484EF91E022E048EF38
:106A000051E064EF71E00E942913AC0180916001B4
:106A1000882351F0443F21E0520711F440E050E058
:106A2000455F514059834883F39486E0C80E94E053
:106A3000F912B7CFD394185FE2E0DE128CCFDF916A
:106A4000CF911F910F91FF90EF90DF90CF90BF906B
:106A5000AF909F908F900895CF93C62F0E94126998
:106A60000E941060C09306058C2F0E94785E809172
:106A7000F3010E942E1482E080930E0181E00E94B7
:106A8000715F0E94106081E0CF9108958F929F9274
:106A9000AF92BF92CF92DF92EF92FF920F931F932C
:106AA000CF93DF93182F89E69BE00E947122F0902C
:106AB000E40780913107811109C081E08093BA0712
:106AC0004FE0612F84EE97E00E94182663E67BE09A
:106AD00080E00E9443650E948460AC0160E086E62D
:106AE0000E944967B090E40780913307823021F417
:106AF0001092E30710923307CB2DDD27C7FDD09509
:106B000080918B079E01281B3109C90118161906AF
:106B10006CF09E012150310937FF02C020E030E0C7
:106B200020938B0770E1A72E812C3EC025303105C4
:106B3000CCF39E01245031092B3031058CF32AE02F
:106B400030E0EECF00E196012F5F3F4F442737FD45
:106B50004095542F62E0E62E6A2D82E10E942A665B
:106B600080910605981205C04AE26A2D81E00E94D4
:106B7000EA644FE067E377E0892D0E94415ECC151F
:106B8000DD05E1F48091E3078823C1F001E12FE006
:106B900047E357E06A2D88E10E94ED64839438E072
:106BA000A30E86E0881661F090908B07980CC92C94
:106BB000D12CCC15DD0531F601E1C5CF00E1E7CFE1
:106BC00080913107882309F453C090910605809184
:106BD000E407981302C003E001C004E0602F8AE2DA
:106BE00092E10E9447308FEF800F0E941E30D82E16
:106BF00000913507602F660F660F660F685F20E013
:106C000044E288E10E94716521E0D21228C001119E
:106C100010C06091E40760930605812F0E942C3517
:106C200080913107823009F58DE795E50E940214C5
:106C30001CC0033031F4812F0E9412691092330777
:106C400004C0013049F400933307B092320785EB5A
:106C50009FE20E94731B09C0D092E30706C032E096
:106C6000D31256C0812F0E9412691092310750C072
:106C7000163638F41436A0F4103649F1113649F0BE
:106C800047C01138B1F11F3BC1F11E3609F040C0B9
:106C90001EC08091E3078823D9F11092E30738C022
:106CA000909106058091E407981749F0812F0E9482
:106CB00012691092350782E08093310729C0109243
:106CC000BA07153609F051C085E499E250C08091A9
:106CD000E307882319F01092E30708C0812F0E9470
:106CE00012691092350781E08093310710928A076C
:106CF0000FC081E00E94501B0BC01092E30710925E
:106D00003107809106058093E40781E00E94835F4C
:106D10008091E307882371F1FB1461F161E06B0D51
:106D200081E08F0D0E9471618091060590E0C81787
:106D3000D90719F4F092060509C02F2D332727FD36
:106D4000309528173907B1F4B092060581E0DF913C
:106D5000CF911F910F91FF90EF90DF90CF90BF9058
:106D6000AF909F908F900C94715F8DE795E50E9496
:106D70000214CECFDF91CF911F910F91FF90EF9032
:106D8000DF90CF90BF90AF909F908F900895DF924B
:106D9000EF92FF920F931F93CF93DF93E82E009112
:106DA000F401CBEBD7E010916404202F332727FDAB
:106DB000309537FF03C031952195310925323105D2
:106DC00054F12D853E854F855889242B352B4B85D5
:106DD0005C85242B352B8989282B8A89282B232B0A
:106DE00029F4802F881F8827881F8A8B101614F497
:106DF0008CED01C084E2800F40E060E00E94EC1660
:106E0000882341F09A89911105C091E029892111C7
:106E100090E0998B8A8B112339F040E060E0812F5C
:106E20000E94EC16882319F0FF24F39402C0F12C81
:106E3000E12C2D853E852F5F3F4F3E872D872F8587
:106E400038892E0D311D388B2F87F89420915F0CD7
:106E50003091600C78948B859C85281B390B2436E7
:106E6000310508F423C18C599F4F9C878B872F8550
:106E70003889ED85FE85C901BF010E94937AE62E0F
:106E8000D62E6E9FC0016F9F900D1124281B390BC9
:106E9000388B2F871E861D868FE0800F8F3110F470
:106EA000198A0DC094E2900F993448F4101614F426
:106EB00081EF800F40E060E00E94EC16898B20910A
:106EC000F401332727FD309537FF03C03195219515
:106ED0003109622F88819981019699838883EA819B
:106EE000FB813196FB83EA83DD2029F08E819F812F
:106EF00001969F838E83613009F4698B8989882389
:106F000041F0FF2031F04C815D814F5F5F4F5D8329
:106F10004C83E694488559854E0D511D5987488705
:106F2000E090F601F090F701FC8AEB8A611102C053
:106F30001A8620C0613031F4111114C0C7018E1BB4
:106F40009F0B16C0603170F420FF06C0E4E0569538
:106F50004795EA95E1F702C04E815F81C701841B26
:106F6000950B06C08C819D819701281B390BC901A7
:106F70009C8B8B8B8A850B891C89813049F018F09A
:106F8000823069F017C08091F401882399F010C015
:106F900017FF10C0E114F10469F082E00AC0053C5B
:106FA0003FEF130714F483E08A87E114F10411F42E
:106FB00081E08A87898D9A8D8017910709F46AC0CC
:106FC0008A85813009F057C080911F0582FF31C04A
:106FD000E114F10471F10E31110519F469E289E14E
:106FE0000BC00431110519F46AE28AE105C00A30C8
:106FF000110531F46BE28BE10E94907381E00DC0CA
:10700000063011054CF417FD03C0602F8CE1F4CF5E
:107010008CE10E948A73F2CF80E090911F0593FF6C
:1070200008C0882331F082E390E09093540180936C
:1070300053018091F50180FF04C0C701801B910BB3
:1070400001C0C8016CE370E00E94A77ADC01CB01AB
:1070500040911F0541FF1EC0AB2BE1F44091280574
:1070600041FF07C0009761F046E260E00E9499731B
:1070700007C080E003C0823069F48CE10E948A730B
:1070800080911F0583FF06C082E390E09093540136
:10709000809353018B899C899A8F898F2091F50168
:1070A00020FF04C0E81AF90AFC8AEB8ADF91CF912D
:1070B0001F910F91FF90EF90DF900895CF93DF9392
:1070C0009091F40197FD91958EEF890F8E3020F508
:1070D000892F85959A3024F40E94466A90E003C077
:1070E000992787FD90950197FC01EE0FFF1FE4554E
:1070F000F84F208131818091F40187FF05C080E045
:1071000094E0821B930B02C0C9019C5FC6E0969578
:107110008795CA95E1F702C080E090E00E94C736EB
:1071200083E00E94466AE82FF0E0EE0FFF1FE6556D
:10713000F84F808191819C5FB6E096958795BA95CE
:10714000E1F72091F50122FF0AC08530910538F062
:107150002091D207211103C023E02093D207C7ED6D
:10716000D7E0288139812F5F3F4F398328832A81D7
:107170003B81280F391F3B832A83F89480915F0C51
:107180009091600C78942C813D81AC01421B530B93
:107190009A01283E334088F19D838C838091F801C9
:1071A000823039F440E060E085E10E94EC16811104
:1071B00020C08A819B81688179810E94937A1B8299
:1071C0001A82198218828091B706893718F48F5F66
:1071D0008093B706E091B80681E08E0F8093B806E1
:1071E000F0E0E754F94F6083883738F01092B80622
:1071F00004C087E00E948A73DCCFDF91CF910895AD
:10720000EBEBF7E012861382128217821682158248
:107210001482118610868091F6019091F701928F69
:10722000818F0895EF92FF920F931F93CF93DF9377
:10723000D82F162FF42E022F22FF02C0C5E001C066
:10724000C3E089E08D0F0E948116006448E04D0F75
:10725000EC2E9C016F2D812F0E94B220DF91CF91E7
:107260001F910F91FF90EF900895EF92FF920F936F
:107270001F93CF93DF93C62F13E0E12EE60E1AE59E
:10728000819F102D1124165FD0E2CE15B8F4FF2493
:10729000F394FC0E40E060E08F2D0E94EC1693E02A
:1072A000C99FA0011124495E5C4F082F23E06D2F78
:1072B000812F0E94ED64D85FCF2DE7CFDF91CF9172
:1072C0001F910F91FF90EF900895CF92DF92EF9270
:1072D000FF92CF93DF936B017C01C0E1D0E040E0EF
:1072E00050E8E0E0F0E89A01DA010E945A7AC61606
:1072F000D706E806F90610F44E275F27F695E795BE
:107300002197209719F04E2B5F2BEDCFCA01DF910B
:10731000CF91FF90EF90DF90CF9008951F9341E0C1
:10732000262F30E0683050F440E055E0529FF001E5
:10733000539FF00D1124E153FC4F0AC0285031092E
:1073400059E0529FF001539FF00D1124E950FC4F7A
:107350009C5F97FD0DC0811528E0920784F04423BF
:1073600019F088E090E002C084E090E0E80FF91F97
:107370002081332727FD3095322F222725C0442333
:1073800029F0492F9927880F991F03C0492F469547
:107390009170242F30E0E20FF31F608140E052E053
:1073A000481B590B5595479564039001659F300D17
:1073B00011241181BC01759567951603A001179FD3
:1073C000500D1124240F351FC90169E170E00E949E
:1073D000A77ACB011F9108956F927F928F929F920F
:1073E000AF92BF92CF92DF92EF92FF920F931F93D3
:1073F000CF93DF93982EDD24D3948091FB078830C0
:1074000008F4D12C88E092E10E947122DD2011F075
:1074100089E001C085E0A82EC12CB7E0EB2EB2E1D7
:10742000FB2E00E020E030E040E0692D85EF97E0A2
:107430000E9490232FEB921202C01092F407409109
:10744000FB0750E04F5F5F4F21E060E084E20E9465
:107450003A67C091FB07DD2061F08C2F90E0089720
:1074600029E0289FE001299FD00D1124C950DC4F4D
:1074700006C045E0C49FE0011124C153DC4F609079
:10748000F5076A94CC2E7D2EAC2EBD2E05E010E0C3
:10749000A0E18A2EE62CFF24E7FCF094F50141914F
:1074A0005F0121E0C8010597E816F90609F020E020
:1074B000552747FD5095682D88E10E943A67DD20E9
:1074C00091F0093081F021E0E016F10609F020E0AA
:1074D000FE01E00FF11F4081552747FD5095682DB3
:1074E00080E30E943A67F8E08F0E0F5F1F4F28E39A
:1074F0008212D4CF11E04FEF641210E0212F40E050
:1075000052E168E08CE00E942365112309F446C033
:107510009092CB0120E044E06CEF8091F4070E9450
:10752000DC138093F40790916001992399F1DD2099
:1075300021F090E164E049E003C098E062E045E0BA
:1075400054E685028001112470E0719561957109FE
:10755000582F56039001579F300D112484E6829FC7
:107560004001839F900C1124EC2DF72D20E030E09A
:10757000A92EB12CC901880D991DB5010E94A77AC9
:107580006193200F311F8E2F8C19841798F382E09E
:107590000E94715FC12C0CE91FEF34C044E66CE916
:1075A0008E010E0D1F1DF80180810E94E813F80165
:1075B0008083F0CF85E090E02817390794F5C90162
:1075C000F5E0880F991FFA95E1F7DD2011F164E0ED
:1075D00070E00E94A77AB62EFE01E20FF31F8081B1
:1075E000F0E28F02C0011124B8010E94A77AE216CE
:1075F000F30691F4625E25E045E08AE38B0D0E947C
:107600004C67C3942C2D30E0DD20A1F289E090E09E
:10761000D3CF62E070E0DDCF615E23E043E08BE337
:10762000EDCFC0E0DCEF10E0E0E2FE2E6091FB0762
:10763000CE010E948E390CE3010F75E09695879577
:107640007A95E1F76F2D681B802F0E948E65812F40
:10765000837021F460E2802F0E948E651F5FA096E8
:10766000103421F740E460E08CE5DF91CF911F9169
:107670000F91FF90EF90DF90CF90BF90AF909F90D1
:107680008F907F906F900C94DE652F923F924F9277
:107690005F926F927F928F929F92AF92BF92CF92A2
:1076A000DF92EF92FF920F931F93CF93DF93CDB7AB
:1076B000DEB76E970FB6F894DEBF0FBECDBF8D8FCD
:1076C0009E8F698780915501882309F448C00EE692
:1076D00016E0D8018D0180918807882319F0815028
:1076E000809388070E942315F80123813481821733
:1076F000930741F0948383831282118281E0809307
:1077000052012DC060911E05665F49F18091020112
:10771000823328F1D80180818F5F80838031F8F037
:10772000F801818192810196928381831C9247E7BF
:1077300051E0649F9001659F300D1124281739078F
:1077400070F48F719927019751F486EF9FEF0E9493
:1077500018146DE280E10E9490730E9436140E941A
:10776000951B8093540580911D05F82FF1708F2E85
:10777000839481FF02C0612C02C033E0632E4091EC
:1077800001024423F1F1E82DF0E0EE0FFF1FE45574
:10779000F84FA081B181E62DF0E0EE0FFF1FE45518
:1077A000F84F0190F081E02D9D010E94527A6B010B
:1077B0007C019F01DF010E94527AC60ED71EE81E8F
:1077C000F91E642F70E080E090E02AE0660F771FDA
:1077D000881F991F2A95D1F724E630E040E050E059
:1077E0000E94DD7ACA01B9010E94837A6C157D0579
:1077F0008E059F0530F4C701B6010E9465397C01F2
:1078000002C0E12CF12C9701A4E6B0E00E945A7A64
:107810006D8B7E8B8F8B988FBAED4B2EB4E05B2EE9
:1078200025E136E03C872B87AE014F5F5F4F5E87D7
:107830004D876CEA77E07A8B698BC12CD12C712C47
:1078400079857170798F89858E708A8F99859A7004
:107850009B8FA985A670AC8F9C2C8C2D0E94131534
:10786000F2013296F88BEF87D2012D913C91821B69
:10787000930B9C01BC01882777FD8095982FAAE087
:10788000660F771F881F991FAA95D1F71216130646
:107890001CF4228D338D04C0EF85F889248535854D
:1078A0002436310514F424E630E0442737FD4095B2
:1078B000542F0E94DD7A89012130FCEF3F073CF014
:1078C000011524E012072CF000E014E002C000E0F3
:1078D0001CEF80911F0580FF11C080911D058170F4
:1078E0008B8B1C8A82E090E04B895C89841B950B12
:1078F000C816D90619F4119501951109A989BA89F3
:107900000D931D93BA8BA98B580117FF03C0BFE0DD
:10791000AB0EB11CF4E0B594A794FA95E1F73A2CBC
:10792000E4E0CE16D1045CF481E0890D0E94466A41
:10793000815091E001C0990F8A95EAF706C091E065
:107940000C2C01C0990F0A94EAF737FE02C03A2CBA
:107950003194F1E0F31544F0311002C0892F03C0D7
:1079600080916D068923782A23E0291508F422C125
:10797000398D31114DC08091F50181FF49C052010F
:1079800049E3A40EB11CF5018181807C09F440C05B
:10799000F20181AD40E061E08595859585950E9475
:1079A000EC168823A9F1D501EC91E770F0E0DF0136
:1079B000AA0FBB1FAE5BBE4FEE0FFF1FE55FFA4F76
:1079C0008D919C9120813181821B930B97FD0196B3
:1079D000AC0155954795F5012181322F330F330FB7
:1079E000359535953403C001359F900D11246FE115
:1079F00070E00E94A77A660F771F660F771F2295A7
:107A0000269526952370213009F0A3C6060F171F6F
:107A1000E114F104C1F0981411F0961014C02091F3
:107A2000010230E0D8010E94697AEAE0660F771F10
:107A3000881F991FEA95D1F72D893E894F89588D66
:107A40000E94DD7A8901892D0E942422A82E892D89
:107A50000E94D016EA2DF0E0882311F1EE0FFF1FEF
:107A6000EE0FFF1F2EE02C9DC0012D9D900D1124C7
:107A7000E80FF91FED56FC4F80810E94C216682F57
:107A8000772767FD7095C8019C5F97FD01969595D6
:107A900087950E94AC308C01000F111FB12C24C0BF
:107AA00081E0101611060CF480E0B82E3EE03C9DFB
:107AB000C0013D9D900D1124EE0FFF1FEE0FFF1F23
:107AC0008E0F9F1F87519E4F8B0D911DFC01E65518
:107AD000FE4F80810E94C216682F772767FD709540
:107AE000C8010E94AC308C014EE04C9DC0014D9D00
:107AF000900D112454E0A59E800D911D11248751F5
:107B00009E4F8B0D911DFC01E455FE4F808144E694
:107B100060E08C590E94AC169801A82FBB27A7FDE6
:107B2000B0950E94527A24E630E040E050E00E9496
:107B3000DD7A8901892D0E94D01681111450892D7A
:107B40000E94C616811106C0692D809154050E94BD
:107B5000E3122AC08091FA0180FFF6CF692D80914F
:107B600054050E94E312282F80911F0580FD219566
:107B7000332727FD3095432F532F23583F4F4F4F27
:107B80005F4FA0E0B4E0A01BB10B0E947B7A20E025
:107B900038E040E050E00E94DD7A211568E03607C9
:107BA0004105510589F2C901880F991FAD85BE8530
:107BB0008D939C93EB85FC8511830083FA8DFF23C5
:107BC000F9F023E02915E0F0892D0E94C6168111F5
:107BD00013C03B8D332349F0065F1F4F053111055C
:107BE00020F0AB85BC851D921C92BC8DBB2321F07F
:107BF000ED85FE8511821082EB85FC85118E108E3D
:107C0000FFEFCF1ADF0A2B853C852E5F3F4F3C8765
:107C10002B874D855E854E5F5F4F5E874D8757E0B2
:107C2000C516D10419F04F84588816CE1091FE0164
:107C3000172180916D068095812319F088E10E94BB
:107C40008A7310936D0680E094E0909324068093ED
:107C50002306909326068093250682E10E94C3683E
:107C6000811108C083E10E94C368882331F080E05D
:107C700090E005C080E09CEF02C080E094E090932B
:107C80005E0680935D0622E431E00DE216E0EBE053
:107C9000F5E060E0D9018D919D919D01643020F463
:107CA00040815181841B950B880F991FD8018D93BA
:107CB0009D938D016F5F3296683061F72DE336E05A
:107CC000E3E7F6E04191519161917191D9014D93B2
:107CD0005D939D01B6E0E33BFB07A1F7E0EAF4E02A
:107CE000AFE5B6E0808128E08202C00111248D93C7
:107CF0009D93329634E0EE3AF307A1F7A09001028B
:107D0000AA2009F46EC0E82CF12CEE0CFF1CA70190
:107D10004B5E594F7A01DA01CD90DC90062D10E0D0
:107D2000000F111F0B5E194FF80140815181960120
:107D3000D6010E94527A1B012C019A01DA010E949D
:107D4000527A260E371E481E591E6A2D70E080E0BA
:107D500090E0EAE0660F771F881F991FEA95D1F738
:107D600024E630E040E050E00E94DD7ACA01B9012B
:107D70000E94837A621573058405950590F5C2010A
:107D8000B1010E9465399C01A4E6B0E00E945A7AD4
:107D90001B012C01B12C9501D6010E94697A2AE0C1
:107DA000660F771F881F991F2A95D1F7A2019101AD
:107DB0000E94DD7AD7012D933C93F801A081B18117
:107DC00095010E94697A3AE0660F771F881F991F14
:107DD0003A95D1F7A20191010E94DD7AD8012D9345
:107DE0003C936091FF01862F807E09F4E9C089856C
:107DF0008A7089F4E82DF0E0EE0FFF1FEB5EF94F7B
:107E000020813181E62DF0E0EE0FFF1FEB5EF94F90
:107E10008081918104C080E090E020E030E04985DD
:107E20004670A1F4FE013196E80DF11DE80DF11D3B
:107E300040815181240F351FFE013196E60DF11D61
:107E4000E60DF11D40815181840F951FE5E1F6E0BB
:107E500040910002442349F0DF01A40FB11DA40F9B
:107E6000B11D12974D915C9102C040E050E062FF5D
:107E700003C031952195310963FF03C09195819528
:107E8000910964FF03C0519541955109629566952A
:107E90006770623009F44AC018F46130B1F090C0E4
:107EA000633009F47DC0643009F08AC0BA01621BF6
:107EB000730B738B628B9A01280F391F358B248BC0
:107EC000481B590B578B468B7BC0BC0197FF02C0E8
:107ED000695F7F4FA3E075956795AA95E1F7DC018F
:107EE000A61BB70BBC0197FF02C061587F4F660FFE
:107EF000672F661F770BA61BB70B97FF02C0815039
:107F00009C4FBC01672F770F770B65956595CD0169
:107F1000861B970BBA01621B730B738B628B37FF47
:107F200002C02F5F3F4F359527953FC0B90137FFFE
:107F300002C0695F7F4FA3E075956795AA95E1F749
:107F4000D901A61BB70BB90137FF02C061587F4F9B
:107F5000660F672F661F770BA61BB70B37FF02C094
:107F600021503C4FB901672F770F770B65956595C9
:107F70009D01261B370BBA01681B790B738B628B33
:107F800097FD019695958795840F951FAC01420F3B
:107F9000531F558B448B821B930B978B868B10C082
:107FA000BA01621B730B738B628B240F351FA901FF
:107FB000480F591F558B448B281B390B378B268B49
:107FC0008091550181110E945E3880E4E3E7F6E07C
:107FD000DF011D928A95E9F78BEC93E09093040101
:107FE000809303018CEC93E090930601809305014C
:107FF0008DEC93E090930801809307018EEC93E061
:1080000090930A0180930901E5E9F5E0FC87EB878D
:1080100025E535E03E872D8745EF55E0588B4F87A6
:10802000312C212C832D0E94B60F7C01FC01828112
:108030000E94C2168987D7018C918150803108F047
:108040006FC2EF85F889D08040E061E0F70183815D
:108050000E94EC16F7012181811111C088EF820F77
:10806000823008F047C287818670843009F442C2AA
:1080700080E0293009F03EC000E01CEF3FC081E005
:10808000D11080E0D82E8FEF820FA82FB0E0FD0135
:10809000EE0FFF1FEB5EF94F00811181843150F02C
:1080A000831540F4AA0FBB1FAA0FBB1FAD58B94FD1
:1080B0000D911C91F7013781832F807361F0832F1D
:1080C00082958370815041E050E002C0440F551FFB
:1080D0008A95E2F7242A36FF10C0253070F4E22F8B
:1080E000F0E0EE0FFF1FEF5FFE4FC7010896918390
:1080F000808303C000E010E001C081E0AF85B88953
:108100008C93F7018781887459F48085882341F026
:108110004DE763E80E94AC160E94D716080F191F9E
:10812000F701F681FB8B2985332727FD30953A8BA4
:10813000298BF11105C0F7018581882309F4F0C06E
:10814000AD85BE85AD90BC90EB85FC85808191812D
:10815000A2819C014A2F552747FD509529013A01DC
:10816000D1100AC0BB2777FCBA95A72D962D852D77
:108170006801C81AD90A3EC0F70187818670843029
:10818000D9F4E081F0E0EE0FFF1FE55CF94FA0812C
:10819000B18120E034E60E94697A2B013C01F98527
:1081A000FF2351F02F2F332727FD3095432F532FD7
:1081B0000E94DD7A29013A01C301B20120E031E0D9
:1081C00040E050E00E94DD7A509540953095219531
:1081D0003F4F4F4F5F4F6801C20ED31EC114D104F1
:1081E00049F0F7018581D7FE82958F70F4E68F9F65
:1081F00050011124A114B10491F0809155018823FC
:1082000031F021E0A21AB108A114B10441F03327E2
:1082100077FC3A95272D162D052DC12CD12CAD8537
:10822000BE85AD92BC92C114D10409F474C048015A
:10823000AA2497FCA094BA2CBB89BB2309F467C07D
:1082400080915501882309F443C0E985EE23A1F00C
:1082500029893A8937FF03C031952195310944278F
:1082600037FD4095542F60E070E080E293E00E947B
:10827000DD7ACA01B90104C060E070E080E293E0F9
:10828000F70126811C141D0444F09095809570958B
:1082900061957F4F8F4F9F4F22952F7030E02115B2
:1082A000310591F0E4E6E29FA001E39F500D112417
:1082B0009A01442737FD4095542F0E94DD7A420EE3
:1082C000531E641E751E04C04424582C692C7A2C3D
:1082D000BB2777FCBA95A72D962D852D1C141D0460
:1082E00034F488169906AA06BB0634F009C088152E
:1082F0009905AA05BB0524F44424582C692C7A2C32
:10830000332777FC3A95272D162D052D04C04424DC
:10831000582C692C7A2CAB85BC854D925D926C9261
:10832000F701878187FF28C044E66CE984810E94B9
:10833000AC16A82FBB27A7FDB0951A161B0644F450
:1083400017FF6AC024E630E02A1B3B0BD90109C0A5
:10835000109709F461C0101611060CF05DC0AC59FD
:10836000BF4F98010E94527A24E630E040E050E08E
:108370000E94DD7A890150C0F7016481862F992718
:1083800087FD9095A92FB92F8730910590F5FC01B5
:10839000EC5AFF4F0C94FC7AF7018181893021F46B
:1083A00017FD35C012500BC017FF36C01BC0F701B8
:1083B0008181893039F41016110664F11E5F000FB7
:1083C000111F2AC0101611066CF026C017FF24C01A
:1083D00011950195110920C010161106DCF002C09C
:1083E00017FD15C000E010E017C01016110694F03C
:1083F0000EC067FF06C0119501951109F6E0F61B46
:108400006F2F6750C8010E948E398C0105C000E0B3
:108410001CEF02C000E014E0F701478140FD10C0EE
:1084200081819FEF980F943058F4FE013196E80F48
:10843000F11DE80FF11D329780819181080F191FFE
:108440009801A989BA890E94527A4B015C0148744B
:10845000483099F4F7018085882379F04DE763E887
:108460000E94AC160E94D71624E630E0DC010E9480
:10847000697A860E971EA81EB91ED7010C9110E0CE
:1084800001501109F701878186958370000F111F34
:10849000000F111F813071F0823029F1F801ED5881
:1084A000F94F80819181A281B381880E991EAA1E05
:1084B000BB1E19C0C501B40124E630E040E050E025
:1084C0000E94DD7AF801ED58F94F60817181828157
:1084D00093810E94837A20E034E040E050E00E94E3
:1084E000DD7A49015A01F801ED58F94F80829182F5
:1084F000A282B38233942B853C852D5F3F4F3C870E
:108500002B874D855E854E5F5F4F5E874D876F85FC
:1085100078896F5F7F4F788B6F8770E2371282CDDB
:1085200010915E0C20FE05C0111103C08EE10E9467
:108530008A7321FE07C0812F877F803419F48FE171
:108540000E948A7322FE09C0812F877F803811F034
:10855000103919F480E20E948A738D8D89879E8D6F
:108560009A8767E6262E64E0362EACE8B7E0BE8731
:10857000AD87E3E7F6E0FC87EB87C12CD12CCF86F3
:108580008C2D0E94BD0F4C01FC0183819481A09031
:108590009904B12CA816B9063CF0B194A194B10885
:1085A000A816B9060CF45C01F40121818501FAE0FA
:1085B0002F02000D111D1124D4012C91F5014AE068
:1085C0002402E00DF11D11249F01285E3340085163
:1085D0001C4F033E54E0150714F002EE14E059015D
:1085E0002E316BEF360724F45EE1A52E5BEFB52E3E
:1085F000302F212F8017910714F4382F292FE32EC5
:10860000F22EEA14FB040CF47501AB85BC854D9089
:108610005D906D907C90C301B20124E630E040E0B3
:1086200050E00E94DD7AEB85FC85219331934193E4
:108630005193FC87EB87AD85BE852D933D93BE8717
:10864000AD874114510461047104A9F077FE04C0A0
:10865000D701AA19BB0903C0D801AE19BF09A301EC
:1086600092010E947B7A20EA36E841E050E00E94C5
:10867000DD7A29013A01C7010E9496167C01E40CBB
:10868000F51CC8010E9496168C01C5010E94961621
:108690000E151F050CF47801E816F9060CF47C01A0
:1086A000F4018281882319F0F194E194F10880911A
:1086B0006504F0E1F81B2F852F17F8F4F601EE0F93
:1086C000FF1FEA59FB4F9081892F880F880F8595EE
:1086D000859599F092959695969593709D5F937078
:1086E000923058F040E060E00E94EC16882329F0B8
:1086F000D1018C910E94D7167C01F894E985FA8506
:10870000E192F192FA87E9877894FFEFCF1ADF0AB6
:1087100022E0220E311C30E1C316D10409F02FCF24
:108720006E960FB6F894DEBF0FBECDBFDF91CF912E
:108730001F910F91FF90EF90DF90CF90BF90AF907F
:108740009F908F907F906F905F904F903F902F9071
:108750000895223009F05CC98B015AC9FF920F932A
:108760001F93CF93DF93CDB7DEB7C054D1090FB6B7
:10877000F894DEBF0FBECDBF63E0CE0181960E94AC
:10878000453B61E0CE0101960E94453BE5E4F3E004
:108790009E012F5D3F4F8E010F5F1F4F4181528120
:1087A0008081882329F0D9018D919C91D80104C042
:1087B000D8018D919C91D9016D917C91861B970B6D
:1087C000840F951F883EB3E09B073CF489314CEF42
:1087D00094073CF0482F892F02C048EE83E0942F85
:1087E00002C098E18CEF9183828335962E5F3F4FD4
:1087F0000E5F1F4F83E0E539F80781F60BEC13E0BD
:10880000F12C8F2D0E94C616811102C0D8011C9236
:10881000F3940F5F1F4FB4E0FB12F3CF86E00E948A
:10882000715F81E00E948A73C05CDF4F0FB6F894DD
:10883000DEBF0FBECDBFDF91CF911F910F91FF9093
:1088400008959F92AF92BF92CF92DF92EF92FF92E4
:108850000F931F93CF93DF93C82FD0911B051D2F2C
:108860001F70D07310926D01803809F43FC098F4E6
:10887000833209F4A2C030F4803271F1823209F4FB
:10888000A9C0F2C0853209F481C008F471C08136F4
:1088900009F4C2C0E9C0843809F461C058F48238D0
:1088A00009F4A6C008F4C8C08CEE92E20E9402143B
:1088B00083E8A5C08E3809F449C08F3B09F4C6C0CF
:1088C000853809F0D1C081E0809386078BE79EE46C
:1088D0000E94731B85E86EC0133009F0C5C08091FB
:1088E000D20791E089278093D207ACC0143071F58C
:1088F000D03259F484E00E948116919581959109B6
:108900009093B4068093B306AFC0D11114C0809188
:108910008904807C803C21F48CEE9DE00E94B97536
:1089200080918D04807C803C09F09EC083EF9DE0A7
:108930000E94B97599C0D03349F410927D0D109200
:108940007C0D1092790D1092780D8EC081E080938D
:1089500086070E94F8130E94731B8C2F2BC081E0A6
:108960008093860786E495E30E94731B84E822C007
:10897000123039F48091F6078F5F833074F080E015
:108980000CC0143009F070C080E10EC0123041F408
:108990008091F607815087FD82E08093F60764C0DE
:1089A000143009F061C080EF8D0F80738460809374
:1089B0001B0548C00E94126957C01F5F153008F0A0
:1089C00010E0812F8D2B80931B0581E00E94715F49
:1089D00083E139C0112311F0115001C014E0812F3F
:1089E0008D2B80931B0581E00E94715F84E12BC079
:1089F000D460D0931B0587E10E948A7382E8DF91DF
:108A0000CF911F910F91FF90EF90DF90CF90BF908B
:108A1000AF909F900C9412698091C507823021F429
:108A200083E08093C5070EC0133019F40E9411141F
:108A300009C01430C9F404C00E9400390E94111406
:108A40000E94137787E10E948A730EC081E00E9422
:108A5000126983E00E94126982E00E94126981E03B
:108A60008093D6071092F60740E060E08091FD0108
:108A70000E94EC16C82F882331F08091D60781110F
:108A800002C00E94AE43C093D607143009F49DC0C3
:108A90009091020180910805981710F4C6E001C07A
:108AA000C4E080E00E9460124C2F406860E185E2E3
:108AB0000E94341046E568E186E20E94EA648091F3
:108AC000C5078823A1F0823011F426E001C024E01C
:108AD0004091CE075091CF07022F60E18DE50E94B3
:108AE000C40F20E040E068E183E30E94C21000E090
:108AF0002091FB014DE258E060E186E20E940F65A3
:108B00008091FA0180FF06C049E258E060E188E305
:108B10000E944965C0E0D0E00FE1E02EFC2EFE018E
:108B2000EB5DF74FD4906C2F809154050E94E312B7
:108B300097FD03969C013595279535952795243EFD
:108B40000CF424EE022F2D310CF00CE18FEF8F0D81
:108B500046E38230E0F464E08D2D0E94DE65809172
:108B60001D058F2580FD04C08091FA0180FD0CC099
:108B700043E06EE18FEF8D0D0E94DE6543E06EE114
:108B800081E08D0D0E94DE656E2D601B14C06BE3CD
:108B900085EE8D0D0E94DB65FF24FA94FD0C43E009
:108BA0006AE38F2D0E94DB6543E06CE38F2D0E940A
:108BB000DB65D00E6BE347E08D2D0E9447222196A6
:108BC000C430D10509F0AACF29C001E12AE049EE5D
:108BD00051E060E080E00E94ED649091020180919C
:108BE0000805981710F442E001C040E060E084E519
:108BF0000E9434108091C507882309F491C0823007
:108C000011F422E001C020E04091CE075091CF073F
:108C1000022F60E08FE60E94C40F82C0123008F07D
:108C2000DCC2E5E6CE2EE7E0DE2E00E0F9E1BF2E65
:108C3000ABE1AA2EF601C191D1916F01802F837013
:108C4000113041F19E01D7FF02C0215E3F4F75E018
:108C5000359527957A95E1F7AE01421B530B9A01A2
:108C6000D7FF02C0C158DF4FAE01440F452F441F4C
:108C7000550B420F531F602F66956695660F660F62
:108C8000660F685D8A9D802D112420E28F5D0E9411
:108C90003A6741C0043018F422E2922E02C09EE5E9
:108CA000992EF82EFF0CFF0CF80E9E01D7FF04C082
:108CB000222733272C1B3D0BB29EA001B39E500DE3
:108CC00011249A013E5FE32EE594E59459E15E1587
:108CD00014F489E1E82E25E543E366E26F0D87EEA3
:108CE000890D0E94AB6545E064E26F0D892D0E94FD
:108CF000DE651C161D0614F4939401C09E1867E2ED
:108D00006F0D4E2D892D0E94DB656F2D6B5D4E2DF5
:108D1000892D0E94DB650F5F083009F08BCF8CC274
:108D2000D03109F4A8C1D03209F078C08091080E82
:108D3000882329F124E040E160E081E00E941239BB
:108D400020E048E364E582E00E9412396BE178E0BC
:108D500080E10E9443658CE00E94811624E4AC010E
:108D600068E08EE40E943A670E948C16A5E0EA2E25
:108D700004E49C0146E060E280E00E94B220809121
:108D80008604882379F067E178E080E30E944365F8
:108D9000EE24E39404E420E04091EC0D68E280E1ED
:108DA0000E94741180918A04882381F043E158E085
:108DB00060E380E40E944965EE24E39404E421E04A
:108DC0004091F30D68E282E50E94741164E773E15B
:108DD00088E30E9443654091820D5091830D20E409
:108DE00068E382E10E943A6748E753E168E380E381
:108DF0000E9449654091840D5091850D20E468E3FF
:108E000082E4DF91CF911F910F91FF90EF90DF905F
:108E1000CF90BF90AF909F900C943A67D03309F0F9
:108E2000E6C08091080E811102C0C2E001C0C0E01E
:108E30006EE078E080E10E9443658AE10E9481163D
:108E40009C01442737FD4095542F6BEFE62EDC2F15
:108E5000D0610D2F60E180E30E942A664EE260E15E
:108E600080E30E94EA648BE10E9481169C01442702
:108E700037FD4095542F7CEFE72E60E188E40E9497
:108E80002A6669E078E088E10E94436587E10E94F4
:108E900081169C01442737FD4095542FEBEFEE2EB1
:108EA00068E180E30E942A664EE268E180E30E9466
:108EB000EA6488E10E9481169C01442737FD4095B1
:108EC000542FFCEFEF2E68E188E40E942A666BEFD6
:108ED00077E080E20E94436586E00E948116AC0143
:108EE00060E288E70E9449676DEE77E088E20E94C1
:108EF000436588E00E9481166C018091F50185FF31
:108F000012C068EE77E088E20E9443658DE492E04B
:108F1000A601489F6001499FD00C589FD00C112496
:108F2000CD2CDD24C6942C2FA60168E288E70E9490
:108F30003A678091080E882309F47EC186E00E947A
:108F40008116AC0160E280E30E94496788E00E94DC
:108F500081162091F50125FF0DC02DE432E0FC01C2
:108F6000E29FC001E39F900DF29F900D1124892F85
:108F700099278695AC0168E280E30E9449676CED11
:108F800077E080E30E94436560ED77E088E30E942C
:108F90004365C0E6DDE010E000E3D02E84E2F82E69
:108FA00080915F0D181708F047C1133021F4A8E332
:108FB000DA2EB4E2FB2E299180916304281710F079
:108FC00000E301C002E330E0220F331F442737FDE6
:108FD0004095542FF4E0EF2E6D2D8F2D0E942A66C0
:108FE000FAE2FF0E153009F427C11F5FD9CF40E325
:108FF00068E08FE30E94DE65CAE9D4E010E0888172
:109000008823B1F081500E94871F9C014881415004
:10901000612F6E70660F660F660F605F10FF02C0F3
:1090200080E401C080E07FE0E72E04E00E94B220EF
:109030001F5F2196163019F722E044E753E168E3F9
:1090400080E00E941D650091820D26E041E369E306
:109050008EE00E94726722E048E753E168E384E70C
:109060000E941D650091840D26E041E369E381E4DF
:109070000E947267E1C046E8A42E44E0B42E5FEE81
:10908000C52E5DE0D52EC0E0D0E010E0F501808176
:10909000882309F44CC049E553E168E1812F0E941F
:1090A0004965FC2E4C2F4F5C68E186E0810F0E94E1
:1090B000EA64EE24E39404E42C2FF6013397408114
:1090C00060E180E1810F0E947411FE01EE0FFF1F2D
:1090D000EE0FFF1FE757FB4F90819295969596955F
:1090E000937008E1902E910E933051F48C2F825F93
:1090F0000E948116AC0160E2892D0E9449670BC075
:10910000EE24E39400E02C2FF6013197408160E2D9
:10911000892D0E947411EE24E39400E42F2DF601B2
:10912000408160E284E2810F0E94741110E4219674
:10913000F4E0AF0EB11C27E0C20ED11CC230D10545
:1091400009F0A4CF8091080E882379F060E278E0DE
:1091500088E00E9443658DE00E948116082F26E07A
:1091600046E669E089E10E94726764E773E180E3A3
:109170000E9443654091FA0D50E024E468E280E1EA
:109180000E943A674091FC0D50E068E388E10E943C
:1091900049674091FD0D50E020E468E384E20E94BD
:1091A0003A6748E753E160E380E40E9449654091F3
:1091B000010E50E024E468E280E50E943A674091A5
:1091C000030E50E068E388E50E9449674091040E71
:1091D00050E020E468E384E614CE123019F50E94D2
:1091E000502B6091F607662329F0862F880F680FB1
:1091F000660F6D5F80E00E9435398091F6078F5FC2
:10920000682F660F680F660F81E0DF91CF911F9185
:109210000F91FF90EF90DF90CF90BF90AF909F9015
:109220000C9435394091D0075091D10704E024E0E7
:1092300068E28CE30E94C40FDF91CF911F910F91E0
:10924000FF90EF90DF90CF90BF90AF909F900895E8
:10925000982F80918B07292F281B19166CF4621701
:109260001CF4892F861B09C03AEF360F23172CF404
:10927000892F861B8A5F01C080E080938B07089549
:10928000BF92CF92DF92EF92FF920F931F93CF93F3
:10929000DF93C82E4EE0682F8BEE97E00E941826D1
:1092A00085E19FE00E947122182F8091FA070E94A9
:1092B000B60FEC0120E0488160E086E0810F0E945B
:1092C0006E10D090EB0766E08D2D0E94284918E0C3
:1092D000F12CBB24B39440918B074F0DEE24E39403
:1092E000D412E12C50E04F30510508F045C1FA018D
:1092F000E55AFF4F0C94FC7A6DE07FE0812F0E94CD
:1093000043652E2D20614981612F84E50E9439102B
:10931000EE2009F431C14CE261E089810E94E8133A
:1093200089832AC165E07FE0812F0E9443650DE7B4
:1093300023E84A81612F80E60E94CA218A831CC1EA
:109340008F8186FF03C04BEF5EE002C044EF5EE01A
:10935000612F8CE00E9449650DE723E84885612F65
:1093600080E60E94CA21888707C18F812E2D48EE92
:109370005EE0612F83FB882780F90E94942C9F81F7
:1093800080FB93F90DC08F812E2D4CED5EE0612F97
:1093900086FB882780F90E94942C9F8180FB96F998
:1093A0009F83EAC08F8181702E2D46ED5EE0612F94
:1093B0009B2D981B892F0E94942C9B2D981B8F818D
:1093C00090FB80F98F83D8C00F8107FB002700F93D
:1093D000002319F040ED5EE002C04AEC5EE02E2D65
:1093E000612F8CE00E942365EE2059F08F8187FB6E
:1093F000882780F961E00E94EB139F8180FB97F939
:109400009F838F8187FB882780F9081709F4B4C0F0
:109410001C82B2C08F8187FF09C004E62CE94C8111
:10942000612F80E60E94CA218C83A6C02E2D4C811C
:10943000612F82E10E941B2FEE2009F49DC046E1BE
:1094400060EF8C810E94E8138C8387300CF494C009
:1094500090E6C91291C087508093FB078CEE99E388
:109460000E94731B89C062EC7EE0812F0E944365DD
:109470000E2D2E2D4B81612F8EE40E94092F8B83A0
:109480007BC069EB7EE0812F0E9443650F810295CE
:10949000037049F0402F50E02E2D2064612F84E5A9
:1094A0000E943A6707C02E2D43E153E0612F8EE4FE
:1094B0000E942365EE2009F45FC063E0802F0E94C4
:1094C000EB1383708295807F9F819F7C1CC061EB32
:1094D0007EE0812F0E9443652F81269523700E2DFB
:1094E00047E95EE0612F8EE40E940F65EE2009F4EB
:1094F00043C08F81869562E083700E94EB13837076
:10950000880F9F81997F982B4BCF4D8142954F704B
:109510002BE83EE06E2D812F0E946E1E8295807F8B
:109520009D819F700BC04D814F7021E83EE06E2DF4
:10953000812F0E946E1E8F709D81907F982B9D833E
:109540001BC04E8142954F7025E73EE06E2D812F66
:109550000E946E1E8295807F9E819F700BC04E81FF
:109560004F702BE63EE06E2D812F0E946E1E8F7095
:109570009E81907F982B9E83F394185F87E0F8126A
:10958000AACEDF91CF911F910F91FF90EF90DF90C6
:10959000CF90BF9008957F928F929F92AF92BF928B
:1095A000CF92DF92EF92FF920F931F93CF93DF93AF
:1095B000C82F89EF91E10E94712240E1E42E0DE075
:1095C0002BE632E146E06C2F83EF97E00E940726FE
:1095D000E090F307EA9466E08E2D0E942849C03699
:1095E00011F0C43669F4E7FC0BC0E092FB078C2F46
:1095F0000E9412691092CB018CEE99E30E94731BBA
:10960000B12CC12C98E0D92EFF24E7FCF09425E082
:10961000A22E39E0932EC0918B07CB0D0C2F10E0BA
:10962000D1E0E016F10609F0D0E088248394C83038
:1096300028F4812C88E38D1528F45BC0E0E3ED1558
:1096400008F457C0C11002C0CD2E02C0CC24C39470
:109650002D2F46EF51E16D2D80E00E942365A8017A
:109660004F5F5F4FC93010F482E101C087E12D2FB9
:109670006D2D0E943A67882051F008501109909E84
:10968000E001919ED00D1124C950DC4F07C0A09E6F
:10969000E001A19ED00D1124C153DC4F8E018AE25E
:1096A000782EF80141918F01552747FD50956D2D7A
:1096B000872D0E944967F5E17F0E83E97812F1CF8B
:1096C00008E00D0D882079F025961AE2499155277A
:1096D00047FD5095602F812F0E9449671B5E1E3702
:1096E000A9F700E10D0DB394E7E0BE1611F0D02EFE
:1096F00092CFC11005C080918B078F5F80938B073D
:10970000DF91CF911F910F91FF90EF90DF90CF905D
:10971000BF90AF909F908F907F900895BF92CF920F
:10972000DF92EF92FF920F931F93CF93DF93C82F97
:109730008AE790E10E947122FAE0EF2E0DE02BE61D
:1097400032E14BE06C2F8EEE97E00E9407261091DD
:10975000EE07115066E0812F0E942849B82EC038CC
:1097600099F480E80E94126989E180938807193092
:1097700019F40E94E66905C0183018F4812F0E9480
:10978000536A81E00E948A73E8E0FE2EC12EDD2438
:10979000C7FCD09488E0B81205C080918807882360
:1097A00089F134C0CB2DD0E0CC16DD0611F401E1F7
:1097B00001C000E19E012F5F3F4F442737FD4095D8
:1097C000542F72E0E72E6F2D82E10E942A6680916D
:1097D0008807811104C021E0CC16DD0609F020E0E5
:1097E000FE01EE0FFF1FE158F34E459154916F2D8E
:1097F00088E10E94236588E0F80EB39480E4F812B3
:10980000C9CF4EC0DD24D394183009F0D12C6BE6BB
:1098100070E18F2D0E9443655AE5C52EC6E0D0E069
:10982000E0912205F0E0E95AFC4F449150E00C2E03
:1098300002C0559547950A94E2F7437055274A5957
:109840005F4E0D2D21E06F2D8C2D0E94ED6422972F
:1098500086E0C80E82E7C812E3CFDD2039F067E169
:10986000809122050E94F3138093220568E06F0D1A
:109870006933B0F480918807811103C021E0193069
:1098800009F020E042E550E186E0DF91CF911F91A1
:109890000F91FF90EF90DF90CF90BF900C942365D5
:1098A000DF91CF911F910F91FF90EF90DF90CF90BC
:1098B000BF9008952F923F924F925F926F927F9246
:1098C0008F929F92AF92BF92CF92DF92EF92FF92D0
:1098D0000F931F93CF93DF9300D000D0CDB7DEB7A7
:1098E000282E8DE09EE00E9471228091340788230B
:1098F00021F00E941230182F01C010E08091630700
:1099000081110BC0E09062070DE02BE632E144E0EC
:10991000622D8AEE97E00E9407266090EA07809108
:10992000CB01803621F08F3B31F08E32A1F4909143
:109930003407992319F0109234070DC090916307F2
:10994000911109C00E9412691092CB01611007C0E9
:109950001092340702C06620D9F3198202C081E058
:10996000898367E0862D0E942849382E80916307FD
:1099700081111092CB0180913407882369F0111670
:109980000CF4B1C11111B1C18091CB01823609F43F
:10999000AAC1833609F4A9C14424439411E0512C8F
:1099A000A32CB12C852D0E94B60F7C01311678F4C2
:1099B000612F70E06A197B096830710544F4660F05
:1099C000660F660F20E0442D81E00E946E109FE13B
:1099D000951508F4C8C0F701F081FA83F411C3C0EB
:1099E000C7010A969C838B83F52CCB80DC809AE0A0
:1099F000C91AD108311608F0A3C0812F90E08A1946
:109A00009B09883091050CF08CC0782E770C770C70
:109A1000770C80913407811113C0611211C0F0924C
:109A2000FA07EA81E093F807F981FF2359F01092D1
:109A3000350781E080936307EE24E394212C04C072
:109A4000E12C02C0EE24E3945F1459F0F601278163
:109A50002695237000E048E05EE0672D83E10E94D8
:109A60000F6520E1EB81FC8139974081672D80E310
:109A70000E9439100DE723E88B809C80F8E08F1A54
:109A80009108F4014081672D8DE20E94CA21F40102
:109A90008083EB81FC8137974081442329F020E0CB
:109AA000672D88E40E949010EB81FC8136974081FD
:109AB000442379F0F601878120E087FF06C044E661
:109AC000672D80E60E945B6404C0672D80E60E94DB
:109AD0001B2FF6018681811102C040E201C043E5DF
:109AE000F6018581882329F0433511F44AE201C04B
:109AF00044E4672D89E70E94EA6480913407882353
:109B0000F9F08091F9078F111BC020E046E6672D20
:109B100088E10E947165F092FA071093EA07612EBE
:109B20000FC0089769F480913407882349F0809129
:109B3000F9078F1105C08091EA078F5F8093EA07CC
:109B40001F5FF394F0E2FF1609F448C08B819C81FB
:109B50000A969C838B83FC013A9780819A818917AE
:109B600009F443CF3BC0611237C04092F8075092CE
:109B7000FA07662D6A19660F660F660F615029E0B5
:109B800049E180E00E944C67E981EE2329F10E94BF
:109B90007D2F811121C060E08091FA070E949F1EF5
:109BA0001092340780E499E40F900F900F900F907B
:109BB000DF91CF911F910F91FF90EF90DF90CF90A9
:109BC000BF90AF909F908F907F906F905F904F90DD
:109BD0003F902F900C94731B1F5FF52C4394F1E181
:109BE0004F1611F05F2CDECE80916307882309F4B5
:109BF00060C02092CB0165E082E492E10E94473090
:109C000084E00E941E30F82E00913507602F660F09
:109C1000660F660F685F20E044E288E10E9471658C
:109C200081E0F81235C0013079F40E947D2F811156
:109C30000DC08091FA078F5F8093FA0760E00E9461
:109C40009F1E1092340702C0023018F480E499E499
:109C50000EC08091FA07043069F480933607809132
:109C6000CB010E9412691092CB0185E99FE20E940C
:109C7000731B0BC0023031F48F5F8093FA0761E0F1
:109C80000E949F1E81E080933407109263070BC0EF
:109C900092E0F91208C0109263078091CB010E94F4
:109CA00012691092CB018091FA078093F907109204
:109CB0008A071150109362070F900F900F900F902A
:109CC000DF91CF911F910F91FF90EF90DF90CF9098
:109CD000BF90AF909F908F907F906F905F904F90CC
:109CE0003F902F90089561E001C060E08091FA07F5
:109CF0000E94392F51CE6F927F929F92BF92CF9246
:109D0000DF92EF92FF920F931F93CF93DF93D82EA2
:109D100080E99AE00E9471221FE1E12E06E02FE522
:109D200032E140E06D2D8DED97E00E940726109105
:109D3000DD07E090640767E0812F0E942849F82E34
:109D400088E1F81208C01B3110F48FEF01C081E0E8
:109D5000D8E1FD2EF80E91E6D916B1F09D1558F018
:109D600084E4D81661F18D1520F092E4D916E0F55F
:109D700041C085E406C094E6D91609F1D916A0F1D0
:109D800085E6D81659F036C080918A07882391F16C
:109D900010928A0781E60E9412692CC0113039F4B2
:109DA000EE2041F180918A07882321F104C0163109
:109DB00009F5EE20F9F08091640781500CC0113054
:109DC00069F498E09E15B0F080918A07882391F09D
:109DD000809164078F5F809364070CC0163151F443
:109DE00086E08E1538F0F4CF80918A07811102C089
:109DF00010926407F1107EC065E87AE088E00E9466
:109E00004365113031F480918A07811102C001E16C
:109E100001C000E12AE04AE255E068E082E40E94E5
:109E2000ED6480918A0781110BC08091870787FFBD
:109E300007C081E080938A07109287071092640719
:109E400080918A07882381F020918707332727FD97
:109E500030958E2D90E08217930734F410928A0784
:109E60001092870710926407113009F0A1C4809105
:109E70008A07882309F49CC480916407909187071E
:109E8000891B87FD03C08093640702C0109264079A
:109E9000809164078A301CF089E0809364071092F7
:109EA0008707CE2DD0E0C752DB4FFE01EF5AFF4FA0
:109EB00080810E94AE332091580130915901232BAB
:109EC00029F49D2D9F7D9254923018F461E40E94F4
:109ED000F3130E94BE33CF5ADF4F88839E2D990F14
:109EE0009E0D990F21E0482F68E082E4890F0E94BF
:109EF0005B645EC491E09F1548F1D8E0C0911C05F9
:109F0000C695C695C695C7706EE77AE08D2F0E94FC
:109F10004365123089F466E08C2F0E94F313C82F3A
:109F20008770880F880F880F90911C05977C982B5D
:109F300090931C0501E001C000E02C2F42E55AE09F
:109F40006D2F8CE50E940F65D85F04C082E0F81287
:109F500023C0D8E0C0912805C43008F0C4E067E40D
:109F60007AE08D2F0E944365133061F464E08C2FFA
:109F70000E94F313C82F843009F487E080932805EA
:109F800001E001C000E02C2F43E15AE06D2F82E494
:109F90000E940F65D85F04C093E0F91231C0D8E089
:109FA000C0913505C95F6CE07AE08D2F0E94436552
:109FB000143039F467E08C2F0E94F313C82F21E48A
:109FC00001C020E44C2F50E06D2F86E60E943A67D6
:109FD00040913505552747FD50952C2F332727FDF8
:109FE0003095275031094217530729F0C750C093C5
:109FF00035050E943614C8E0CD0FC93328F0DAC306
:10A0000084E0F8121EC0C8E06DEF79E08C2F0E944A
:10A010004365153051F444E661E0809126050E94C5
:10A02000F0138093260521E401C020E44091260529
:10A0300050E06C2F86E60E943A67C85FC93328F06B
:10A04000B9C395E0F9121DC0C8E06CEE79E08C2F21
:10A050000E944365163049F465E0809127050E940F
:10A06000F3138093270521E401C020E440912705E4
:10A0700050E06C2F86E60E943A67C85FC93328F02B
:10A0800099C386E0F81220C0C8E063EE79E08C2F17
:10A090000E944365173061F44DE26AE08091070544
:10A0A0000E94F013809307050E94E16721E401C03C
:10A0B00020E44091070550E06C2F86E60E943A6745
:10A0C000C85FC93328F076C397E0F9121DC0C8E015
:10A0D00063ED79E08C2F0E944365183051F448E716
:10A0E00068E2809108050E94F0138093080521E43E
:10A0F00001C020E4409108056C2F86E60E941E10E6
:10A10000C85FC93328F056C388E0F81222C0C8E0FF
:10A1100060EC79E08C2F0E944365193051F44EE6D3
:10A1200066EF80911E050E94F01380931E0521E0CA
:10A1300001C020E040911E05552747FD5095465F20
:10A140005F4F6C2F80E70E943A67C85FC93328F0E1
:10A1500031C399E0F91217C0C8E021E01A3009F0C4
:10A1600020E080911F054FEA59E06C2F81700E941A
:10A17000742C90911F0580FB90F990931F05C85F88
:10A18000C93328F017C38AE0F81218C0C8E021E0EC
:10A190001B3009F020E080911F0543EA59E06C2F45
:10A1A000869581700E94742C90911F0580FB91F917
:10A1B00090931F05C85FC93328F0FCC29BE0F912D9
:10A1C00019C0C8E021E01C3009F020E080911F0593
:10A1D00044E959E06C2F82FB882780F90E94742C97
:10A1E00090911F0580FB92F990931F05C85FC933BA
:10A1F00028F0E0C28CE0F81219C0C8E021E01D3060
:10A2000009F020E080911F0546E859E06C2F83FBA0
:10A21000882780F90E94742C90911F0580FB93F988
:10A2200090931F05C85FC93328F0C4C29DE0F9129E
:10A230001DC0C8E069E779E08C2F0E9443651E309D
:10A2400051F446E16AEE80910A050E94F013809372
:10A250000A0521E001C020E040910A056C2F80E64C
:10A260000E949010C85FC93350F0A4C28EE0F81667
:10A2700029F0D8E000E0C0E1BC2E4CC0C8E021E0ED
:10A280001F3009F020E08091250548E659E06C2F49
:10A2900086FB882780F90E94742C9091250580FB0D
:10A2A00096F990932505D8E0DC0FD93318F382C2D4
:10A2B000011133C068E579E08D2F0E9443650111DB
:10A2C0002FC0C09121051B112EC068E78C2F0E9462
:10A2D000F313C82F21E0CC2341F1206495E0C99FFE
:10A2E000A00111246D2F86E60E943A6743E76D2F87
:10A2F00080915D0C0E94EA6401111EC0C09321058B
:10A30000D85FD93308F056C281E08B0D0F5F8231E0
:10A31000B1F0B82EFB14C0F7CBCF68E479E0CCCF16
:10A32000C0912905D0CF20E0D6CF43E153E06D2F77
:10A3300086E60E942365E0CFC0932905E1CF81E145
:10A340008F15E0F021E0123109F020E080911F0527
:10A3500082958170C1E04AE359E06D2F9C2F981BD4
:10A36000892F0E94742CC81B80911F05C0FB84F9A3
:10A3700080931F05D85FD93308F01CC282E08B0D93
:10A38000F816D8F421E0181320E080912505829575
:10A390008170C1E04EE259E06D2F9C2F981B892FF0
:10A3A0000E94742CC81B80912505C0FB84F9809302
:10A3B0002505D85FD93308F0FDC183E08B0DF81671
:10A3C000D0F421E0181320E080911C058170C1E0D9
:10A3D0004DE159E06D2F9C2F981B892F0E94742C02
:10A3E000C81B80911C05C0FB80F980931C05D85FB9
:10A3F000D93308F0DFC184E08B0DF816D8F421E0E2
:10A40000181320E080911C0586958170C1E04AE612
:10A4100054E16D2F9C2F981B892F0E94742CC81B10
:10A4200080911C05C0FB81F980931C05D85FD9334E
:10A4300008F0C0C1B5E0CB2ECB0CFC1408F079C0FD
:10A4400062E179E08D2F0E944365ABE66A2EA3E1BD
:10A450007A2EC2E49924939480913405892101E0F5
:10A4600009F400E021E0A3016D2F8C2F0E94ED6420
:10A47000990CCA5F8FEF681A780AC23769F71C1106
:10A4800054C08091640790918707891B87FD03C0A2
:10A490008093640702C010926407809164078A3039
:10A4A0001CF089E080936407109287074E2D50E0DE
:10A4B00045595C4E8E2D880F8E0D880F02E021E0ED
:10A4C0006D2F8E5B0E94ED6490E6D91649F08EE602
:10A4D000D81631F08091580190915901892B29F1BA
:10A4E0008D2D0E94126910928A0721E030E002C08F
:10A4F000220F331FEA94E2F7409134054227C90145
:10A5000088739927892B19F44093340509C0842F47
:10A51000822319F0276C242301C0242B20933405B7
:10A5200081E00E94715F0E941060D85FD93308F00B
:10A5300041C186E08B0DF816E0F421E0181320E00D
:10A5400080911C0582FB882780F9C1E043E059E037
:10A550006D2F9C2F981B892F0E94742CC81B8091F3
:10A560001C05C0FB82F980931C05D85FD93308F025
:10A5700021C187E08B0DF816E0F421E0181320E0EC
:10A5800080911C0587FB882780F9C1E045EF58E0E2
:10A590006D2F9C2F981B892F0E94742CC81B8091B3
:10A5A0001C05C0FB87F980931C05D85FD93308F0E0
:10A5B00001C188E08B0DF816E0F421E0181320E0CB
:10A5C00080911F0585FB882780F9C1E04BEE58E09C
:10A5D0006D2F9C2F981B892F0E94742CC81B809173
:10A5E0001F05C0FB85F980931F05D85FD93308F09C
:10A5F000E1C089E08B0DF816B8F421E0181320E0D3
:10A600008091250587FB882780F94FED58E06D2F55
:10A610000E94742C9091250580FB97F99093250555
:10A62000D85FD93308F0C6C08AE08B0DF816E0F485
:10A6300021E0181320E080911F0586FB882780F910
:10A64000C1E047ED58E06D2F9C2F981B892F0E9489
:10A65000742CC81B80911F05C0FB86F980931F05D1
:10A66000D85FD93308F0A6C08BE08B0DF816B8F48C
:10A6700021E0181320E08091250549EC58E06D2F6A
:10A6800085FB882780F90E94742C9091250580FB1A
:10A6900095F990932505D85FD93308F08BC08CE0ED
:10A6A0008B0DF816A8F421E0181320E080913905ED
:10A6B0004FEB58E06D2F81700E94742C90913905FA
:10A6C00080FB90F990933905D85FD93308F072C0B8
:10A6D0008DE08B0DF816E0F4C0911F05C7FBCC2769
:10A6E000C0F921E0181320E04EEA58E06D2F8C2FBE
:10A6F0000E94742C90911F0580FB97F990931F0581
:10A700008170C8130E943D78D85FD93308F052C0D9
:10A710008EE0B80EFB1408F04DC049EA58E06D2FEA
:10A7200086E00E944965D83328F008E00D0F093310
:10A7300078F040C004E2C0E02C2F45E852E16D2FD4
:10A74000802F0E941664CF5F085EC430A9F7EDCF5A
:10A750001B1115C080918A07882399F063E08091CE
:10A760001D050E94F31390911D05891761F09091CA
:10A7700025059F779093250580931D0504C020E053
:10A7800003C021E001C022E040911D054F5C602F15
:10A7900082E10E945B64D4E2C0E0CF5F20E04C2FF6
:10A7A000602F8D2F0E943910D85EC430B1F702C0DF
:10A7B000D0E1A4CBDF91CF911F910F91FF90EF904B
:10A7C000DF90CF90BF909F907F906F9008958F9271
:10A7D0009F92AF92BF92CF92DF92EF92FF920F9330
:10A7E0001F93CF93DF93C82F89ED9FE00E947122C2
:10A7F0006CE0A62ECC24C39477EDE72E7FE0F72EF5
:10A800000DE02BE632E147E06C2F8CEE97E00E94E2
:10A810009023C090EC07CA94F090640766E08C2DFA
:10A820000E942849A82E18E0DD24C7FCD0942A2DC8
:10A8300030E0C216D30639F480918A07882329F0C4
:10A8400052E0B52E04C0B12C02C0BB24B394E90180
:10A85000CC0FDD1FC20FD31FC15CDB4F65ED7FE066
:10A86000812F0E94436588E08A1510F448E301C0F7
:10A8700041E34A0D612F85E00E94EA64FF2011F058
:10A8800000E001C00B2D2A812F704AE65FE0612FA6
:10A890008DE00E940F658A818F700E94A80F982E0C
:10A8A000811131C091E0F91611F020E001C02B2D8B
:10A8B0004881612F86E30E94391088818532B4F087
:10A8C0009BED892E880E6981882D0E94101F9C01A6
:10A8D00082E0F81611F000E001C00B2D82E0E82EB6
:10A8E000482D612F84E60E94B22073C092E0F916D1
:10A8F00011F020E001C02B2D4981552747FD5095CF
:10A90000612F83E664C081E0981216C0F81611F03A
:10A9100020E001C02B2D4881612F86E30E9490101A
:10A9200092E0F91611F020E001C02B2D4981612F32
:10A930008DE40E9490104DC082E0981217C091E003
:10A94000F91611F020E001C02B2D4881612F86E31C
:10A950000E94391082E0F81611F020E001C02B2D82
:10A960004981612F80E50E94391033C066E67FE09F
:10A97000812F0E944365488147FF03C0409580E2D4
:10A9800001C080E091E0F91202C02B2D01C020E04F
:10A99000282B552747FD50954F5F5F4F612F89E466
:10A9A0000E943A67498147FF03C0409580E201C099
:10A9B00080E092E0F91202C02B2D01C020E0282B8C
:10A9C000552747FD50954F5F5F4F612F8BE60E94E3
:10A9D0003A674A8142954F7049300CF04F5F83E0EF
:10A9E000F81611F020E001C02B2D612F88E60E949F
:10A9F000901080918A07811107C080915801909131
:10AA00005901892B09F467C0BB2009F464C091E0A7
:10AA1000F91639F1F916A0F082E0F81609F43EC0F3
:10AA200093E0F91258C08A816FE082958F700E947E
:10AA3000EB138295807F9A819F70982B9A834BC0ED
:10AA40008A816EE08F700E94EB138F709A81907FE5
:10AA5000982B9A830E94A80F9816E9F11882198200
:10AA60003AC081E0981681F0981648F092E0991665
:10AA700071F083E098122FC043E66EEC0AC065E4E3
:10AA800088810E94EB1308C046E16AEE02C045E4EB
:10AA900060E088810E94E81388831DC091E09916C8
:10AAA00071F0991648F082E0981661F093E09912DF
:10AAB00012C043E66EEC0BC04DE763E808C046E108
:10AAC0006AEE05C065E489810E94EB1303C08981A9
:10AAD0000E94E8138983A394185F103409F0A7CE6D
:10AAE000DF91CF911F910F91FF90EF90DF90CF906A
:10AAF000BF90AF909F908F900895AF92BF92CF92EA
:10AB0000DF92EF92FF920F931F93CF93DF93B82EB4
:10AB100089E99DE00E947122B3E1AB2ECDE0CC2EFD
:10AB2000DBE8ED2EDDE0FD2E0DE02BE632E140E02E
:10AB30006B2D88EE97E00E9490231091E807D0904B
:10AB4000640767E0812F0E942849C82F20910605DD
:10AB500030E02F5F3F4F442737FD4095542F02E0F0
:10AB6000E02E01E160E08AE20E942A66C1113BC04A
:10AB700066E87DE088E00E94436500E12AE049EE56
:10AB800051E068E082E40E94ED64113009F0A4C352
:10AB900029E040E467E080E40E944C678D2D880F37
:10ABA0008D0D880F20918A0746E068E08E5B0E9439
:10ABB000716580918A07882309F48EC3CD2DD0E07A
:10ABC000C751DE4F88810E94AE3361E40E94EB13CF
:10ABD0000E94BE339881981709F47EC3888382E06F
:10ABE0000E94715F79C3C23020F5C8E065E77DE05F
:10ABF0008C2F0E944365123081F420E6B21204C00B
:10AC00008091F3010E942E1461E38091F3010E9470
:10AC1000EB138093F30121E001C020E04091F301A8
:10AC200050E04C5F5E4F6C2F88E50E943A67C85F2A
:10AC300003C0C23091F4C8E063E573E18C2F0E9439
:10AC40004365133009F0A7C381E0D81247C3809150
:10AC50008A078111A2C301E0A1C3C330D1F4C8E0C7
:10AC60006DE67DE08C2F0E944365143051F449E37A
:10AC700067EC8091F4010E94E8138093F40141E0B5
:10AC800001C040E021E06C2F8CE30E94C210C85F3D
:10AC900003C0C430E1F4C8E064E67DE08C2F0E947C
:10ACA0004365153051F445E16BEE809164040E94D8
:10ACB000E8138093640441E001C040E022E06C2F7F
:10ACC0008CE30E94C210C85FC93320F069C3C5304D
:10ACD00021F5C8E063E573E18C2F0E9443651630CF
:10ACE00071F48091F50161E081700E94EB13909105
:10ACF000F50180FB90F99093F50101E001C000E0BF
:10AD00002091F50121704EE45DE06C2F8CE30E94F0
:10AD10000F65C85FC93320F043C3C630B9F4C8E03B
:10AD200021E0173009F020E08091FA0147E45DE06E
:10AD30006C2F81700E94942C9091FA0180FB90F905
:10AD40009093FA01C85FC93320F02AC3C730C1F419
:10AD5000C8E021E0183009F020E08091FA0140E4D9
:10AD60005DE06C2F829581700E94942C9091FA0185
:10AD700080FB94F99093FA01C85FC93318F010C3AF
:10AD8000C830E9F467E37DE08C2F0E9443651930F9
:10AD900049F464E08091FB010E94EB138093FB0176
:10ADA00001E001C000E02091FB0147E15DE06C2F74
:10ADB0008CE30E940F65C85FC93320F0F1C2C9302F
:10ADC000D1F4C8E06FE07DE08C2F0E94436521E064
:10ADD0001A3009F020E0022F4091FD016C2F86E32C
:10ADE0000E94092F8093FD01A8E0EA2EEC0E88E373
:10ADF0008E1530F4D5C2CA3009F050C0F8E0EF2EFD
:10AE000066E07DE08E2D0E944365ECE3CE2EC0E02F
:10AE1000D0E0DC1202C01B3061F02091FE0130E076
:10AE20000C2E02C0359527950A94E2F7022F017087
:10AE300001C002E0AE014250534F21E06E2D8C2D37
:10AE40000E94ED64219626E0C20E86E6C812E1CF8C
:10AE50001B30F9F420E6B21631F020915801309100
:10AE60005901232BB1F08B2D0E94126910928A0791
:10AE700021E030E00D2C01C0220F0A94EAF7809106
:10AE8000FE0182278093FE0182E00E94715F0E9492
:10AE90001060C8E0CE0DC93328F082C2CB3009F073
:10AEA000DAC0C8E068EF7CE08C2F0E9443651C305C
:10AEB00041F4D11006C080918A07882321F002E076
:10AEC00003C000E001C001E04091F80186E0489F26
:10AED000A00111244752534F26E06C2F84E20E94B8
:10AEE000ED648091F801882359F09DEF980F92301E
:10AEF000F0F56FEC7CE08C2F0E944365D8E406C02F
:10AF000063ED7CE08C2F0E944365DCE31C3049F448
:10AF100021E0D21206C080918A07882321F002E046
:10AF200003C000E001C001E02091F9012E5F41EB78
:10AF30005CE06C2F8D2F0E940F651C3049F482E07D
:10AF4000D81206C080918A07882321F022E003C02E
:10AF500020E001C021E04091FC0182E34802A00111
:10AF60001124445D5E4F6C2F88E28D0F1EC081302E
:10AF7000F1F46AEA7CE08C2F0E9443651C3049F4AE
:10AF800021E0D21206C080918A07882321F022E0B6
:10AF900003C020E001C021E04091F901552747FDA1
:10AFA00050954F5F5F4F6C2F8EE70E943A671C30C1
:10AFB00009F04DC080918A07811107C02091580186
:10AFC00030915901232B09F442C0D091F8018091AE
:10AFD000250585FF02C064E001C063E081E0D8166A
:10AFE00061F0D81620F022E0D216F1F02BC08D2FA0
:10AFF0000E94EB138093F80125C0DD2321F08DEF33
:10B000008D0F823038F444E06EEF8091F9010E9498
:10B01000E81307C0D130B1F46CE78091F9010E94C8
:10B02000EB138093F9010EC0DD2321F08DEF8D0F1E
:10B03000823040F44AE06CEF8091FC010E94E813FA
:10B040008093FC018091F8018D131092F901C85F83
:10B05000C93328F0A5C1CC3009F077C0C8E0809191
:10B06000F801882321F09DEF980F923010F56BE9DD
:10B070007CE08C2F0E9443651D3011F421E201C059
:10B0800020E24091020285E04802A00111244F51C4
:10B090005F4F6C2F8CE40E943A671D3009F051C05D
:10B0A00044E16CEE809102020E94E8138093020258
:10B0B00048C08130B9F4D1E01D3009F0D0E02D2F27
:10B0C00045E85CE06C2F80E00E942365DD23C9F138
:10B0D00020E8B21236C081E08093990C80E00E9493
:10B0E0008A732FC06CE77CE08C2F0E9443654091EF
:10B0F000F90147FD04C043301CF042E001C040E0CC
:10B100004093F9011D3031F480918A07882321F0A2
:10B1100002E003C000E001C001E089E04802A001B4
:10B120001124405A534F29E06C2F8CE30E94ED64A8
:10B130001D3039F462E08091F9010E94EB13809395
:10B14000F901C85FC93320F02BC1CD3051F5C8E0FB
:10B1500063E57CE08C2F0E9443651E3099F480915A
:10B16000FA0167E08295869587700E94EB138295BD
:10B17000880F807E9091FA019F71982B9093FA012D
:10B1800021E001C020E04091FA01429546954770C8
:10B190004F5C6C2F82E70E945B64C85FC93320F06C
:10B1A000FFC0CE3021F5C8E069E47CE08C2F0E941E
:10B1B00043651F3071F48091FF0161E081700E944E
:10B1C000EB139091FF0180FB90F99093FF0101E058
:10B1D00001C000E02091FF01217041E45CE06C2F90
:10B1E0008CE30E940F65C85FC93320F0D9C0CF300F
:10B1F000C1F4C8E021E0103109F020E08091FF01A6
:10B2000047E35CE06C2F869581700E94942C9091AE
:10B21000FF0180FB91F99093FF01C85FC93320F0D3
:10B22000BFC0C031C1F4C8E021E0113109F020E015
:10B230008091F5014FE25CE06C2F869581700E9451
:10B24000942C9091F50180FB91F99093F501C85FE2
:10B25000C93320F0A5C0C131C9F4C8E021E01231E2
:10B2600009F020E08091F50146E25CE06C2F82FB62
:10B27000882780F90E94942C9091F50180FB92F927
:10B280009093F501C85FC93328F08AC0C23109F034
:10B2900087C0C8E06AE17CE08C2F0E9443651331CF
:10B2A00049F464E6809199040E94EB138093990419
:10B2B00021E201C020E24091990450E06C2F8EE71A
:10B2C000DF91CF911F910F91FF90EF90DF90CF9082
:10B2D000BF90AF900C943A67C0E188CCD1105BC0AE
:10B2E00080918A0700E0882311F022E001C021E06C
:10B2F0004091F6015091F7016C2F87E40E94C40F32
:10B30000133009F046C080918A07811106C0209150
:10B31000580130915901232BE1F16CE370E08091E9
:10B32000F6019091F7010E94A77A962FD82FDD2081
:10B3300021F021E0D21691F02CC06BE3892F0E94FE
:10B34000EB132CE38202C00111248D0F911DD7FD58
:10B350009A959093F7018093F6011BC04EE361E04C
:10B3600082E08D0F0E94E813D81BDE5F2091F6016A
:10B370003091F7012D1B3109D7FD339537FD05C0FD
:10B380003093F7012093F60104C01092F701109258
:10B39000F601C85F65CC00E001C002E020E0A8CF64
:10B3A000DF91CF911F910F91FF90EF90DF90CF90A1
:10B3B000BF90AF900895AF92CF92EF92FF920F930C
:10B3C000CF93DF93C82F8EED9BE00E94712286E021
:10B3D000A82EC12C9DEDE92E9BE0F92E0DE02BE669
:10B3E00032E141E06C2F85EE97E00E949023C091FE
:10B3F000E50767E08C2F0E942849D091FF01D29584
:10B40000D695D77062ED7BE088E00E944365C1303D
:10B4100089F464E08D2F0E94EB13D82F982F92951A
:10B42000990F907E8091FF018F71892B8093FF018E
:10B4300001E001C000E02D2F42EB5BE068E084E515
:10B440000E940F6567EA7BE080E10E944365C2309D
:10B4500049F464E2809100020E94EB1380930002A1
:10B4600021E001C020E04091000260E184E50E94FB
:10B4700039106CE97BE088E10E944365C33049F4F0
:10B4800064E6809101020E94EB138093010221E4A3
:10B4900001C020E44091010250E068E184E50E948F
:10B4A0003A6721E0C43009F020E08091FF014EE8C6
:10B4B0005BE060E282FB882780F90E94D32E9091A6
:10B4C000FF0180FB92F99093FF0121E0C53009F064
:10B4D00020E08091FF0140E85BE068E283FB882781
:10B4E00080F90E94D32E9091FF0180FB93F99093F5
:10B4F000FF0121E0C63009F020E08091FF0142E722
:10B500005BE060E3829581700E94D32E9091FF01F1
:10B5100080FB94F99093FF01DF91CF910F91FF9001
:10B52000EF90CF90AF9008955F926F927F928F923D
:10B530009F92AF92BF92CF92DF92EF92FF920F93C2
:10B540001F93CF93DF93D82E8FEE91E10E9471224B
:10B55000B1E1AB2ECC24C394CDEEEC2EC1E1FC2E98
:10B560000DE02BE632E145E06D2D82EF97E00E9481
:10B570009023C090F207CA94B090640766E08C2DC7
:10B580000E942849982E80E8D81227C09FE09C1579
:10B5900020F14C2D552747FD5095FA01E919F10985
:10B5A000EE0FFF1FEB59F84F20813181B11015C00C
:10B5B00085E0849FF001859FF00D1124ED5BFC4F29
:10B5C0008281882319F031952195310934832383B1
:10B5D00082E00E94715F0E941060E8E0AE2EEC2CC9
:10B5E000FF24E7FCF09480E1981609F4BEC0892D91
:10B5F0000E94BD0FEC01092D10E0F801EE0FFF1FB6
:10B60000EB59F84F208131818A81EB81FC818823BD
:10B6100019F0F195E195F1092E1B3F0B233331050C
:10B620001CF081110AC09EC02E3C3F4F1CF48823A1
:10B6300021F098C06DE2862E02C05FE7852E9394BC
:10B6400020E0492D6A2D80E00E946E10482D6A2D61
:10B650008BE40E94EA648091FF0181FF03C04DE703
:10B66000642E02C034E6632E812C562C5194E016D1
:10B67000F10641F4B81006C080918A07811105C017
:10B6800021E004C020E0712C09C022E080918907EC
:10B690008823C9F37724739410926D0182E0881691
:10B6A00091F193E0891609F443C081E08816B1F066
:10B6B00020624B815C816A2D80E30E943A6777208B
:10B6C00009F446C022E048EE53E068E17CEF8B814C
:10B6D0009C810E9429139C838B833AC048814456E5
:10B6E000552747FD50956A2D88E40E943A677720D8
:10B6F00079F188818456888349E1652D0E94E81399
:10B700008C59888325C049814C59552747FD509550
:10B710006A2D86E60E943A677720D1F089818C599C
:10B720008983462D67EE0E94E8138456898310C0F2
:10B730004A816A2D8CE60E948423772049F061E0DB
:10B740008A810E94EB1391E0811101C090E09A83FD
:10B75000839494E089128BCF88E08A0D803491F134
:10B76000A82E41CF2EE7822E6ACFC1E090E1C91208
:10B77000C0E080918807811123C02C2F4CED51E14E
:10B780006A2D82E10E942365CC23E1F080E8D81283
:10B7900019C089E18093880780E80E941269DF91CF
:10B7A000CF911F910F91FF90EF90DF90CF90BF90BE
:10B7B000AF909F908F907F906F905F900C94AE436E
:10B7C00020E0DCCFDF91CF911F910F91FF90EF90A0
:10B7D000DF90CF90BF90AF909F908F907F906F90B1
:10B7E0005F9008956F927F928F929F92AF92BF92D7
:10B7F000CF92DF92EF92FF920F931F93CF93DF933D
:10B80000C82F82E490E10E94712241E1A42E52E00F
:10B81000C52E6FE3E62E60E1F62E0DE02BE632E159
:10B8200048E06C2F8DEE97E00E949023A090ED07EA
:10B83000AA949090640766E08A2D0E942849B82E49
:10B8400018E0CA2CDD24C7FCD094B11020C06FE2F0
:10B8500070E1812F0E944365A1100FC080918A077B
:10B86000882311F0C2E001C0C1E060E1809165046D
:10B870000E94EB138093650401C0C0E04091650411
:10B8800050E02C2F612F8CE60E943A675FC180E167
:10B890008B1508F45BC100E180916504081BEB2C5B
:10B8A000F12CE701CC0FDD1FCC59DB4F20E04B2DF5
:10B8B000612F80E00E946E100B1508F4C3C0812C2C
:10B8C000CE14DF0441F4981006C080918A078111DC
:10B8D00005C001E004C000E0712C07C002E08091C7
:10B8E00089078823C9F3772473948881811021C044
:10B8F000807C803421F0803821F446E503C041E4A7
:10B9000001C043E5202F612F8EE10E945B64772008
:10B9100009F493C0888162E082958695869583704C
:10B920000E94EB138295880F880F807C98819F730B
:10B9300030C091E0891230C0982F907C903819F077
:10B9400026E1622E02C099E1692E482F440F440F70
:10B950004595459547314CF029EE240F48E150E1DB
:10B96000612F8AE20E940F6505C0202F612F8AE2B5
:10B970000E949010772009F460C08881880F880F9A
:10B98000462D6AEE859585950E94E8138F73988100
:10B99000907C982B988351C0982F907C498190344B
:10B9A00091F447FD03C04F3024F401C040E0242F40
:10B9B00001C02FE0298341EF52E1612F80E60E9410
:10B9C0000F654FE017C0903841F5880F880F893513
:10B9D0009CF047FD04C040321CF040E201C040E052
:10B9E000498321E0240F40EE53E1612F80E60E945D
:10B9F0000F6540E260E01BC04F360CF04FE6498314
:10BA0000552747FD509540585F4F202F612F80E606
:10BA10000E943A674FE660E80AC0552747FD5095F7
:10BA2000202F612F80E60E943A674DE763E8772078
:10BA300021F089810E94E8138983839483E088122E
:10BA40003FCF84C065E170E1812F0E944365812C66
:10BA5000CE14DF0441F4981006C080918A0781114A
:10BA600005C001E004C000E0712C07C002E0809135
:10BA700089078823C9F3772473948881811013C0C0
:10BA8000482F4F71202F612F8EE10E949010772058
:10BA900009F458C0888165E18F710E94EB138F71A2
:10BAA0009881907E1CC091E089121CC0282F22959D
:10BAB0002695277049EE5FE0612F8CE30E940F65A9
:10BAC000772009F43FC0888166E08295869587706B
:10BAD0000E94EB138295880F807E98819F71982B2E
:10BAE000988330C082958695877090E0498106974B
:10BAF00074F0403208F040E2498321E0240F40EE28
:10BB000053E1612F80E60E940F6540E210C04B3F79
:10BB100038F450E0202F612F86E60E943A6706C075
:10BB2000485F202F612F84E50E94B2214FEF7720DC
:10BB300049F050E0898122E060E070E090E00E94EE
:10BB400029138983839483E0881282CFB394185F8A
:10BB5000103409F07ACEDF91CF911F910F91FF90B1
:10BB6000EF90DF90CF90BF90AF909F908F907F909D
:10BB70006F9008951F93CF93DF93EC011AE08881B3
:10BB80000E94AE330E94BE3389931150C1F7DF91FA
:10BB9000CF911F910895EAEDF4E080E090E02191CB
:10BBA0003191820F931F24E0E23FF207C1F708951D
:10BBB00081E6E9EDF4E0DF011D928A95E9F78AE07C
:10BBC0008093D90489E1809307058AE5809308056D
:10BBD00081E080931D05EAEDF4E020E032E080E8AA
:10BBE00091E02193319395878487938F828FB4E07E
:10BBF000E83EFB07B1F74AE050E065EB74E18AE20A
:10BC000095E00E94067B0E94CB5D90930505809392
:10BC100004050895EF920F931F93CF93C82F20EF41
:10BC200032E0E9EEF1E0DF01C9011D920197E9F789
:10BC30004AE050E06AEA74E1CF010E94067B8C2F53
:10BC400090E06AE070E001960E94A77A605D6093E0
:10BC5000EE01805D8093EF0180E00E94536A61E015
:10BC60006C0F88ECE82E00EF12E029EE31E042E0A4
:10BC700080E198E00E948463CF911F910F91EF9033
:10BC800008950F931F93CF93DF93EB01042F80311F
:10BC900038F561E0680F80E198E00E94BC6110E037
:10BCA000A80160E270E0CE010E94277B4AE050E0EC
:10BCB000BE0180E198E00E9440620A9789F480E129
:10BCC00098E00E94AE61C00FD11F009749F06AE072
:10BCD00070E00E94A77A805D8A93862F972FF5CF18
:10BCE000DF91CF911F910F9108958F5F0C94636145
:10BCF000CF93C82F8031C0F561E0680F80E198E0F4
:10BD00000E94BC6120EF32E0E9EEF1E0DF01C90101
:10BD10001D920197E9F740EF52E0BF0180E198E002
:10BD20000E9440628F3F910509F018F48C2F0E9409
:10BD30000A5E89EE91E00E94BA5D809191048111C2
:10BD400007C08091FA01869583708E5F809391047D
:10BD50000E9400390E9411148091590D80648093D3
:10BD6000590DCF910C943D78CF910895FF920F9388
:10BD70001F93CF93DF93CDB7DEB72F970FB6F8940D
:10BD8000DEBF0FBECDBF01E0080F102F1031C8F489
:10BD9000FF24F394F10E8F2D0E94636181110FC077
:10BDA000602F80E198E00E94BC6161E0610F28E5AE
:10BDB00032E042E087E098E00E94286306C01F2D31
:10BDC000E5CF103169F780E01AC04FE050E0BE01C6
:10BDD0006F5F7F4F80E198E00E94D961882351F026
:10BDE000482FBE016F5F7F4F87E098E00E94A562F9
:10BDF000A895EBCF87E098E00E94536381E02F96EF
:10BE00000FB6F894DEBF0FBECDBFDF91CF911F916B
:10BE10000F91FF900895EF920F931F93CF93DF93AD
:10BE20000E942261882381F10E94946087FD2CC0CA
:10BE300060E080E198E00E94BC6181E6E9EDF4E019
:10BE4000DF011D928A95E9F741E650E0BF0180E1EC
:10BE500098E00E9440628AE295E00E94BA5D80917B
:10BE6000D9048A3028F480919201816080939201F4
:10BE70008AE08093D904C0910405D09105050E9401
:10BE8000CB5DC817D90721F161E08AE994E10E94EE
:10BE90000E1B88E894E10E9498120E94FD600E94A7
:10BEA000D85D98ECE92E01E610E029ED34E041E0A0
:10BEB00060E080E198E00E9484638136910529F07A
:10BEC00060E089E794E10E940E1B80E00E940A5E18
:10BED00080910605DF91CF911F910F91EF900C9407
:10BEE000785E882379F090911B08982B90931B081B
:10BEF000F89480915F0C9091600C789490931A085C
:10BF0000809319080895EF920F931F93CF93409158
:10BF10001B08442309F47FC0811110C0F89480915C
:10BF20005F0C9091600C78942091190830911A0858
:10BF3000821B930B8436910508F46DC08091FD0738
:10BF4000811169C0C42FC47042FD02C081E001C0EC
:10BF500083E08093FD0710921B0840FF26C034E168
:10BF6000E32E01E610E029ED34E041E061E18EEFDF
:10BF700097E00E9484638136910519F461E180E0C5
:10BF800029C080910408823051F480911B0881609F
:10BF90002BC080910408823001F1C1113AC060E0E9
:10BFA00080EC94E10E940E1B34C041FF32C024E1BA
:10BFB000E22E00EF12E029EE31E042E061E18EEF87
:10BFC00097E00E948463803F924019F780910605B4
:10BFD00061E18F5F0E9471611CC080911B08C111DB
:10BFE00002C0826001C0866080931B08F894809133
:10BFF0005F0C9091600C78948456910990931A0884
:10C000008093190880919B0C833019F4A8951092A5
:10C010009B0C1092FD07CF911F910F91EF90089507
:10C0200080911B08882359F081E00E94835F8091F2
:10C030009B0C8330A9F7A89510929B0CF1CF089523
:10C0400040E450E060E070E08CE198E00C941F6800
:10C0500041E050E062E070E08EE198E00C941F68EF
:10C06000CF93DF931F92CDB7DEB7698390E1899FAD
:10C07000B001112441E050E0CE0101960E941F68FA
:10C080000F90DF91CF910895CF93DF931F92CDB79B
:10C09000DEB790E1899FB001112441E050E0CE016C
:10C0A00001960E942E7B89810F90DF91CF91089598
:10C0B000CF93DF93D82FC82F8C2F0E944460882302
:10C0C00029F08C2F0E944460C82FF6CF60911E0883
:10C0D0008C2F0E943060D0931E08DF91CF910C947A
:10C0E0002860CF93C0911E08CC2359F08C2F0E945A
:10C0F000446080931E080E94286060E08C2F0E949C
:10C1000030608C2FCF910895CF93DF9380911E08DC
:10C11000C0E0D0E0882321F02F960E944460FACF3F
:10C12000CE01DF91CF910895DF92EF92FF920F93AE
:10C130001F93CF93DF9380E091E0E9EEF1E0DF0120
:10C140009C011D9221503040E1F7C0E2D8E0F12C73
:10C1500034E1F31205C080911E080EE118E002C020
:10C160008E01888190E0E12CDD24D394DF0C0097D0
:10C1700001F19C01245031092C3F310530F4FC01C0
:10C18000E751FE4F2081222371F0EE2029F060E07C
:10C190008E2D0E94306004C0D8011C920E94206045
:10C1A00080E090E0E4CFD082E82E0E94446090E0EE
:10C1B000DECFF3942396B5E1FB12CACFC4E0D0E002
:10C1C000FE01E751FE4F8081811109C060911E0878
:10C1D0008C2F0E943060C0931E080E942860219618
:10C1E000C115F1E0DF0761F780E0DF91CF911F918A
:10C1F0000F91FF90EF90DF900895CF9380E4ECE1F2
:10C20000F8E0DF01982F1D929A95E9F796E0909358
:10C210001C0880931D0880E180931F0884E0C1E022
:10C22000C80F6C2F0E943060CF3F11F08C2FF7CFDA
:10C2300060E08FEF0E94306084E080931E08CF9111
:10C240000C942060CF93DF9340E450E060E070E016
:10C250008CE198E00E942E7B80911C08843031F59F
:10C2600080911D08803411F5C0911E08DC2FCC236D
:10C2700031F08C2F0E944460DC2FC82FF8CF80E86B
:10C28000C1E0C80F6C2F0E943060CF3F11F08C2F9F
:10C29000F7CF60E08FEF0E94306060E88D2F0E9442
:10C2A000306086E080931C080E94206080911C080A
:10C2B000863029F481E090911D08903409F080E0E7
:10C2C000DF91CF91089590E0FC01EE0FFF1FE80F82
:10C2D000F91FE45EF74F81E09481911101C080E085
:10C2E0000895CF93DF9390E0EC01CC0FDD1FC80FD2
:10C2F000D91FC45ED74F8C819D81AE8170E0FB0158
:10C30000EE0FFF1FE60FF71FE45EF74F2481358124
:10C3100046812C833D834E8384839583A683DF915E
:10C32000CF910C942060CF9390E09C01220F331F9B
:10C33000280F391FF901E45EF74FC481F901E05E6F
:10C34000F74F1082118212820E942060CC2321F0CC
:10C350008C2FCF910C945860CF910895FC0180816F
:10C3600090E0FC01EE0FFF1FE80FF91FEF5DF74FA4
:10C37000918180819F700895CF93DF93FC0160834A
:10C380001282118270E0CB01880F991F860F971FD0
:10C39000EC01C45ED74F2C81238314821582168250
:10C3A000FC01EE5DF74F808182958F70DF91CF9118
:10C3B0000895AF92BF92CF92DF92EF92FF920F93C8
:10C3C0001F93CF93DF931F92CDB7DEB78C01FC0193
:10C3D000808190E0FC01EE0FFF1FE80FF91FEF5D79
:10C3E000F74F80812181922F9F70F8012181328146
:10C3F000821B930B7A018417950708F47C015B017B
:10C400006701C114D10429F1F8018381882309F15E
:10C4100064816F5F648370E0F0E18F9F600D711D38
:10C42000112441E050E0CE0101960E942E7B8981CB
:10C43000F50181935F01F80184818F3030F014821F
:10C4400083810E944460F8018383F1E0CF1AD10810
:10C45000D8CFF801818192818E0D9F1D8C199D0985
:10C46000928381838E2D8C190F90DF91CF911F9134
:10C470000F91FF90EF90DF90CF90BF90AF90089515
:10C480007F928F929F92AF92BF92CF92DF92EF9264
:10C49000FF920F931F93CF93DF934C016B018A019F
:10C4A000C0E0D0E05C0125E0A20EB11CC017D107AE
:10C4B000E8F5F40185818F7781F0F4014581F42F4F
:10C4C000FF777F2E2F2F30E0C8018C1B9D0B82172A
:10C4D000930760F4702E7C1A09C041E050E0B5016A
:10C4E000C4010E94D961813041F320C0E72CF12CB6
:10C4F000C6018C0F9D1F47FF06C0A70160E070E0DA
:10C500000E94277B0CC0A701BC01C4010E94D96115
:10C51000871529F0FE01E80FF11DCF0108C0CE0DEF
:10C52000DF1DF401858187198583C0CFCE01DF919E
:10C53000CF911F910F91FF90EF90DF90CF90BF9020
:10C54000AF909F908F907F900895AF92BF92CF92BF
:10C55000DF92EF92FF920F931F93CF93DF93EC0143
:10C560008B01D42E8B81811111C089819A81892BF5
:10C5700069F4E880F12C0E9471608B83F701EE0F63
:10C58000FF1FEE0DFF1DE45EF74F8483CD2C8FE07F
:10C59000A82ECC2009F445C02F813885F8948091CD
:10C5A0005F0C9091600C7894281B390B37FF02C008
:10C5B00082E004C08B81811103C081E08E8331C091
:10C5C0009C819F3078F01C820E944460811106C0DB
:10C5D0000E947160682F8B810E9430608B810E9465
:10C5E00044608B838B81882341F36C819A2D961B49
:10C5F000BC2C9C1508F4B92EEB2CF12C70E090E1CA
:10C60000899F600D711D11246F5F7F4FA701C801C5
:10C610000E941F680E0D1F1D8C818B0D8C83CB1803
:10C62000B8CF6D2D70E06C19710929813A81260F00
:10C63000371F3A8329838D2D8C19DF91CF911F915C
:10C640000F91FF90EF90DF90CF90BF90AF90089543
:10C65000EF92FF920F931F93CF93DF93EC01F62E8F
:10C66000E42E89010E94BC616F2D70E0FB01EE0F8A
:10C67000FF1FE60FF71FEF5DF74F1082E29430EFD8
:10C68000E322E182F89440915F0C5091600C789421
:10C69000400F511F58874F83DF91CF911F910F910A
:10C6A000FF90EF9008951F93CF93DF93EC01888163
:10C6B00090E0FC01EE0FFF1FE80FF91FEF5DF74F51
:10C6C000898180839A819F708181807F892B81837A
:10C6D0008B81882329F00E944460182F81110BC0A0
:10C6E00010E00E942060112359F0812FDF91CF913B
:10C6F0001F910C94586060E08B810E943060F1CFF4
:10C70000DF91CF911F9108957F928F929F92AF9268
:10C71000BF92CF92DF92EF92FF920F931F93CF932E
:10C72000DF931F92CDB7DEB76C0159012E2D30E09B
:10C730000E94286319824501E12CF12C772473941F
:10C74000F40181914F019981811108C071104EC08F
:10C750008081811105C0772473941CC071100AC0B8
:10C7600080E09F3718F4E016F10679F5772089F01C
:10C77000782E01C0712C992341F19068998341E092
:10C78000BE016F5F7F4FC6010E94A5628130E1F05C
:10C7900027C0782E9923C9F041E0BE016F5F7F4F1B
:10C7A000C6010E94A5628130D9F44981B701641B9A
:10C7B00071096A0D7B1DC6010E94A56299818917C6
:10C7C00019F0981B99830CC0198289818F5F898326
:10C7D000FFEFEF1AFF0A0E151F0508F0B1CF08C0D2
:10C7E00089818F778701081B110902C0872DB9CF76
:10C7F000C6010E945363C8010F90DF91CF911F9132
:10C800000F91FF90EF90DF90CF90BF90AF909F90EF
:10C810008F907F90089580E094E0EDE5F8E0DF01EF
:10C820009C011D9221503040E1F70895FF920F9333
:10C830001F93CF93DF93FA0174913196A491B0E0E6
:10C84000179693E0B595A7959A95E1F71A2FDA0117
:10C850001396FA0132964491249FA00DB11D112424
:10C8600066956695669590E0F0E86F9F800D911D46
:10C87000112420E030E060E0835A974F472F50E0CA
:10C88000611798F40A2FEC01C20FD31FFD01FE2E91
:10C89000F01AF71620F4F490F9923196F8CFA40F1D
:10C8A000B51F6F5F20583F4FEBCFDF91CF911F91A6
:10C8B0000F91FF900895CF93DF93382F46312CF4DA
:10C8C000842F880F840F880F82C086E0830F20FD9D
:10C8D00008C021FD02C090E005C090915E0C96FF5B
:10C8E000FACF91E0669566956695A32FB0E050E883
:10C8F000659FA00DB11D1124A35AB74F22FF40C060
:10C900004E3211F08CE0830F24ED240F2F3010F401
:10C910004B5211C02FEB240F2A3110F441530BC09E
:10C920002FE9240F2A3110F4465305C04F3511F476
:10C930004AE201C040E0E4E14E9FA00111244452CC
:10C940005B4E6BE062302CF0FA0174913A96E49100
:10C9500002C070E0E0E04F5F5F4F992311F07095E7
:10C96000E0959D012F573F4F2D553C4030F47C936F
:10C97000ED01C058DF4FE8831196615018F727C0CA
:10C9800023FF07C0892F81958D9385E0830F31E0C8
:10C9900001C030E025E04202F0011124ED55F64ED1
:10C9A00025E04491332311F0243039F05CE0AD35BB
:10C9B000B50718F4911140954D93215031962111EE
:10C9C000F0CFECE0AD35BE0710F491959C93DF916C
:10C9D000CF91089520E00C945B64EF92FF920F9347
:10C9E0001F93CF93DF93F62E122F902F9071E92E85
:10C9F000EA01112369F0EE2011F0488102C0FE0126
:10CA00004491202F6F2D0E945B6411502196F1CF2D
:10CA1000DF91CF911F910F91FF90EF9008950F93A9
:10CA2000FA0194914F5F5F4F929F400D511D112469
:10CA3000292F0E94ED640F9108950F9300E00E944A
:10CA4000ED640F910895FF920F931F93CF93DF939F
:10CA5000062F122F922F9071F92EFA01FF2011F05C
:10CA6000408101C04491EF012196442331F0212FF0
:10CA7000602F0E945B64FE01F1CFDF91CF911F9187
:10CA80000F91FF900895AB0120E0682F80E00C9497
:10CA9000236520E00C942365FF920F931F93CF939F
:10CAA000DF93082FF62EEA0114E1180F15504C2FD2
:10CAB0004F704A301CF0495C28E002C0405D20E025
:10CAC0006F2D812F0E945B6424E0D695C7952A952F
:10CAD000E1F71013EBCFDF91CF911F910F91FF90F2
:10CAE0000895222321F090915E0C96FD0895480F41
:10CAF000669566956695E82FF0E090E8699FE00DF1
:10CB0000F11D1124E35AF74F8E1B982F9E0F941797
:10CB100020F4908190959193F8CF0895962F969553
:10CB200096959695E82FF0E080E8989FE00DF11D2E
:10CB30001124E35AF74F8CE0ED35F80758F467708D
:10CB400081E090E0062E01C0880F0A94EAF79081F8
:10CB500098279083089547FF02C0840F4195962F30
:10CB6000969596959695E82FF0E080E8989FE00DD1
:10CB7000F11D1124E35AF74F677031E001C0330F04
:10CB80006A95EAF74423B1F08CE0ED35F80790F4AC
:10CB9000822F90E020FF08C02081232720839595D5
:10CBA0008795282F206803C095958795282F415099
:10CBB0003196E8CF08952FEF0C94AB65962F96959C
:10CBC00096959695282F30E0F90180E8989FE00D22
:10CBD000F11D1124E35AF74F962F940F96959695D1
:10CBE000969580E8989F200D311D1124235A374FC8
:10CBF000862F8770A1E0B0E001C0AA0F8A95EAF7FE
:10CC0000A1958081A827A083E217F30750F4E0588C
:10CC1000FF4F8CE0ED35F807E0F49081909590831C
:10CC2000F3CF8CE0ED35F807A0F4842F992787FD2A
:10CC30009095860F911D68E070E00E94A77A21E030
:10CC400030E001C0220F8A95EAF721958081822782
:10CC5000808308953F924F925F926F927F928F925E
:10CC60009F92AF92BF92CF92DF92EF92FF920F937B
:10CC70001F93CF93DF93182FB62E802F05FF04C08C
:10CC800004FF04C002E003C000E001C001E0982FEF
:10CC90009F77C92EE7FE04C0E1946624639401C027
:10CCA000612C57FF0AC050954095309521953F4F14
:10CCB0004F4F5F4F7724739401C0712C82FF06C0E1
:10CCC0009CE090935D0CCAE0DC2E05C096E090934A
:10CCD0005D0CB5E0DB2E86FF28C071101D0D283ECF
:10CCE00083E038074105510514F01D0D05C02436B9
:10CCF00031054105510514F01D0D05C02A303105DF
:10CD0000410551050CF01D0D002381F0023031F476
:10CD100024363105410551054CF41D0D2A303105ED
:10CD2000410551051CF41D0D01C01D1980915D0CBC
:10CD3000810F80935D0C023011F490EFC90E8824AE
:10CD40008394F2E09F2EA12CFF24E7FCF094A6E050
:10CD50005A2E5B0CE82DF0E0EE16FF060CF460C0D6
:10CD60006AE070E0C9010E94A77A382EEB01E0E387
:10CD70004E2E480E2C2D442D6B2D812F0E945B646E
:10CD8000081131C0C2FE1AC08FEF830D833008F442
:10CD90009394CE016AE070E00E94A77A823011F08D
:10CDA0008430E9F484E3481204C0AA24A394A10EB9
:10CDB00017C0AA24AA94A10E939412C07EEF472E06
:10CDC000410E8FEF810FC0FE05C047E06B2D0E9422
:10CDD000DE6503C0652D0E948E65142D01C0A12E55
:10CDE000209709F000E09E01442737FD4095542F1D
:10CDF000211531054105510581F4002331F0023040
:10CE000059F491E0981540F008C0C4FE09C06110C3
:10CE100004C080EFC80E01C000E01D1983949ACFB2
:10CE2000AA2061F0492D6CE06B0D8A2D0E94DB6514
:10CE3000492D6DE06B0D8A2D0E94DB65772039F05E
:10CE40002C2D4DE26B2D812F8D190E945B6480E0AB
:10CE5000DF91CF911F910F91FF90EF90DF90CF90D6
:10CE6000BF90AF909F908F907F906F905F904F900A
:10CE70003F900895EF920F93022F9A01442737FDB8
:10CE80004095542F95E0E92E0E942A660F91EF906D
:10CE9000089520E00C943A670F931F93CF93DF938C
:10CEA000182FC62F042FD22F422F0E94DE6502308A
:10CEB00038F04D2F6C2F8FEF800F810F0E94DE65B1
:10CEC00002501F5F6FEF6C0F6D0F402F812F0E947C
:10CED000DB65402F6C2F812FDF91CF911F910F9138
:10CEE0000C94DB650F931F93CF93DF93182FC62FFE
:10CEF000D22FE42FF0E03297053608F004E60E9FBB
:10CF0000C0010F9F900D112464E670E00E94A77A83
:10CF1000062F2D2F6C2F812F0E944C67002369F064
:10CF2000D150DC0FCF5F1F5FCD1738F4402F6C2F2F
:10CF3000812F0E94DB65CF5FF7CFDF91CF911F91EB
:10CF40000F910895A998AB98AC988BBBAD9AAD980A
:10CF5000AB9AA99A0895CF93DF9381E080935C0800
:10CF6000AA982AE02A95F1F700C0AA9A8CED95E0DC
:10CF7000E5E0EA95F1F7000001970097C9F7C0EDE9
:10CF8000D4E1FE0184910E94A2672196F4E1CC3D98
:10CF9000DF07B9F782E28093070510925C08DF9102
:10CFA000CF910895CF93C82F81E080935C0881E8EA
:10CFB0000E94A2678C2F0E94A26710925C08CF91FA
:10CFC0000895809107050C94D2671F93CF93DF9348
:10CFD00081E080935C0810E0CDE5D8E084E00E9419
:10CFE000A26780E10E94A267812F806B0E94A267E6
:10CFF000A998AB9AAC98FE01CE0180589F4F208132
:10D000002BBBAD9AAD9821812BBBAD9AAD982281F7
:10D010002BBBAD9AAD9823812BBBAD9AAD983496BE
:10D02000E817F90761F7EF01AB9AA99A1F5F18306B
:10D03000A9F610925C08DF91CF911F910895BF92DD
:10D04000CF92DF92EF92FF920F931F93CF93DF93D4
:10D050007B018A01080F191FEC01E81AF90A670120
:10D06000CC0EDD1EC017D107C1F0B9908091FD072D
:10D070008270E19B05C08823E1F30E94B11BF6CFCB
:10D08000DFBACEBAE09A8DB3B81649F3BDBA8FB7FE
:10D09000F894E29AE19A8FBFE2CFDF91CF911F918E
:10D0A0000F91FF90EF90DF90CF90BF900895809107
:10D0B0008E0C10928E0C0895FC0180818F70880F69
:10D0C000611181608F709081907F982B9083818116
:10D0D0008F5F81838281882351F09F7041F4833672
:10D0E00021F0842F806280938E0C118212828281C3
:10D0F000883069F148F4813091F188F0823039F15B
:10D10000843009F03FC023C08F35C1F018F480315E
:10D11000F1F00895813649F0823671F108958081E9
:10D120008F708F3079F581E62BC0406640938E0C6E
:10D130001092700610926F068FE522C081818032B6
:10D1400011F4406816C08832E9F480E119C0918179
:10D15000903328F090E095958795828311828281A3
:10D1600090E00197218130E082239323892B51F4B1
:10D17000406440938E0C08958181803418F088E0DB
:10D1800082831182089540916300282F30E02F3070
:10D1900031056CF4F901EE0FFF1FE20FF31FEF5999
:10D1A000F34F90819F7081E09F3051F52AC090E04D
:10D1B000FC013F97E930F10518F5E659FF4F0C9453
:10D1C000FC7A91B1947019C093B3907816C0942FE3
:10D1D000917013C0942F909598700FC043FF10C0AA
:10D1E00091B102C091B19095907407C091B19071C6
:10D1F00004C093B3F9CF91B1907281E0911101C055
:10D2000080E008958F7090E08F30910551F0FC011F
:10D21000EE0FFF1FE80FF91FEF59F34F82E68283ED
:10D22000118208958F7090E08F30910549F0FC01D4
:10D23000EE0FFF1FE80FF91FEF59F34F83E68283CC
:10D240000895EF92FF920F931F93CF93DF938091F6
:10D250005F0C9091600C01969093600C80935F0C32
:10D2600080935E0C96B3909580918F0C882321F06B
:10D27000282F2877292349F4892F807609F050C078
:10D2800093FD4AC094FF4AC080E1182F166019230D
:10D2900080938F0CC1E6DCE0F12C11FB662760F96E
:10D2A0004F2DCE010E945C68F3941695239686E07C
:10D2B000F812F3CFE0B2E094C3E2DCE100E010E06A
:10D2C000FC1AFE0184914C2F4F0D8E2161E009F470
:10D2D00060E0C8018D58934F0E945C6821960D5FF5
:10D2E0001F4F0831110569F79091D00161E0C92FF6
:10D2F000C07295FF60E04EE08BE89CE00E945C68A5
:10D3000086B390E0809590958E7799278C2B51F07D
:10D3100089E080936C0106C088E0B7CF80E0B5CF8C
:10D3200080E6B3CFDF91CF911F910F91FF90EF90E7
:10D330000895EF92FF920F931F93CF93DF93F82EF0
:10D3400080E04AE0282F30E0429FF001439FF00D3B
:10D350001124E751FE4F928DF91650F5803261F19C
:10D360008AE0E82EE29E8001E39E100D1124E80180
:10D37000CD5FDD4F6FE170E0621B730BE69EA00195
:10D38000E79E500D11242F5F3F4FE29EC001E39EA8
:10D39000900D1124BE018D5F9D4F0E94157BFE01F3
:10D3A0001192EA94E9F7F801E751FE4FF28E06C0B8
:10D3B0009923A1F28F5FC6CFC3E0D2E0CE01DF9107
:10D3C000CF911F910F91FF90EF90089580E491E02D
:10D3D000E3E0F2E0DF019C011D9221503040E1F7D3
:10D3E000089588E2EFECF3E0DF011D928A95E9F7FA
:10D3F00088E4E7EFF3E0DF011D928A95E9F70895ED
:10D40000FB018830A8F029E0829FC00111248751D8
:10D410009E4F20E030E04191DC01A20FB31FAA53E0
:10D42000BE4F4C932F5F3F4F29303105A1F7089530
:10D4300025E0829FC001112487519E4F20E030E0FB
:10D440004191DC01A20FB31FAA51BE4F4C932F5F35
:10D450003F4F25303105A1F7089590E00197FC0179
:10D46000EE0FFF1FE80FF91FDF01AF5BBB4F6F70BF
:10D470008C91807F862B8C93E751FE4FDF01AA5A57
:10D48000BD4F4C93E95AFD4F2083089590911D059F
:10D49000E82FF0E084E0989FE00DF11D1124E250A8
:10D4A000FD4F849108958F929F92AF92BF92CF9239
:10D4B000DF92EF92FF920F931F93CF93DF93CDB73D
:10D4C000DEB76D970FB6F894DEBF0FBECDBFF82E56
:10D4D00085E0E7E2F1E0DE01559601900D928A9534
:10D4E000E1F785E0ECE2F1E0DE01509601900D926B
:10D4F0008A95E1F785E0E1E3F1E0DE011B9601901A
:10D500000D928A95E1F785E0E6E3F1E0DE011696FB
:10D5100001900D928A95E1F785E0EBE3F1E0DE0101
:10D52000119601900D928A95E1F71A8E1B8E1C8E32
:10D530001D8EE0912205F0E0E95AFC4F46E050E0F4
:10D54000A1E0E4910E2F10E021E030E0C801042EAC
:10D5500002C0959587950A94E2F783709927BC01DC
:10D560006F5F7F4FEAE1F0E0EC0FFD1F8E0F9F1F12
:10D570006217730711F4FC01A0832F5F3F4F253022
:10D580003105B1F7AF5F42505109A530E9F6F1100E
:10D5900028C00E94E6698A8D0E9499698C0181E009
:10D5A0000E94466AF801818354E6F52EF2828B8D43
:10D5B0000E9499698C0182E00E94466AF801818389
:10D5C000F2828C8D0E9499698C0183E00E94466AE8
:10D5D000F8018183F2828D8D0E9499698C0184E02B
:10D5E0008AC0F1E0FF120EC08C8D0E949969FC0187
:10D5F00088E081838CE98283F3828781897F8460DC
:10D600008783F2C182E0F81249C08C8D0E9499692B
:10D61000FC0118E011833CE9E32EE28285E183837B
:10D620008781897F846087838EE00E94996902E206
:10D63000FC01018344E6F42EF2828EE00E94996997
:10D64000FC011183E28284E183838781897F846086
:10D6500087838EE00E949969FC011183F28281E048
:10D6600083838781897F8460878383E00E94466A01
:10D6700090915F04907F926090935F0480935D042B
:10D680008DE980935E0480916204807F8160809345
:10D6900062040093600410926104A6C1F3E0FF12DB
:10D6A00030C00E94E669EA8C8E2D0E9499698C0137
:10D6B00081E00E94466AF801818324E6F22EF2821C
:10D6C0008E2D0E9499698C0182E00E94466AF801C1
:10D6D00081838CE98283EB8C8E2D0E9499698C0169
:10D6E00081E00E94466AF8018183F2828E2D0E94B9
:10D6F00099698C0182E00E94466AF8018183F28276
:10D7000073C1F4E0FF1230C00E94E669EB8C8E2DED
:10D710000E9499698C0182E00E94466AF801818327
:10D7200094E6F92EF2828E2D0E9499698C0184E094
:10D730000E94466AF8018183F282ED8C8E2D0E9450
:10D7400099698C0182E00E94466AF8018183F28225
:10D750008E2D0E9499698C0184E00E94466AF8012E
:10D7600081838CE9828340C1F5E0FF12D1C00E9421
:10D77000E6690E94F16981E00E9499695AE0B52E3C
:10D78000FC01B18264E6D62ED28282E00E949969C1
:10D790007BE0C72EFC01C182D28283E00E9499699E
:10D7A000ECE0EE2EFC01E182D28284E00E949969D5
:10D7B0008C0181E00E94466AF8018183D28285E073
:10D7C0000E9499698C0183E00E94466AF801818376
:10D7D000D282A4E0AA2EA38287E08483878181601D
:10D7E000878385E00E9499698C0183E00E94466AE4
:10D7F000F8018183D282F382B8E08B2E8482878104
:10D800008160878385E00E9499698C0183E00E9492
:10D81000466AF8018183D28216E0D12ED38209E0D4
:10D82000902E948287818160878385E00E94996928
:10D83000FC0181828CE9828381E083838781897FF7
:10D840008460878386E00E949969FC0191828EE161
:10D85000828388EF83838BE00E9499698C0183E047
:10D860000E94466AF801818386E4982E9282A38200
:10D87000B4828781816087838BE00E9499698C01E3
:10D8800083E00E94466AF80181839282F382C48217
:10D890008781816087838BE00E9499698C0183E096
:10D8A0000E94466AF80181839282D382E482878152
:10D8B000816087838091FF018F7180628093FF0177
:10D8C0008FE180930002BE016B5E7F4F80E00E947B
:10D8D000006ABE01605F7F4F81E00E94006ABE0166
:10D8E000655F7F4F82E00E94006ABE016A5F7F4FE2
:10D8F00083E00E94006ABE016F5F7F4F84E00E9458
:10D90000006ABE016F5F7F4F85E00E94006A6CC0B5
:10D91000F6E0FF1216C086E00E949969FC01F182D0
:10D9200082E3828388EF838314E6108786E00E9477
:10D930009969FC01F1828EEC828388E083831087F1
:10D9400053C087E0F81250C08FE00E949969FC0133
:10D9500014E2118384E6828388E8868380E10E9452
:10D960009969FC0189E081830EE602838AE0838362
:10D9700080E10E949969FC0148E0F42EF18282E97D
:10D9800082838BE083838781897F8460878380E1C2
:10D990000E949969FC01F18202838CE08383878174
:10D9A000897F8460878380914104807F8B6080932E
:10D9B000410493E290933F04109340048091440407
:10D9C000807F8160809344049093420489E6809331
:10D9D000430480914704807F826080934704909342
:10D9E000450487E98093460482E00E94715F0E94AB
:10D9F00010606D960FB6F894DEBF0FBECDBFDF91FD
:10DA0000CF911F910F91FF90EF90DF90CF90BF903B
:10DA1000AF909F908F9008950F931F93CF93DF93B4
:10DA20009091FF0191FF03C060E075E002C060E0EB
:10DA300074E01091FA01129516951770882331F051
:10DA4000A4EEBCE0833021F420E103C0ACE9BCE0EB
:10DA500028E09091F901990F910F920F4091FC01EC
:10DA600024E64202A0011124485A5D4F00910202AF
:10DA7000E8EEF3E09F010203E001039FD00D1124C3
:10DA80009E0128533045241B350BFD01882339F0B6
:10DA900032964D935C93833011F418EF190FCC2715
:10DAA000DD27C61BD70B1917F0F4A12FB0E0AA0F82
:10DAB000BB1FAB59B84F0D90BC91A02D6A177B07C7
:10DAC0000CF4DB01AC17BD070CF4DE01A854B44F15
:10DAD0002A1B3B0BA41BB50BB183A083538342834A
:10DAE0001F5F3496E0CF31832083DF01882371F0FC
:10DAF0001296285E33403093980C2093970C1D9219
:10DB00001C92DF91CF911F910F910895149653832A
:10DB10004283F5CFE0912501F091260129E090E1C3
:10DB200030E0482F4170341302C0905F04C0915020
:10DB30009083319690E186958068215011F0342FC2
:10DB4000F0CF915F9193F0932601E0932501089522
:10DB50001F93CF93DF93182F2CE93CE030932601DD
:10DB600020932501C09113018C2F877461F080915F
:10DB7000F901882321F0813021F4C0E906C0C0E812
:10DB800004C0C8E902C0C7FF06C087E10E94C3689D
:10DB9000882309F45AC0C7FD5AC040E060E085E11F
:10DBA0000E94EC16882309F452C0C062C09313018E
:10DBB000809106058F5F80931401E6E1F1E0A5E610
:10DBC000B7E090E06DE0911729F14D915D91649F70
:10DBD0009001659F300D112485E0359527958A9534
:10DBE000E1F73E5F37FD06C02F3F83E038072CF496
:10DBF000822F05C080E030E002C08FEF33E0EF01FC
:10DC00002197292F220F220F232B288380839F5FA8
:10DC10003296D9CFC3E1D1E089910E948A6D81E02B
:10DC2000C132D807C9F7E0912501F0912601108291
:10DC300031978FEF80838CE99CE09093240180934F
:10DC40002301DF91CF911F910895CF77A4CFCF7D8E
:10DC5000ADCF1F920F920FB60F9211240BB60F92F9
:10DC60002F938F939F93EF93FF9388B391E089272E
:10DC700088BBE0912301F09124012191F0932401CC
:10DC8000E0932301822F90E097BD86BD293C08F0E8
:10DC9000C09A80919B0C816080939B0CFF91EF91C7
:10DCA0009F918F912F910F900BBE0F900FBE0F90F1
:10DCB0001F9018951F920F920FB60F9211240BB65A
:10DCC0000F922F933F938F939F93EF93FF9388B37C
:10DCD00091E0892788BBE0912501F09126018081A0
:10DCE00028B539B580FD03C0205E3F4F02C0205FDC
:10DCF0003F4F39BD28BD90E095958795009791F4E9
:10DD0000CF01019690932601809325018181811195
:10DD10000AC080917800909179008053984F99BD06
:10DD200088BD01C0808380919B0C816080939B0C97
:10DD3000FF91EF919F918F913F912F910F900BBE8B
:10DD40000F900FBE0F901F901895EDE7F0E08081C7
:10DD5000857E808317981F9AAAE8B0E01C921092E3
:10DD60008B0082E88C938081806280830895EDE748
:10DD7000F0E080818F7D8083179AAAE8B0E01C9242
:10DD800010928B008AE08C93808188618083089553
:10DD90001F920F920FB60F9211240BB60F928F9312
:10DDA0009F93EF93FF9380912C0D882321F01F9A6E
:10DDB00010922C0D04C01F9881E080932C0DE091EF
:10DDC0001101F091120180819181909387008093DD
:10DDD00086008091970C9091980C90938500809389
:10DDE000840082819381892B11F0329607C0809143
:10DDF000FF01817080932C0DE4EEFCE0F0931201A2
:10DE0000E093110180919B0C816080939B0CFF91AA
:10DE1000EF919F918F910F900BBE0F900FBE0F90BF
:10DE20001F901895E0E9FCE0208126952695282B87
:10DE3000208381818F5F8183843048F0A281B38108
:10DE4000CD010196938382832C93108211820895D1
:10DE5000882339F08091960C8F5F8093960C80E830
:10DE600003C01092960C80EC0E94126F8091960C69
:10DE70008530B8F70895CF93DF93C82FE091940CC5
:10DE8000E827F0E0EE0FFF1FE157F34E25913491A4
:10DE90004091950C50E0242735273093950C209322
:10DEA000940CD8E08C2F80780E94286FCC0FD15032
:10DEB000C9F7DF91CF910895CF9380EC0E94126F44
:10DEC000C6E080E80E94126FC150D9F780ECCF9174
:10DED0000C94126FE82FF0E0EE0FFF1FEB59F84F94
:10DEE00020813181C901880F991F820F931F97FDEF
:10DEF000039695958795959587958653974F0895A1
:10DF0000FF920F931F93CF93DF93C091F8018091FD
:10DF1000250585FF04C08091E5018111C4E0809151
:10DF20009A0C8C1709F48EC0C0939A0C1EBC1DBCB1
:10DF30001CBC87B7837C87BF80917D008E7F8093D8
:10DF40007D008CE386BF8FE380937C00C23079F143
:10DF500018F4C130A1F006C0C33009F444C0C43085
:10DF600009F45DC00E94A56E80E49CE99BBD8ABD5A
:10DF700087B7806187BF1FBC8AE08EBD63C00E94E7
:10DF8000A56E80E797E199BD88BD80EA9FE09093F8
:10DF900079008093780087B7886087BF80917D0083
:10DFA000816080937D001FBC82E08EBD56C00E94C0
:10DFB000A56E88EC90E090937900809378008CE2D5
:10DFC00091E09DBD8CBD80EE9BEA97BD86BD87B775
:10DFD000806287BF80917D00816080937D001FBC3F
:10DFE0008AE18EBD9DC080E49CE99BBD8ABD87B758
:10DFF000806187BF1FBC8AE08EBD83E00E940C6DEC
:10E0000080E593EC909387008093860088E893E105
:10E0100090938500809384000E94B76E8AC084E04C
:10E020000E940C6D80E593EC9093870080938600AE
:10E0300088E893E190938500809384000E94B76EF6
:10E04000C0987FC0C13049F008F473C0C23009F4F1
:10E0500067C0C33009F46DC074C07894E0E9FCE097
:10E060008CE99CE090932601809325019383828321
:10E07000158214821082118216820E945C6F809138
:10E08000F9010E943B6F8091990C0E943B6F80E0E8
:10E090000E943B6F1092990C10E0812F0E946A6FD2
:10E0A000F82E092F81E0810F0E946A6FEC018F2DFD
:10E0B0000E943B6F0F708C2F8295807F802B0E9477
:10E0C0003B6FCE0174E0969587957A95E1F70E94B3
:10E0D0003B6F1E5F183009F7C091940C8091950C2E
:10E0E0000E943B6F8C2F0E943B6F0E945C6F80915F
:10E0F000910C882321F080E00E94126FF8CFE0910C
:10E10000920CF091930C108280917800909179009C
:10E11000805C93469093790080937800C09A11C0F8
:10E12000789486E0DF91CF911F910F91FF900C942E
:10E13000A86D80E0DF91CF911F910F91FF900C941B
:10E140000C6DDF91CF911F910F91FF9008951F9259
:10E150000F920FB60F9211240BB60F922F933F938D
:10E160004F935F936F937F938F939F93AF93BF93DF
:10E17000CF93DF93EF93FF938CB59DB520912D0D39
:10E18000222321F0C09A10922D0D04C0C09821E0E6
:10E1900020932D0DC0912101D0912201FE012191EA
:10E1A00031913BBD2ABDF0932201E0932101EFE0C4
:10E1B000F1E0282F3181381708F48183308123174B
:10E1C00008F480838A819B81892BD9F48CE99CE0B7
:10E1D00090932201809321018091FF0180958170AD
:10E1E00080932D0D87B78F7E87BF0E94806F8091AF
:10E1F000F801882311F0833021F487B7806187BF4D
:10E20000789480919B0C816080939B0CFF91EF919F
:10E21000DF91CF91BF91AF919F918F917F916F913E
:10E220005F914F913F912F910F900BBE0F900FBEBA
:10E230000F901F9018951F920F920FB60F921124F6
:10E240000BB60F922F933F934F935F936F937F93F0
:10E250008F939F93AF93BF93EF93FF938091F801B8
:10E260008230C1F480E492EA97BD86BD8091780047
:10E27000909179008F3F910538F488E598E9909363
:10E2800079008093780008C088EC90E09093790042
:10E29000809378000E94806FFF91EF91BF91AF91C2
:10E2A0009F918F917F916F915F914F913F912F91AE
:10E2B0000F900BBE0F900FBE0F901F9018951F92DE
:10E2C0000F920FB60F9211240BB60F922F933F931C
:10E2D0004F935F936F937F938F939F93AF93BF936E
:10E2E000EF93FF938091F801789490919A0C98178E
:10E2F00071F0943061F48091E501882321F08091E0
:10E30000250585FD03C00E94806F03C084E00E9444
:10E310000C6DFF91EF91BF91AF919F918F917F9184
:10E320006F915F914F913F912F910F900BBE0F9086
:10E330000FBE0F901F901895FC01A5E6B0E08C91E0
:10E340008B7F8C93148215821082118216A617A6D9
:10E3500008950C949C7121E0FC018481811101C01D
:10E3600020E0822F0895FC0121818081281B2770E5
:10E3700098E0921B81E0933008F480E00895CF93F9
:10E38000DF93FC0184818823F1F0815084838281B2
:10E390009381890F828386A58823F1F187A59FEF5A
:10E3A000980F97A7882331F080916500846080934F
:10E3B000650032C0809165008B7F809365008091FD
:10E3C000270587A729C01B98809165008B7F8093C4
:10E3D00065008581882319F0815085831DC0808167
:10E3E00091818917C9F090E0EF01C80FD91F2E81E4
:10E3F00022832E8924832E8523832E8D258328A98D
:10E4000026A717A62EA13FEF320F3EA3211104C06D
:10E410000196877099278083DF91CF910895EF92BD
:10E42000FF920F931F93CF93DF93EC01F62E142FDF
:10E43000E22E0E94B371882309F44FC080911C051D
:10E44000887309F44AC0302F32953695369533706B
:10E45000402F4F70333009F43FEFFF2021F09091AF
:10E460002605965FF90E803129F48BEA189F112D4D
:10E47000112402C0883111F4169509C0883211F4B4
:10E48000110F05C0803319F4812F880F180F2881D0
:10E4900004FF0DC0FA821C83ED8205FB882780F9FA
:10E4A0008EA71FA63B8329834423B9F001C04F5F89
:10E4B000E981F0E0CF01019687709927281769F06C
:10E4C000EC0FFD1FF682168BE68E05FB002700F988
:10E4D00000AB415046A336878983DF91CF911F91CE
:10E4E0000F91FF90EF9008950F931F93CF93DF93B9
:10E4F000EC01062F642F80911C05869586958695E4
:10E50000877038812981321300C110E00332110570
:10E5100008F0FBC0F801ED58FF4F0C94FC7A00E3C3
:10E520002AC000E321E0CFC002EA22E04AE064E62C
:10E53000E9C00AE222E045E06FE5CE010E940F72D9
:10E5400001E22AE045E06FE5CE010E940F720AE287
:10E5500022E045E06FE5D6C002EC23E04AE060E54A
:10E56000CE010E940F7202E423E04AE06CE3CE0188
:10E570000E940F7200E221E06FC001E221E045E05D
:10E5800066E4CE010E940F7222E04FE062E3CE010A
:10E590000E940F7222E04FE06BC002E221E045E0F2
:10E5A0006EE6CE010E940F7203E221E045E09FC0BB
:10E5B00000E025E045E062E3CE010E940F7225E015
:10E5C00045E06AE5CE010E940F7202E024E043E0DC
:10E5D0006EE698C003E22AE045E060E5CE010E94C5
:10E5E0000F7201E224E145E060E5CE010E940F7266
:10E5F00003E22AE045E03CC002E625E044E16AE0AF
:10E6000081C002E22AE044E062E3CE010E940F7280
:10E6100001E224E148E066E4CE010E940F7202E2CA
:10E620002AE048E062E3CE010E940F7201E224E199
:10E6300044E04EC00AE22AE002C002E222E345E0E2
:10E640004CC001E203C002E201C003E22AE044E15F
:10E6500060E058C002E122E04AE03AC002E423E070
:10E6600044E16CE3CE010E940F7202EE23E044E12C
:10E6700060E548C000E321E048E22AC0813009F4A7
:10E6800044C000E121E04AE06BE43CC08130E9F1A4
:10E6900000E121E04AE061E435C000E121E046E02C
:10E6A00031C000E3D8CF813081F100E1D4CF00E167
:10E6B00012C003E303C002E301C001E323E04FE023
:10E6C0000CC001E329E144E103C000E321E04EE195
:10E6D00066E418C001E321E04AE068E713C002E302
:10E6E00021E04AE06AE70EC003E321E04AE06CE77C
:10E6F00009C000E520E04AE062E804C000ED20E047
:10E700004AE062E3CE010E940F72DF91CF911F9128
:10E710000F91089546E4682F83E991E00C94747298
:10E720009091280591FF03C0862F0C9433140C940C
:10E730008A73FF920F931F93CF93DF93EC01162FF1
:10E74000F42E47FF03C0842F0E943314D7FF06C066
:10E75000D195C195D1098AE10E943314112371F03A
:10E76000123019F464E670E002C06AE070E0CE0195
:10E770000E94A77A262FC22FD72F082F64E670E0B9
:10E78000CE010E94A77A9B01562F482FC82FD92F60
:10E790002115310551F12A303105DCF06AE070E0D5
:10E7A000C9010E94A77A9B018C01EC0165317105BA
:10E7B0001CF48EE6820F05C08CE8820F0E942E1496
:10E7C0008EE60E9433140115110559F1502F11E006
:10E7D00001C010E084E6850F0E943314111121C09E
:10E7E0002097F9F08C2F845715C08CE8840F0E9475
:10E7F0002E141123B1F0123081F46AE070E0802F02
:10E8000090E00E94A77AC82F86E0860F0E943314FA
:10E810008CE88C0F0E942E1404C086E0800F0E94AA
:10E8200033141F1444F48F2DDF91CF911F910F915A
:10E83000FF900C943314DF91CF911F910F91FF90B3
:10E8400008950895CF93C82F843089F48AE09B01FE
:10E85000829FB001839F700D11248091340E882314
:10E8600091F17093330E6093320EC8E22CC0853064
:10E8700039F58091340E6A30710510F4816001C061
:10E8800083608093340E8091340E81FF05C0CB01EC
:10E890006AE070E00E94937A2091320E3091330E3C
:10E8A000121613062CF044275527461B570B01C0A0
:10E8B000AB01240F351F3093870D2093860D03C0C5
:10E8C000893208F0AFC08091F501EC2FF0E084FDB3
:10E8D00007C0EE0FFF1FE258F24F718360831AC02A
:10E8E000C43059F1EE0FFF1FE258F24F718360837D
:10E8F000C63081F420918A0D30918B0D4AE0429F01
:10E90000C001439F900D11249093870D8093860D35
:10E91000C4E013C0C03279F420918E0422952F7088
:10E920008091BE0D9091BF0D821B91099093BF0DF8
:10E930008093BE0D77C0C930A8F42C2F30E0220F91
:10E94000331FF901E258F24F40815181F901E45936
:10E95000F24F20813181241735070CF047C05183D5
:10E96000408344C0C03139F5462F42954F70842F03
:10E9700090E020915F0D30E08217930754F08530CE
:10E98000910524F026E020935F0D03C04F5F409374
:10E990005F0DFC01E05AF24FCB018F709927982F41
:10E9A0008827672F7727860F971F6AE070E00E94FD
:10E9B000937A608337C0CC30C9F4A091960DB091A2
:10E9C000970D2CE330E00E94697A20919104211187
:10E9D00003C021E02093910430E040E050E00E9429
:10E9E000BB7A3093970D2093960D1CC0C232D1F4A0
:10E9F0008091C00D9091C10D4AE0489F9001499FC0
:10EA0000300D1124260F371F45E1429FC001439F5F
:10EA1000900D11246BE070E00E94937A7093CB0DFF
:10EA20006093CA0DCF9108959091F50193FD42C076
:10EA30009091D30D911105C08E3509F04DC081E044
:10EA400026C08E35E1F38D3521F481E08093D20D1F
:10EA500008952091D20D222321F01092D20D20E6AC
:10EA60008227913079F48A3308F08151803309F498
:10EA700087E2E82FF0E0E157F14EE491E093D10D09
:10EA800082E005C0923031F48093D00D83E0809312
:10EA9000D30D0895682F70E0762F66278091D00DF2
:10EAA000680F711D8091D10D8F770E942274109292
:10EAB000D30D08959091080E903518F48093D00DE1
:10EAC0000895682F70E0762F66278091D00D680F2B
:10EAD000711D84E00C94227408951F920F920FB65A
:10EAE0000F9211240BB60F928F939F93EF93FF9386
:10EAF000EAE0FEE08389882359F08150838B848982
:10EB000091E0980F948BE80FF11D80818CB901C0C2
:10EB10005598FF91EF919F918F910F900BBE0F90A1
:10EB20000FBE0F901F9018959EE790930A0E80934A
:10EB30000B0EECE0FEE083E8860F8230A0F082E06E
:10EB40006083E1E0E80FF0E0E65FF14F408321836E
:10EB5000128213821482158216829EE79783875F42
:10EB600080931D0E089560528DE78083319683E077
:10EB7000E7CFFC018181848310820895FC018581A7
:10EB80009681860F911D9683858320915C0D20319F
:10EB900010F124E0959587952A95E1F781832481EA
:10EBA000281710F4821B01C080E08083A42FB0E0FE
:10EBB000AA0FBB1FA258B24F90E08D939C93838104
:10EBC000861708F463838281882311F0681708F49C
:10EBD0006283168215820895FF920F931F93CF933D
:10EBE000DF93EC0188818D3F78F4893F98F4863F6C
:10EBF00009F448C0873F09F05CC089818093E30D28
:10EC00008B818093E10D55C08D3F09F442C08E3F4A
:10EC1000A1F04FC090E0895F9109FC01EE0FFF1F4A
:10EC2000E80FF91FEC52F24F898182838A8181704B
:10EC300081838B81837080833CC080915C0D8F5F6A
:10EC400080935C0D40E069818CEE9DE00E94BE7572
:10EC500041E06A8183EF9DE00E94BE7542E06B81D6
:10EC60008AEF9DE00E94BE756C81669543E081E06D
:10EC70009EE00E94BE7580915C0D8031D0F01092B4
:10EC80005C0D17C089818093E20D8B818093E00D2C
:10EC900010C0198117701D5F239603E03AE5F32E2B
:10ECA000011738F489910E941475F092080E0F5FD5
:10ECB000F7CF83E28093090EDF91CF911F910F91DF
:10ECC000FF9008951F920F920FB60F9211240BB66A
:10ECD0000F922F933F934F935F936F937F938F93F5
:10ECE0009F93AF93BF93EF93FF93579878949BB103
:10ECF0008CB19C7119F01092360E80C09091350E37
:10ED00009230D9F030F4992309F440C0913049F0A1
:10ED100075C0943009F446C030F1953009F44AC00A
:10ED20006DC08E3709F46AC092E09093350EE09181
:10ED3000360EE33108F062C00DC08D3711F483E068
:10ED40002AC08E3729F48FE19EE00E94EC7554C0F2
:10ED5000E091360E91E09E0F9093360EF0E0E15E6A
:10ED6000F14F80834BC092E09093350EE091360EC8
:10ED7000E33108F043C091E09E0F9093360EF0E02F
:10ED8000E15EF14F90E29827908338C08E3731F4DE
:10ED90001092360E81E08093350E30C08B3171F5C4
:10EDA00084E0F9CF95E09093350E80935B0D10923F
:10EDB0005A0D24C090915A0D91110CC0982F9F7339
:10EDC00049F494B3906C94BB25B3982F907C2F7327
:10EDD000922B95BB90915A0D913019F48093CE01EE
:10EDE00004C0923011F48093D3019F5F90935A0D29
:10EDF00080915B0D981302C01092350EF894579ACB
:10EE0000FF91EF91BF91AF919F918F917F916F9102
:10EE10005F914F913F912F910F900BBE0F900FBEBE
:10EE20000F901F901895ECEEFDE012821382118670
:10EE30001286108A118A178A108E10929B0D1092DA
:10EE40009A0D10929D0D10929C0D1092C50D10926E
:10EE5000C40D10925E0D10925D0D1092C70D1092B0
:10EE6000C60D08958CE0E4EDFDE0DF011D928A956A
:10EE7000E9F70E941377109818981092900087E68F
:10EE800089B959981AB886E0809395005F9B02C0B3
:10EE90008CB1FCCF10921D0E539A559A549A579AE2
:10EEA0000895E4EEFDE09091EC0D882319F034967E
:10EEB0009091F30D22813381290F311D33832283F9
:10EEC000408151814217530778F4241B350B33835B
:10EED000228390E0880F991F8656924FFC01808113
:10EEE000918101969183808308958091090E8823F2
:10EEF00049F081508093090E811104C01092850D54
:10EF00001092840D8091080E882319F0815080930F
:10EF1000080E2091590D222309F47AC08091580DD2
:10EF2000882321F081508093580D72C080911D0E6E
:10EF300081116EC091E0392F322321F48F5F990F38
:10EF40008730C9F7909592239093590D843008F03B
:10EF500041C0982F969521E0622F691B982F9170E0
:10EF6000922720911F0570E027FD13C0FB01EE0FD3
:10EF7000FF1FEE0FFF1FE757FB4F20812F7030E080
:10EF8000492F440F02C0359527954A95E2F7237023
:10EF900001C020E0FB01EE0FFF1FEE0FFF1FE75740
:10EFA000FB4F40814295437050E0092E02C05595B9
:10EFB00047950A94E2F74170660F771F660F771F37
:10EFC00067517E4F690F711DFB01E256FD4F608155
:10EFD000875016C0863070F48170282F30E0D90138
:10EFE000A052B24FF901EE51F24F2C9140E06081F6
:10EFF0008A5006C0863061F420E040E060E081EF96
:10F000000E94947585E08093580D10921E0E559ABB
:10F010008091090E882381F080918904807C803C56
:10F0200019F480E00E94517780918D04807C803CAF
:10F0300019F481E00E9451778091080E8823E1F055
:10F040008091BE0D9091BF0D20915D0D30915E0DB0
:10F05000820F931F81312EE0920750F080519E4025
:10F06000E6ECFDE0208131812F5F3F4F318320832B
:10F0700090935E0D80935D0D0895CF92DF92EF9295
:10F08000FF9210925F0D8091590D8F608093590D02
:10F090002091860430E040E050E060E4C62E6EE748
:10F0A000D62E65E0E62EF12CC701B6010E94DD7A6E
:10F0B0003093E50D2093E40D20918A0430E040E088
:10F0C00050E0C701B6010E94DD7A3093E90D20932C
:10F0D000E80DFF90EF90DF90CF90089586B3809574
:10F0E0008E7708958FEF8ABB1BBA91E897BB9EE796
:10F0F00098BB9EE394BB91EC95BB11BA82BB88E0B0
:10F1000082B987EF83B9109261001092620084E1A6
:10F11000809364008BEF809365000E94AB670E9430
:10F12000327780E487B985E886B987E083BF8CE9C8
:10F1300081BF82E085BD87B7836487BF1FBC8AE03B
:10F140008EBD10928B0082E880938A0080917D00B2
:10F15000806280937D00789481E294E490936301CF
:10F160008093620189E10E94D2670E940B5FD09078
:10F1700006050E946E78C0E081FD05C08695CF5FD0
:10F18000C730D1F71FC0C630E9F08C2F0E94755EE2
:10F190008823C1F0C09306058C2F0E94785E81E021
:10F1A0000E94715F0E940B6424E04DEA51E060E030
:10F1B00086E10E94236588E10E9460120E94E56753
:10F1C0000E942B120E94E16781E0809352010E940D
:10F1D0002F18109252010E94361480911F0584FF4F
:10F1E00005C080911C0582FD4FC044C08091280558
:10F1F000882321F06CE187E00E9490730E940E1832
:10F200000E940B6420E046E753E060E080E00E944B
:10F2100016648091250584FD08C000E12AE04AE2D9
:10F2200055E068E380E00E94ED640E94E5670E947B
:10F23000E1670E942B120E94900F0E9423158C01FF
:10F24000F894C0915F0CD091600C7894C057DE4F59
:10F250000E94E5670E940E180E94900F0E942315DD
:10F260007C010E946E788111BCCFE016F10609F492
:10F2700006C1B7CF0E948460883C910528F460E005
:10F280008EE991E00E940E1B0E94900F80911C0558
:10F2900080FD3DC080911D05817012E0181B0E9409
:10F2A000900FE12FF0E0EE0FFF1FE752FB4F21819F
:10F2B000328180911F0580FF06C03195219531096B
:10F2C000458D568D02C047855089241B350BE901B9
:10F2D0006096812F0E943D15C817D907C4F46FE8C6
:10F2E00071E08DE791E00E9432120E94E5670E9472
:10F2F0002B120E94900F0E940E18812F0E943D1524
:10F30000C817D90724F40E946E78882391F3D0910E
:10F31000340580911C0581FD5AC08D2F887388307B
:10F3200041F0803131F0803221F0D77CD860D09329
:10F33000340501E016E1C0E0812F0E94C368CC0FC4
:10F34000C82B11501E30C1F71C2F1D2767E671E036
:10F350008AE694E10E94321210FF04C060E082E06D
:10F360000E94541211FF04C063E087E10E9454120E
:10F3700012FF04C066E08CE20E945412812F887351
:10F3800071F0C3FF02C069E007C0C4FF02C06CE0B7
:10F3900003C0C5FF04C06FE081E40E94541216FF51
:10F3A00004C062E186E50E94541217FF04C065E1C3
:10F3B0008BE60E9454120E94E56701110E942B12F5
:10F3C000CD1729F00E946E78882309F463C08091DC
:10F3D0001C05887B29F460E087E591E00E940E1B04
:10F3E00080919201882351F060E08CE291E00E94CC
:10F3F0000E1B809192018E7F809392010E942B12AE
:10F4000080EF90E090930101809300018091F301DF
:10F410000E942E140E94806F2DE088E190E00FB6CC
:10F42000F894A89581BD0FBE21BD60E085E697E008
:10F430000E94453B86E495E39093650180936401C7
:10F440000E94E16780910605D81629F081E00E94AC
:10F45000715F0E9410608091590D80648093590DF6
:10F4600080ED97E09BBD8ABD80E186BF81E08093FF
:10F47000E60187B7806187BF0E94B11BFDCFF8947A
:10F4800080915F0C9091600C7894C817D90709F0AF
:10F49000DFCEA7CE0E940E1800E04CCF83E991E0AA
:10F4A0000C94A9710E945A7A332312F48A1B9B0B85
:10F4B0000C946B7AA29FB001B39FC001A39F700D03
:10F4C000811D1124911DB29F700D811D1124911D6C
:10F4D00008950E945A7AB7FF0895821B930B0895EE
:10F4E0000E945A7AA59F900DB49F900DA49F800D05
:10F4F000911D11240895B7FF0C94707A0E94707AC0
:10F50000821B930B0895DB018F939F930E94707A67
:10F51000BF91AF91A29F800D911DA39F900DB29FAF
:10F52000900D11240895AA1BBB1B51E107C0AA1F0F
:10F53000BB1FA617B70710F0A61BB70B881F991F94
:10F540005A95A9F780959095BC01CD01089597FB38
:10F55000072E16F4009407D077FD09D00E94937A05
:10F5600007FC05D03EF4909581959F4F08957095C6
:10F5700061957F4F0895A1E21A2EAA1BBB1BFD01C6
:10F580000DC0AA1FBB1FEE1FFF1FA217B307E40782
:10F59000F50720F0A21BB30BE40BF50B661F771FDA
:10F5A000881F991F1A9469F76095709580959095BA
:10F5B0009B01AC01BD01CF010895052E97FB1EF400
:10F5C00000940E94F47A57FD07D00E94BB7A07FC92
:10F5D00003D04EF40C94F47A5095409530952195D3
:10F5E0003F4F4F4F5F4F089590958095709561956F
:10F5F0007F4F8F4F9F4F0895EE0FFF1F0590F4919F
:10F60000E02D09940790F691E02D0994FB01DC01AF
:10F610004150504048F005900D920020C9F701C0BC
:10F620001D9241505040E0F708956817790768F43B
:10F63000FB01DC01E40FF51FA40FB51F02C002900F
:10F640000E9241505040D8F708950C943E7BDC0157
:10F6500001C06D9341505040E0F70895DC01CB01AB
:10F66000FC01E199FECF06C0FFBBEEBBE09A3196EC
:10F670000DB20D9241505040B8F70895FB01DC01E6
:10F6800002C001900D9241505040D8F70895F8946F
:02F69000FFCFAA
:10F69200F0004ACB03CC03CD03CE0364000A02FF81
:10F6A20000E40CFF0000AA05FF09FF0DFF1354142C
:10F6B200AA9C0C9C0C9C0C9CEC1E465A50463C4648
:10F6C20064645A505A64E2F10032649CCE0032649F
:00000001FF
